:020000022000DC
:106000000000042079A80200BD8F06005991060007
:10601000BD8F0600BD8F0600BD8F0600000000008A
:10602000000000000000000000000000BD8F06001E
:10603000BD8F060000000000BD8F0600BD8F06006A
:106040006DA70200BD8F0600E9AB0200BDAA0200E9
:10605000CDAA0200BD8F060001830200BD8F06009D
:10606000BD8F0600C9AB0200D9AB020049A80200EF
:10607000BD8F0600BD8F0600BD8F0600BD8F0600D8
:1060800021B2020059A80200BD8F0600BD8F060094
:10609000BD8F0600BD8F06002DAB0200BD8F060030
:1060A000BD8F0600BD8F0600BD8F0600BD8F0600A8
:1060B000BD8F0600BD8F060000000000000000003C
:1060C000BD8F0600BD8F0600BD8F0600DDAA020051
:1060D00069A80200BD8F0600BD8F060009AC020052
:1060E000F9AB0200BD8F0600BD8F060005AB0200B4
:0860F00000000000BD8F060056
:1070000040F8044B40F8045B40F8046B40F8047B04
:1070100040F8048B40F8049B40F804AB40F804BBF4
:1070200040F804CB40F804DB6846704781F000412B
:1070300002E000BF83F0004330B54FEA41044FEA5D
:10704000430594EA050F08BF90EA020F1FBF54EAF8
:10705000000C55EA020C7FEA645C7FEA655C00F094
:10706000E2804FEA5454D4EB5555B8BF6D420CDD65
:107070002C4480EA020281EA030382EA000083EAE8
:10708000010180EA020281EA0303362D88BF30BD88
:1070900011F0004F4FEA01314FF4801C4CEA1131DE
:1070A00002D0404261EB410113F0004F4FEA03333D
:1070B0004CEA133302D0524263EB430394EA050FC8
:1070C00000F0A780A4F10104D5F1200E0DDB02FA37
:1070D0000EFC22FA05F2801841F1000103FA0EF2CB
:1070E000801843FA05F359410EE0A5F120050EF191
:1070F000200E012A03FA0EFC28BF4CF0020C43FAC2
:1071000005F3C01851EBE37101F0004507D54FF0CE
:10711000000EDCF1000C7EEB00006EEB0101B1F51E
:10712000801F1BD3B1F5001F0CD349085FEA300064
:107130004FEA3C0C04F101044FEA445212F5800F6F
:1071400080F09A80BCF1004F08BF5FEA500C50F10C
:10715000000041EB045141EA050130BD5FEA4C0CEF
:10716000404141EB0101013C28BFB1F5801FE9D24C
:1071700091F0000F04BF01460020B1FA81F308BF6F
:107180002033A3F10B03B3F120020CDA0C3208DD3B
:1071900002F1140CC2F10C0201FA0CF021FA02F116
:1071A0000CE002F11402D8BFC2F1200C01FA02F186
:1071B00020FA0CFCDCBF41EA0C019040E41AA2BFAB
:1071C00001EB0451294330BD6FEA04041F3C1CDA73
:1071D0000C340EDC04F11404C4F1200220FA04F093
:1071E00001FA02F340EA030021FA04F345EA03013D
:1071F00030BDC4F10C04C4F1200220FA02F001FAFF
:1072000004F340EA0300294630BD21FA04F0294680
:1072100030BD94F0000F83F4801306BF81F4801119
:107220000134013D4EE77FEA645C18BF7FEA655C8C
:1072300029D094EA050F08BF90EA020F05D054EA5E
:10724000000C04BF1946104630BD91EA030F1EBF63
:107250000021002030BD5FEA545C05D14000494167
:1072600028BF41F0004130BD14F580043CBF01F55A
:10727000801130BD01F0004545F0FE4141F4700140
:107280004FF0000030BD7FEA645C1ABF194610461B
:107290007FEA655C1CBF0B46024650EA013406BF1C
:1072A00052EA033591EA030F41F4002130BD00BFDB
:1072B00090F0000F04BF0021704730B54FF4806498
:1072C00004F132044FF000054FF0000150E700BF19
:1072D00090F0000F04BF0021704730B54FF4806478
:1072E00004F1320410F0004548BF40424FF0000165
:1072F0003EE700BF42004FEAE2014FEA31014FEAA8
:1073000002701FBF12F07F4393F07F4F81F06051F6
:10731000704732F07F4208BF704793F07F4F04BF41
:1073200041F40021704730B54FF4607401F000451E
:1073300021F000411CE700BF50EA010208BF70477E
:1073400030B54FF000050AE050EA010208BF70476F
:1073500030B511F0004502D5404261EB41014FF4D8
:10736000806404F132045FEA915C3FF4D8AE4FF0E0
:1073700003025FEADC0C18BF03325FEADC0C18BFC3
:10738000033202EBDC02C2F1200300FA03FC20FA14
:1073900002F001FA03FE40EA0E0021FA02F1144461
:1073A000BDE600BF4FEA4102B2F1E04324BFB3F5AE
:1073B000001CDCF1FE5C0DD901F0004C4FEAC0026C
:1073C0004CEA5070B2F1004F40EB830008BF20F050
:1073D0000100704711F0804F21D113F13872BCBF0A
:1073E00001F00040704741F480114FEA5252C2F15F
:1073F0001802C2F1200C10FA0CF320FA02F018BFA8
:1074000040F001004FEAC1234FEAD32303FA0CFCFA
:1074100040EA0C0023FA02F34FEA4303CCE77FEA89
:10742000625307D150EA01331EBF4FF0FE4040F4D3
:107430004000704701F0004040F0FE4040F4000082
:10744000704700BF80F0004002E000BF81F00041C3
:1074500042001FBF5FEA410392EA030F7FEA226CFA
:107460007FEA236C6AD04FEA1262D2EB1363C1BF8A
:10747000D218414048404140B8BF5B42192B88BFF9
:10748000704710F0004F40F4000020F07F4018BF1C
:10749000404211F0004F41F4000121F07F4118BF3C
:1074A000494292EA030F3FD0A2F1010241FA03FCE4
:1074B00010EB0C00C3F1200301FA03F100F00043CC
:1074C00002D5494260EB4000B0F5000F13D3B0F194
:1074D000807F06D340084FEA310102F10102FE2A03
:1074E00051D2B1F1004F40EBC25008BF20F0010073
:1074F00040EA03007047490040EB0000013A28BF12
:10750000B0F5000FEDD2B0FA80FCACF1080CB2EB94
:107510000C0200FA0CF0AABF00EBC2505242184312
:10752000BCBFD0401843704792F0000F81F40001B7
:1075300006BF80F400000132013BB5E74FEA41038A
:107540007FEA226C18BF7FEA236C21D092EA030FF6
:1075500004D092F0000F08BF0846704790EA010F70
:107560001CBF0020704712F07F4F04D1400028BF9D
:1075700040F00040704712F100723CBF00F500007F
:10758000704700F0004343F0FE4040F400007047B5
:107590007FEA226216BF08467FEA23630146420261
:1075A00006BF5FEA412390EA010F40F48000704774
:1075B0004FF0000304E000BF10F0004348BF40421A
:1075C0005FEA000C08BF704743F0964301464FF056
:1075D00000001CE050EA010208BF70474FF00003B2
:1075E0000AE000BF50EA010208BF704711F00043F3
:1075F00002D5404261EB41015FEA010C02BF8446C3
:107600000146002043F0B64308BFA3F18053A3F521
:107610000003BCFA8CF2083AA3EBC25310DB01FA68
:1076200002FC634400FA02FCC2F12002BCF1004FEC
:1076300020FA02F243EB020008BF20F0010070477D
:1076400002F1200201FA02FCC2F1200250EA4C00D1
:1076500021FA02F243EB020008BF20EADC70704717
:107660007BB972B90029BEBF00204FF0004106E08F
:1076700008BF00281CBF6FF000414FF0FF3000F042
:107680001DBBADF1080C6DE904CE002909DB002B10
:107690001ADB00F081F8DDF804E0DDE9022304B034
:1076A0007047404261EB4101002B1BDB00F074F896
:1076B000DDF804E0DDE9022304B0404261EB410162
:1076C000524263EB43037047524263EB430300F0C3
:1076D00063F8DDF804E0DDE9022304B0404261EB29
:1076E00041017047524263EB430300F055F8DDF867
:1076F00004E0DDE9022304B0524263EB4303704728
:1077000053B94AB9002908BF00281CBF4FF0FF3108
:107710004FF0FF3000F0D2BAADF1080C6DE904CEA5
:1077200000F03AF8DDF804E0DDE9022304B0704728
:1077300007EE900AF5EEC07AF1EE10FA01D400F0EF
:107740000BB8F1EE677A08B517EE900A00F004F86E
:10775000404261EB410108BDD0B5FFF7CBFD0C4BBA
:10776000002206460F4600F07FF900F0A9FA044611
:10777000FFF79EFD074B002200F076F902460B460C
:1077800030463946FFF756FC00F09AFA2146D0BD44
:107790000000F03D0000F0412DE9F047089D04464F
:1077A0008E46002B4DD18A42944669D9B2FA82F2B4
:1077B00052B101FA02F3C2F1200120FA01F10CFAF0
:1077C00002FC41EA030E94404FEA1C48210CBEFB28
:1077D000F8F61FFA8CF708FB16E341EA034306FBB1
:1077E00007F199420AD91CEB030306F1FF3080F040
:1077F0001F81994240F21C81023E63445B1AA4B28D
:10780000B3FBF8F008FB103344EA034400FB07F72E
:10781000A7420AD91CEB040400F1FF3380F00A816F
:10782000A74240F207816444023840EA0640E41B64
:1078300000261DB1D4400023C5E900433146BDE810
:10784000F0878B4209D9002D00F0EF800026C5E9B2
:10785000000130463146BDE8F087B3FA83F6002ECA
:107860004AD18B4202D3824200F2F980841A61EB42
:10787000030301209E46002DE0D0C5E9004EDDE760
:1078800002B9FFDEB2FA82F2002A40F09280A1EB48
:107890000C014FEA1C471FFA8CFE0126200CB1FB9D
:1078A000F7F307FB131140EA01410EFB03F0884296
:1078B00008D91CEB010103F1FF3802D2884200F223
:1078C000CB804346091AA4B2B1FBF7F007FB1011B5
:1078D00044EA01440EFB00FEA64508D91CEB040453
:1078E00000F1FF3102D2A64500F2BB800846A4EBAE
:1078F0000E0440EA03409CE7C6F12007B34022FA99
:1079000007FC4CEA030C20FA07F401FA06F31C43C7
:10791000F9404FEA1C4900FA06F3B1FBF9F8200CD4
:107920001FFA8CFE09FB181140EA014108FB0EF01A
:10793000884202FA06F20BD91CEB010108F1FF3A6A
:1079400080F08880884240F28580A8F10208614476
:10795000091AA4B2B1FBF9F009FB101144EA014184
:1079600000FB0EFE8E4508D91CEB010100F1FF342F
:107970006CD28E456AD90238614440EA0840A0FBC7
:107980000294A1EB0E01A142C846A64656D353D09D
:107990005DB1B3EB080261EB0E0101FA07F722FAC1
:1079A00006F3F1401F43C5E9007100263146BDE8EA
:1079B000F087C2F12003D8400CFA02FC21FA03F34D
:1079C000914001434FEA1C471FFA8CFEB3FBF7F0CE
:1079D00007FB10360B0C43EA064300FB0EF69E42F3
:1079E00004FA02F408D91CEB030300F1FF382FD28C
:1079F0009E422DD9023863449B1B89B2B3FBF7F634
:107A000007FB163341EA034106FB0EF38B4208D90C
:107A10001CEB010106F1FF3816D28B4214D9023E4D
:107A20006144C91A46EA004638E72E46284605E76B
:107A30000646E3E61846F8E64B45A9D2B9EB02083C
:107A400064EB0C0E0138A3E74646EAE7204694E7CC
:107A50004046D1E7D0467BE7023B614432E73046FF
:107A600009E76444023842E770B54FF0FF0C4CF46C
:107A7000E06C1CEA11541DBF1CEA135594EA0C0F6C
:107A800095EA0C0F00F0DEF82C4481EA030621EAA7
:107A90004C5123EA4C5350EA013518BF52EA0335E2
:107AA00041F4801143F4801338D0A0FB02CE4FF094
:107AB0000005E1FB02E506F00042E0FB03E54FF0C4
:107AC0000006E1FB03569CF0000F18BF4EF0010EBC
:107AD000A4F1FF04B6F5007F64F5407404D25FEAB8
:107AE0004E0E6D4146EB060642EAC62141EA55516B
:107AF0004FEAC52040EA5E504FEACE2EB4F1FD0CAD
:107B000088BFBCF5E06F1ED8BEF1004F08BF5FEA2A
:107B1000500E50F1000041EB045170BD06F00046DC
:107B200046EA010140EA020081EA0301B4EB5C0489
:107B3000C2BFD4EB0C0541EA045170BD41F4801181
:107B40004FF0000E013C00F3AB8014F1360FDEBFA6
:107B5000002001F0004170BDC4F10004203C35DA82
:107B60000C341BDC04F11404C4F1200500FA05F305
:107B700020FA04F001FA05F240EA020001F00042A6
:107B800021F0004110EBD37021FA04F642EB06011C
:107B90005EEA430E08BF20EAD37070BDC4F10C0446
:107BA000C4F1200500FA04F320FA05F001FA04F20A
:107BB00040EA020001F0004110EBD37041F10001F6
:107BC0005EEA430E08BF20EAD37070BDC4F1200501
:107BD00000FA05F24EEA020E20FA04F301FA05F269
:107BE00043EA020321FA04F001F0004121FA04F211
:107BF00020EA020000EBD3705EEA430E08BF20EAE1
:107C0000D37070BD94F0000F0FD101F0004640001A
:107C100041EB010111F4801F08BF013CF7D041EA9C
:107C2000060195F0000F18BF704703F000465200A0
:107C300043EB030313F4801F08BF013DF7D043EA71
:107C40000603704794EA0C0F0CEA135518BF95EA27
:107C50000C0F0CD050EA410618BF52EA4306D1D1AE
:107C600081EA030101F000414FF0000070BD50EACD
:107C7000410606BF1046194652EA430619D094EA57
:107C80000C0F02D150EA013613D195EA0C0F05D141
:107C900052EA03361CBF104619460AD181EA030195
:107CA00001F0004141F0FE4141F470014FF000004D
:107CB00070BD41F0FE4141F4780170BD704700BFD6
:107CC0004A0011D212F5001211D20DD56FF478735B
:107CD000B3EB62520ED44FEAC12343F0004343EAB0
:107CE000505323FA02F070474FF00000704750EAFB
:107CF000013002D14FF0FF3070474FF00000704765
:107D000030B5144685B019A3D3E90023FFF7F8FC7A
:107D10000546A5F16150A0F5351001A9A0F56070E8
:107D20003AF05AFE9DF807309DF806200E491B04D4
:107D300043EA42539DF8082043EAC2239DF80920F4
:107D400043EA42139DF80A2043EA5203BDF8042097
:107D500025F00105A2F2BC7243EA4263A5FB0101D2
:107D6000236005B030BD00BF00CA9A3B00CA9A3BF1
:107D700000000000182A2DE9F74F0446C0F8002142
:107D800022D0202A23D0102A24D140F20A43A4F87A
:107D90000431204641F0CEF90022034694F8055103
:107DA000AA4201F1040103F1040315D3364EDFF8B2
:107DB000DCE000EB850394F804210132B5EB820F7F
:107DC0001CD303B0BDE8F08F40F20C63DFE740F650
:107DD0000E03DCE70023DAE711F8045C03F8045C27
:107DE00011F8035C03F8035C11F8025C03F8025C11
:107DF00011F8015C03F8015C0132CFE794F805212A
:107E0000B5FBF2FA02FB1A5913F8041C13F8038CA1
:107E100013F802CC13F8017C0192B9F1000F0AD1DA
:107E200016F808B016F80C8016F807C0775C1EF834
:107E30000A108BEA0101D4F80021202A08D1B9F1F7
:107E4000040F01BF715C16F8088016F80CC0F75DCE
:107E5000019AAA1A043310F8229000EB820281EAF8
:107E6000090103F8041C517888EA010803F8038C1F
:107E700091788CEA010C03F802CCD278574003F8D1
:107E8000017C013597E700BFA02A0900E02809001E
:107E90002DE9F04FDFF8A0C1614E624FDFF89CE1A1
:107EA000002901DCBDE8F08F436C5F4C1A4684FB6F
:107EB00002825E4CD0F84880254684FB0898A2EBED
:107EC000080252004264584C826C84FB028285FB9B
:107ED000038313445B008364036C554C1A4684FB94
:107EE000028205F1AF6505F5A435D0F84C809F35C9
:107EF00085FB0898A2EB080252000264C26C84FB66
:107F0000028285FB038313445B00C364C36B494C4B
:107F10001A4684FB0282D0F8508086FB0898A2EBB8
:107F200008025200C263026D84FB028286FB038357
:107F300013445B000365836B1A4687FB0282D0F80B
:107F400054808CFB0898A2EB080252008263426DB9
:107F500087FB02828CFB038313445B004365436B06
:107F60001A468EFB0282DFF8D880D0F8589088FB42
:107F700009A9A2EB090252004263826D8EFB0292B4
:107F800088FB039313445B008365036BDFF8B490B5
:107F90001A4689FB0282DFF8B080D0F85CA088FB2B
:107FA0000ABAA2EB0A0252000263C26D89FB02A266
:107FB00088FB039313445B00C365C36ADFF88C90AE
:107FC0001A4689FB0282DFF88880D0F860A088FB1F
:107FD0000ABAA2EB0A025200C262026E89FB02A236
:107FE00088FB039313445B000366836ADFF86490A5
:107FF0001A4689FB0282DFF86080D0F864A088FB13
:108000000ABAA2EB0A0252008262426E89FB02A205
:1080100088FB039313445B004366013948303FE714
:108020004A3FE3D7A740DD7DF053C26DAA0025BECD
:10803000E4EBDC70736E8D797611B7E8B7206D7F55
:108040002FFEE4F3407EE47FC7A3C1FA63B2FC7F56
:10805000C6BD2EFE94C6FF7F5DC286FF2DE9F04FA0
:10806000044685B0084641F065F88A46024603900A
:108070002146002040F077FF231D019304F11003F7
:1080800001260293039A25462146002311F8230076
:10809000334F385C01F823000133042BF6D1019BE8
:1080A00001318B42F1D1617963786170617A6171DC
:1080B000617B6172A17A6373A378A170A17BA372C3
:1080C000A379A171E17BA373E378E170E17AE173B5
:1080D000E179E172E3719AF80431B34239D095F84D
:1080E00000B095F80180AF78E9788BEA080087EA5C
:1080F000010380EA0309039356F08AFE8BEA00002D
:1081000089EA0000287088EA070056F081FE039B88
:1081100088EA000089EA00006870184656F078FE88
:10812000784089EA0000A8708BEA010056F070FEE2
:108130004840029B89EA000985F803900435AB4268
:10814000CDD13046214601360392F6B240F00BFF06
:1081500098E72146304605B0BDE8F04F40F003BF38
:10816000A02A09002DE9F04F594D8146884659480B
:1081700003F0030189B005EB811550F8211001913E
:1081800099101F298C46A8BF4FF01F0C1C290E46C2
:10819000A8BF1C266C68EB680292033626EAE676D6
:1081A00034410594AC680020344133410490069476
:1081B000079359F8046B484B1E4226F0004412D135
:1081C00008AB03EB840454F8103C002E40EA030093
:1081D000B8BF5B4248F8043B029B013B0293E8D1E5
:1081E00009B0BDE8F08F3D4B1E420AD1002955F879
:1081F0002440BABFCCF1000304FA03F344FA0CF3B1
:10820000E3E7374B1E4214D1103C364B019F53F825
:10821000243083FB0747ACF10304002C54DA64429A
:108220006FF0004343FA04FEBE45CEDB07FA04F3C9
:10823000CBE76304B3F1006FB6BF630500240424E9
:10824000B3F1005FBCBF9B000234274F274AB3F154
:10825000804FBCBF5B000134BB4207F14F4707F5BD
:10826000F21707F58267D8BF3A469346204F214A56
:10827000CCBFBE4696469A465A4682FB0ABADEF8FC
:10828000047057449A4687FB0ABADEF808705744D0
:108290009A4687FB0ABADEF80C70574487FB03A3A3
:1082A000154ADEF8107052F8242003923B4417461A
:1082B00083FB07E7FB00019F83FB07E70F4B53F8A6
:1082C0002440ACEB0404A8E747FA04F37DE700BFC1
:1082D000243A090014390900FCFFFF7FF0FFFF7FFB
:1082E000C0FFFF7F643909009979825A63218510A4
:1082F000EC38090000390900443909002439090023
:108300002DE9F04F00248DB0CDE90644634B64485D
:108310006449012225461E6846B1D0F8046316421E
:1083200004D01D601E680396039E144304338B42E1
:108330004FEA4202EFD15A4BD3F87C218AB1002296
:10834000C3F87C21D3F87C310493049B4FF0A04305
:1083500044F00044D3F810350693534BD3F810354E
:108360000793E3B2D3B1514F01260025344210D018
:10837000AB0003F1804303F5C043D3F81005D3F8F5
:10838000101557F8253023B1C1F30141C0F3052082
:1083900098470135082D4FEA4606E7D1002C79DAD7
:1083A0000AAE00230A9373604FF0FF33CDE9083320
:1083B000DFF8F8903E4F0025A84617F9013B5C1CFA
:1083C0004FD0C3F3C20103F00702DCB203F03F0A4F
:1083D0000CAB0B4413F8100CD040C00741D509EB8F
:1083E0000A00A40990F9280059F820B0BBF1000F49
:1083F0000CD1032C35D1012000FA02FC705C40EA5C
:108400000C00705404E04FF00108D6E7032CF2D0C2
:1084100005A80193CDF814A02DF01EFA0599019B33
:1084200001F5E07113F8183C50F82110D340DB0738
:10843000C1F3014105D5022913D1032C0BD12146EB
:1084400004E003290DD1032C05D10221504652F03E
:1084500043F90135EDB2BBF1000F02D02146504681
:10846000D847B8F1000FCED0A5B14FF0A043069980
:10847000D3F8102503F540739142D3F8103502D19B
:108480000799994206D006920A9ACDE907320B9BCA
:1084900009938FE70DB0BDE8F08F00BF0061004089
:1084A0000060004020610040000300502460012073
:1084B0007C6001202DE9F04FB1B00E46099302F522
:1084C0000863049300F13C0303930023CDE90133D7
:1084D000DDF8E8B00592039B019AA3F13C07DBF8B5
:1084E0000030934229DC059B243603EB8203019A7A
:1084F0000493DBF804309342A6F1240500F32081B5
:1085000016460027DBF80830019A934200F30682F2
:108510000022019B1F2B40F35182029B002B00F095
:1085200061820023029A002A80F25782013B304682
:10853000CBF81C3031B0BDE8F08F099BD3E905932F
:1085400033B1DBF81430019A9342C8BF4FF00009F1
:10855000DBE903A3019ADBF818709342C8BF4FF020
:10856000000A049B062FA3F5086306937FDC002511
:108570000398C7F107070DF1500C06F124012B46B3
:1085800082683A41D21A43683B41551B9B1A51F805
:10859000042DCCF824503A41B1424CF804390A6019
:1085A000A0F10800ECD1159B5B1015930C9B0CA857
:1085B0005B100C931CF0D4F815A81CF0D1F859EA04
:1085C0000A0567D1DFF8F0C3DFF8E4A3B646284612
:1085D0000DF15008D8F824305AF8042958F8041935
:1085E00082FB0393A3EBA102DEF8009003EBA1034F
:1085F0004EF8043BC9F100035CF8081B9B1A83FB8F
:10860000014102EB81015CF8042C83FB0242069BD2
:10861000049C43F820106FF003034343C9EB82022C
:10862000E250002381EAE173A3EBE173002182EAC7
:10863000E271A1EBE27120300B43B0F5907F45EA87
:108640000305C7D13B463146019A069840F0B7FC76
:10865000029B284303430293019B01330193049B34
:1086600004330493039B48332436039333E7039B7B
:10867000002014AD0246A3F148079968891A5A6888
:10868000083B081A521ABB42686245F80429F4D123
:10869000002788E70DF1780852463046414602F03F
:1086A000D3FDC24B902000FB09302FAB089300256F
:1086B000BF4B079300F148092A460DF1500A079C69
:1086C000DAF8243054F804C95AF8041907948CFBDA
:1086D00003E3C3EBA10E03EBA10346F8223050F8ED
:1086E00022108EFB0131089C58F8223059F804CD35
:1086F0000B4454F8041908949B008EFB0C4C069C08
:1087000061444FEAC21C890044F80C306FF07F04CA
:1087100004FB02FC049C44F80C104FF0000C83EAAC
:10872000E37CACEBE37C002381EAE173A3EBE17330
:1087300001324CEA0303092A45EA0305BFD181E768
:10874000DBE903A3019A9342C8BF4FF0000ADBF8AC
:108750001830062B00F3DF80C3F10703039329468B
:108760003B4607F148001A68039C22411A605A6888
:1087700022415A6051F8042B08332241834241F8C8
:10878000042CF0D10CA938461CF074F812A9381D3D
:108790001CF070F818A907F108001CF06BF852469D
:1087A0001EA9284602F050FD049A82490020069036
:1087B00002F5C0701EAB0DF130080DF138090B90B9
:1087C00053F8040B0024800080EAE074A4EBE0740A
:1087D00010609868079480004FF0000A80EAE07A01
:1087E000AAEBE07AC2F8800151F8040BD8F80CC06B
:1087F00080FB0CEC586900240CEB800080EAE074EC
:10880000A4EBE074C2F8000388680894D9F80CE07F
:10881000CC46044684FB0E0E186A00240EEB800042
:1088200080EAE074A4EBE074C2F880044869DCF8E4
:1088300000C00994A9F1040980FB0CEC51F8040C68
:10884000D8F824E0044684FB0E0ED86AF4440CEBFE
:108850008000002480EAE074A4EBE074C2F8000613
:10886000D8F800C0086A0A9408F1040880FB0CECF0
:108870008868D9F828E0044684FB0E0E986BF4440F
:108880000CEB80004FF0000C80EAE07CACEBE07C6D
:10889000079CC2F8800744EA0A0A089C0B984AEA37
:1088A000040A099C4AEA040A0A9C4AEA040A069C49
:1088B0004AEA0C0C803244EA0C04824206947FF4AB
:1088C0007FAF129B9B1046F8243C139B9B1046F8ED
:1088D000203C149B9B1046F81C3C18A9A6F11803D9
:1088E00051F8042B921043F8042BB342F8D1039BA8
:1088F000019A0498294640F062FB069B0343184600
:10890000029B03430293019B01330193049B48376D
:1089100024360433EBE50023039333E7DBE9032339
:10892000019928468B42C8BF00221EA902F08CFC88
:10893000019B019A43F3000A059B03EB820105F1B9
:1089400020031EA8A5F1040E4FF0000C02F001094F
:108950001C46026892000A60B84682EAE278A8EBF8
:10896000E27843688AEA83034B441A434CEA020CD8
:10897000C1F880303A4683EAE372A2EBE372029BCD
:108980004EF8047F42EA08021343A645029300F121
:10899000080001F58071DCD1019BBCF1000F18BF0C
:1089A0001E46013324350193ACE500BF6460090025
:1089B000BC37090084610900A4380900059B0199AE
:1089C00003EB8101002341F823202033B3F5107F0E
:1089D000F9D1019B013301939BE5029A52000133C7
:1089E00002929FE52023A1E52DE9F04F04468DB0CA
:1089F000084640F09FFB0D46024607EE900A2146CE
:108A000095F8040140F0AFFA95F80461231D013E8A
:108A1000099304F11003F6B20A93627A637B6273DE
:108A20006279627262786271A27A6370A378A270CE
:108A3000A27BA372A379A271E279A373E378E270B7
:108A4000E27AE271E27BE272E3732546224600237A
:108A500012F823105348415C02F823100133042B11
:108A6000F6D1099B01329342F1D117EE902A2146AB
:108A7000304640F078FA002E00F0918095F800A082
:108A8000EB780793504656F0C3F9029056F0C0F9C0
:108A9000039056F0BDF995F8019095F80280834651
:108AA000484656F0B5F9024656F0B2F9049056F031
:108AB000AFF90746404656F0ABF9059056F0A8F9D5
:108AC000069056F0A5F9079B019018460B9356F0B7
:108AD0009FF9079056F09CF9089056F099F9029B7F
:108AE0001946039B81EA030C8BEA0C0C0499069B44
:108AF00082EA0C0C8BEA02024A4005997A404A400D
:108B000001994A40089987EA0C0C83EA0C0C4A4008
:108B1000019B0599424083EA0C0C8AEA02020B9BF6
:108B200088EA02025A406A70039A82EA0B027A408B
:108B300080EA0C0C4A40069989EA0C0C88EA0C0C75
:108B40004A40019983EA0C0C85F800C04A40079915
:108B50004A4042408AEA020289EA02025340AB706C
:108B6000029B019983EA0B0B049B83EA0B0B87EAB8
:108B70000B07079B79405940089B594048408AEAB7
:108B8000000A89EA0A090A9B88EA090885F803802D
:108B90000435AB427FF472AF013EF6B23DE70DB053
:108BA000BDE8F08FA02909002DE9F04F2DED028BD3
:108BB0000D4608EE103AA9B016468346002801F08B
:108BC000B78509683FF0DCFD031E0493C1F2B4854C
:108BD0002B6803442B60DBF80080B8F1000F0BD149
:108BE000584618EE101A40F0BBFA6FF0060029B094
:108BF000BDEC028BBDE8F08FDBF80470002FEFD0E6
:108C000098F8004098F81C20002C3AD1032A4FF025
:108C100009010CBF4FF011094FF0200920A8CDE940
:108C20002034CDE9224956F080F8386098F81C309D
:108C3000032B0CBF0521032120A856F076F807F17D
:108C4000080A7860DBF8BC379C420CDB4FF0000A66
:108C5000DBF8C4379A4580F2C580902303FB0A7481
:108C6000002305938FE00AF11003012120A805934A
:108C700056F05BF8059B4AF8040B9A45F5D1013490
:108C8000E0E7032A4FF008010CBF4FF009094FF04D
:108C90001109209320A80023CDE92133CDF88C9031
:108CA00056F043F8386098F81C30032B0CBF0121B4
:108CB000022120A856F039F87860C7E70C2120A8D7
:108CC00056F033F80921A06220A856F02EF80821AA
:108CD000E06220A856F029F8206398F80030002BB5
:108CE0000CBF0421092120A856F01FF80121606360
:108CF00020A856F01AF8A063002855D0022120A819
:108D000056F013F80121E06320A856F00EF8052173
:108D1000206420A856F009F80521606420A856F0C8
:108D200004F80023E364A064032120A855F0FDFFAC
:108D30000321206520A855F0F8FF0321606520A8D5
:108D400055F0F3FFE36BA0652BBBC4E90A33636303
:108D5000E36DC3F11403236698F80030002B3FD174
:108D6000012120A855F0E1FF6066012120A855F0FF
:108D7000DCFF0121A06620A855F0D7FF059BE06627
:108D8000013305934834DBF8BC37059A9A4295DBEA
:108D90000AF1010A5CE7022B04D1236C13B9082302
:108DA000E365D5E70723FBE7C4E90F00052120A809
:108DB00055F0BBFF0521606420A855F0B6FF0521E2
:108DC000A06420A855F0B1FF0421E06420A855F06C
:108DD000ACFF0321E06520A855F0A7FF2066BBE7A4
:108DE0000020C1E73B68CBF8D8372B684B442B6099
:108DF000049B03EB090433681B1B3360DBF8B827C3
:108E0000DBF8B03772B1002B59D1DBF8CC273368CF
:108E10009A4264DD584618EE101A40F0A1F94FF05E
:108E2000FF30E4E6002B4AD10123CBF8B037D5F868
:108E30000080D6F800A0A8EB040447465146384607
:108E400040F0A2F9002807EB000324DB395C22780C
:108E500091421BD159786278914217D1A1789A78C2
:108E60004A4012F0FC0F11D18C0748BF03F1FF33C9
:108E7000A3EB0803002BCBF8B4370FDA584618EEF3
:108E8000101A40F06DF96FF00200B0E60330DF1CFD
:108E9000AAEB000AD2E74FF0FF33EBE7049ADBF8C6
:108EA000C8171A441346DBF8C0274B445343DBF87A
:108EB000C427DB004A4393FBF2F3CBF8B837DBF867
:108EC0000030DBF8B4273BB15B69003B18BF0123DE
:108ED0001344CBF8CC3798E74FF0FF33F8E7DBF8D3
:108EE000DC07DBF8D8370BF11C01984209913FDB16
:108EF000C11A1A46099B194418464AF089FC099B75
:108F0000DBF8D807DBF8CC27296818444AF058FC6E
:108F1000DBF8CC17DBF8D8270A44CBF8DC272B6822
:108F20000B442B603368DBF8CC279B1A3360DBF8EB
:108F3000DC37DB000C930BF5FC63149300230593E3
:108F400028230F93002307930493DBF8C437049A74
:108F50009A4281F2F583902353431993059B0A9318
:108F60000F9B1393149B1893002308939A46D7E200
:108F7000099B2968034418464AF022FCDBF8CC1709
:108F8000DBF8DC270A44CBF8DC272B680B442B608A
:108F90003368DBF8CC279B1A584618EE101A33605A
:108FA00040F0DEF86FF0010021E6002D00F0768140
:108FB000DBF804300693002B00F07081DBF80840EA
:108FC000002C00F06B81099B20930023CDE9213315
:108FD000079A0C9B9A18D31D48BF02F10E03DB10B1
:108FE0002393079B1BB1194620A855F09EFE2A78B3
:108FF000002A40F04281049990234B43482101FB11
:109000000A3306990B44A849586B11F8106001EB1C
:1090100040014F78D96B022940F08D80D3F8408011
:10902000B8F1000F0ED00A9B154604EB0308314639
:1090300020A855F07AFE0135082D08F8010BF6D16D
:109040004FF00308089B059A08EB480513441D449C
:1090500025440DF180093146484655F066FE3146FB
:10906000E875484655F061FE31462876484655F089
:109070005CFE08F10108B8F1060F687605F10305FA
:10908000E9D10A9BE5183946484655F04EFE394667
:1090900085F82900484655F048FE394685F82A00EB
:1090A000484655F042FE08F10108B8F10C0F85F86A
:1090B0002B0005F10305E6D1049B7C225A433E2395
:1090C00003FB0A221444002384F83B30A387049A4C
:1090D00090235343482202FB0A33069A1A44936AA8
:1090E000189A1360209A099BD31A229AC2EBC302E2
:1090F000D31002F007020D92079A18980D99C2EB4F
:10910000C3020A4450F8041B1890881A0690099864
:10911000184412900C98002BA0EB02021E9202DB66
:10912000884280F2C380584618EE101A40F018F8B2
:109130006FF007005BE5049BBBB9089B049D1C44D2
:10914000A1460DF180083146404655F0EEFD01354F
:109150000B2D09F8010BF6D13946404655F0E5FDD7
:1091600060550135152DF7D1B1E74FEA0A13069A7C
:10917000083302EB0308D558D5B1089B0599E218CE
:109180000139062312F8010B5054013BFAD1D8F8EB
:109190000430D3B90A9B062504EB0309314620A805
:1091A00055F0C3FD09F8050001350B2DF6D11FE080
:1091B0000A9B04EB0309314620A855F0B6FD0135A2
:1091C000062D09F8010BF6D1E1E7049D3E2303FBD0
:1091D0000AF37C20E21800FB05332344917999714E
:1091E000D179D971117A1972517A5972927A9A7227
:1091F000D8F808302BB3089B05990B3323440B2276
:109200000139013213F8010B5854102AF9D1D8F85A
:109210000C3023B3089B05991033234410220139E5
:10922000013213F8010B5854152AF9D1049B7C2202
:109230005A433E2303FB0A22144400236375A3759B
:1092400045E70A9B0B2504EB0309394620A855F096
:109250006CFD09F805000135102DF6D1D7E70A9B02
:10926000102504EB0308394620A855F05EFD08F8E8
:1092700005000135152DF6D1D8E7089B059A1398FE
:1092800006999A1804F1F80301932B6A009301449C
:109290005346224420A801F08BFE18E7079B0D934C
:1092A0004FF0FF3328E700BF04370900DBF8004028
:1092B000002C00F0D681DBF804300793002B00F07F
:1092C000D081DBF80830002B00F0CB81DBF80C30CC
:1092D0001093002B00F0C581069B002BC0F2C181CA
:1092E000049A616B902353434820079A00FB0A338A
:1092F00013449A6B002A00F03E81DA6B022A40F098
:109300003A811B6C002B40F01E81049A902353433A
:1093100000FB0A30079B18440322C36D013393FB03
:10932000F2F301EB4301B1F92E2002EB42024FF4BC
:109330001071049890234343482000FB0A33079898
:1093400003444FF41069DC6A6300B3F5107FA8BFD3
:109350004FF410739342D4BF21932192109A099332
:1093600002EB8A021C9202F580528B42D4BF2293F8
:1093700022912393099900232093C2F80012109A96
:10938000119309FB0A22199B1B9220AA17924033C2
:109390000D9A0E92C318129A0B921F93179B1C687A
:1093A000119B01331193179B53F8045F17932D1BE7
:1093B000002D40F38682069B002BC0F25281119A49
:1093C0001F9B0B9953F82260BF4B03EBC6031B791D
:1093D0000C930E9B0C985B4213F007031EBF11F811
:1093E000017BC3F1200207FA02F21B9F08BF1A4655
:1093F00007EB8404002840F0D080231D002244F8AD
:10940000202043F8202002308542F7DC90460E9B56
:109410000B9A434402EBE30203F007030E93069B0F
:109420000B92A3EB08030693119B032BB6D1069B6B
:10943000002B40F3C982049A0B99099D9023534352
:10944000482202FB0A33079A1A444FF00009D36EF0
:109450009E4A52F823009E4A52F823600E9B5B42BC
:1094600013F007031EBF11F8014BC3F1200204FAE9
:1094700002F21B9C04EB85040794069CC6F12006AF
:10948000A4EB0305099C0996924EC4F50F74304471
:1094900008BF1A464F4601340C90BC4200F31882B4
:1094A0001C9B03F580530021D3F800020744C3F846
:1094B00000724FF41070109BB7F5107FC7F5107253
:1094C00000FB0A704FEA820203EB8000C8BF002253
:1094D0004AF0B6F9069A0E9B134403F0070207926E
:1094E0000B9A02EBE303199A48321992139A483205
:1094F0001392089A3E3208920A9A3E320A92129ABF
:109500009B1A00F1AE80129A1A4409920D9AC2EB8E
:10951000C303079A13441E9AD31A0C930AF1010A43
:10952000DBF8BC37DBF800509A45FFF63EAD002D66
:1095300040F04E82584618EE101A3FF011FE6FF0C0
:109540000900FFF754BB23785BB9049A9023534377
:1095500000FB0A30079B1844C36D013331F9132017
:10956000E5E6B1F93620B1F93430D31AB1F90C205F
:1095700002EB4302DBE6049B90205843482303FBA5
:109580000A00079B1844C36D006E013331F91320A4
:109590000344013331F91310CBE64F4F57F826C07F
:1095A0004E4F07EB4C0015900698A0EB03080C9863
:1095B000012840F0958037F81C6006F00F064FF048
:1095C000000EC6F12006B8F10F0F53DD0F46C3F1B0
:1095D000180017F802CB49780CFA00F0C3F1100C10
:1095E00001FA0CF101430A431033A8F1100839467F
:1095F00004F1080722FA06F0159C013034F8100037
:10960000040B10F0F00F02FA04F2A3EB103318BFB2
:1096100002F00044C0F3031C1EBF520003F1FF33ED
:1096200044EA0C0C10F4706FC0F303241FBF03F165
:10963000FF3302F000402043520008BF204673452C
:109640000FDB023D002D47E902C03C4637DCA3EBAF
:109650000E039844069BA3EB0808B8F1000F80F2B4
:109660003281584618EE101A3FF07AFD6FF008006C
:10967000FFF7BDBA08EB03000028F2DDB8F1000FD8
:10968000C1BF11F8017BC3F1180C07FA0CF73A437C
:10969000B8F1080FC1BF11F8017BC3F1100307FA3D
:1096A00003F31A434FF00047431E47FA03F31A40EF
:1096B0004FF00B0E00F10B034FF0000898E70A2B58
:1096C00007F1080796DC7EE7C03D0900CC6609007B
:1096D000C4660900D4660900C03E0900403F090085
:1096E0000C98871E012FBCD8B848159F50F836C07B
:1096F000002016900CF101001A90CCF120001D9072
:10970000B8F10F0F2ADD8E46C3F118061EF8029B32
:10971000497809FA06F6C3F1100901FA09F1314353
:109720000A431033A8F1100871460A2BE8DDB7F898
:1097300000E00EF00F0ECEF1200622FA06F60136FA
:1097400037F816605FEA16392FD107EB4607A3EB0F
:109750000E0302FA0EF226463446E6E708EB03064D
:10976000002E7FF77EAFB8F1000FC1BF11F801EBFB
:10977000C3F118090EFA09FE42EA0E02B8F1080F09
:10978000C1BF11F801EBC3F110030EFA03F31A4342
:109790004FF00040731E40FA03F30B201A4016905E
:1097A00006F10B034FF00008BFE7A3EB090302FA31
:1097B00009F2C6F30319B9F10F0FC6F303263746B2
:1097C00027D10C98032827D11A9803EB080E002EF6
:1097D00018BF0130704581463FF743AF9945AEEB66
:1097E000030857DCB8F1000F0ADA73464FF0004067
:1097F0000EF1FF3E40FA0EFE02EA0E024FF00008A4
:109800001D9822FA00F909F10F09A3EB0C0302FAE3
:109810000CF2B9F1000F05D002F0004E4EEA090932
:109820005200013B0F2E22D10C98032844D11A98E4
:1098300003EB080E70453FF714AF1A989842AEEB51
:10984000030831DCB8F1000F09DA0EF1FF364FF0F2
:10985000004040FA06F6734632404FF000081D986B
:1098600022FA00F70F37A3EB0C0302FA0CF227B130
:1098700002F0004637435200013B16988342FFF640
:10988000F0AE2646023D002D46F8089B676015DDC8
:10989000159F61E711F8018BC3F1180008FA00F871
:1098A00042EA0802083399E711F8016BC3F118077F
:1098B000BE4032430833C0E73746D9E7169A9B1AB1
:1098C000C7E64FF00008069B98457FF7A0ADC8E6B5
:1098D0000F2D57DD0E46C3F1180016F802CB49785C
:1098E0000CFA00F0C3F1100C01FA0CF101430A4329
:1098F0001033103D3146079E1036099822FA00FCBD
:109900000C9810F80C004FEA101C02FA0CF210F040
:109910000808A3EB10131FBF02F0004803F1FF3348
:10992000520048F0010810F0040E1FBF02F0004E74
:1099300003F1FF3352004EF0010E10F0020C1FBF76
:1099400002F0004C03F1FF3352004CF0010C10F018
:1099500001001FBF02F0004003F1FF3340F001009F
:1099600052004B45FFF69CAD0437A74246E9048EF2
:1099700046E902C00796BFF690AD092B06F1100626
:10998000BBDC8AE5E81800287FF78AAD002DC1BF4F
:1099900011F8016BC3F1180C06FA0CF63243082DCE
:1099A000C1BF11F8015BC3F1100305FA03F31A43B9
:1099B0004FF00045431E45FA03F31A404FF00A09E1
:1099C00000F10A03002596E7002769E5C03D09007C
:1099D000DBF80470002F3FF4ADADDBF80890B9F16F
:1099E000000F3FF4A7ADDBF80C40002C3FF4A2AD14
:1099F000DBF8101000293FF49DAD01F54673069386
:109A00000F9B00261F44059BCDE9206609EB030A46
:109A100004F59058069B089308F10808DBF8BC375A
:109A20009E42C0F2A5832B6A002B40F0BA832B6ABA
:109A30005A0840F0F4832A6AD30714D504F58053FA
:109A40002E78D3F80012059B3E334B44521020A8C9
:109A5000002E40F02B84CDE90120069A009220468A
:109A60002A463EF0F7FB2B6AA3B120983FF08FFA0D
:109A700004F580540138C4F8080221983FF087FAB1
:109A8000D4E980239342B8BF1346C4E98033013838
:109A9000C4F80C020F9B049A0693902353430024AE
:109AA0004FF012080893DBF8BC379C42C0F20B84DD
:109AB000049ADBF8C847544318EE102A5C4302EBC3
:109AC0004404DBF80C20002A00F02986DBF814207F
:109AD0000A92002A00F02386DBF818200692002A5A
:109AE00000F01D86022B40F08D840A9B1093231DED
:109AF000089300230E9302F500530B930E9B0B9AD1
:109B00000699109803F001030D930A9B03F5805406
:109B10000025D4F8183B0093D2F800220D9B3EF0AC
:109B200085F8D4F81C3B0B9A069910980093D2F84C
:109B300000220D9B803100F510603EF077F80B9B02
:109B40000D99D3F800324FF4886202FB0133069A74
:109B500002EB83094FF0007452F82320D9F85C30EF
:109B60002F46C2FB07456FF07306C3FB06454FF057
:109B70000072D9F88000D9F8DC103B46C0FB0723FF
:109B8000C1FB06234FF45578D9F80400D9F85810D2
:109B9000C0FB0845A6F5D766C1FB0645D9F8840089
:109BA000D9F8D810C0FB0823C1FB062341F6D47EA8
:109BB000D9F80800D9F85410C0FB0E457B4EC1FB04
:109BC0000645D9F88800D9F8D410C0FB0E23C1FB94
:109BD000062346F2B86CD9F80C00D9F85010C0FB37
:109BE0000C45734EC1FB0645D9F88C00D9F8D0104E
:109BF000C0FB0C23C1FB06236E4FD9F81000D9F827
:109C00004C10C0FB07456C4EC1FB0645D9F89000CF
:109C1000D9F8CC10C0FB0723C1FB0623D9F81400E8
:109C2000D9F84810C0FB0C4545F28406C1FB064537
:109C3000D9F89400D9F8C810C0FB0C23C1FB062347
:109C4000D9F81860D9F84410C6FB0E4540F22C77BD
:109C5000C1FB0745D9F89860D9F8C410C6FB0E239C
:109C6000C1FB0723D9F81C60D9F84010C6FB084592
:109C70007427C1FB0745D9F89C60D9F8C010C6FB12
:109C8000082316469846C1FB07680C2720464FF06C
:109C9000140A05FA07F345FA0AF520FA0AF040EA31
:109CA00003003FF07FF9089B23F8040C304608FAC4
:109CB00007F348FA0AF820FA0AF040EA03003FF0F6
:109CC00071F9089B09F5805423F8020C22684FF4BF
:109CD000D0764FF000730025C2FB06354FF00070C0
:109CE000D4F880200021C2FB060141F67C066268A0
:109CF000C2FB0635D4F88420C2FB060149F2FC768B
:109D0000A268C2FB0635D4F88820C2FB06012B4EA0
:109D1000E268C2FB0635D4F88C20C2FB0601284E4F
:109D20002269C2FB0635D4F89020C2FB06016FF011
:109D3000B3066269C2FB0635D4F89420C2FB060163
:109D40004FF41276A269C2FB0635D4F89820C2FB04
:109D500006016FF01306E269C2FB0635D4F89C20B9
:109D60000446C2FB0641184605FA07F245FA0AF511
:109D700020FA0AF040EA02003FF014F9089B9887A5
:109D8000204601FA07F341FA0AF120FA0AF040EA04
:109D900003003FF007F9089BDFF828A0D8870433B9
:109DA0001193089B043B12930EE000BF7CAFFFFFB2
:109DB0003CB6FDFF78940400C44902004CE803005F
:109DC0002464FFFFA4620900DAF840E0D9F800013A
:109DD000D9F85C114FF000730022C0FB0E324FF037
:109DE0000074DAF844500027C0FB0547C5F1000CA9
:109DF000C1FB0C321393C1FB0E47D9F8DC31D9F803
:109E0000801116934FF000754FF00008C1FB0E58FB
:109E1000D9F880014FF0007103460026DAF84400BB
:109E2000C3FB0016169BC3FB0C580B461699C1FBCF
:109E30000E361593DAF848E0D9F804C1D9F858017C
:109E4000139BCCFB0E32DAF84C10CCFB0147C1F16E
:109E5000000CC0FB0C321393C0FB0E47D9F8D8316D
:109E6000D9F884111693C1FB0E58D9F884011599BD
:109E70000346DAF84C00C3FB0016169BC3FB0C58D4
:109E80000B461699C1FB0E361593DAF850E0D9F857
:109E900008C1D9F85401139BCCFB0E32DAF85410E8
:109EA000CCFB0147C1F1000CC0FB0C321393C0FB8B
:109EB0000E47D9F8D431D9F888111693C1FB0E5842
:109EC000D9F8880115990346DAF85400C3FB001647
:109ED000169BC3FB0C580B461699C1FB0E36159307
:109EE000DAF858E0D9F80CC1D9F85001139BCCFB33
:109EF0000E32DAF85C10CCFB0147C1F1000CC0FB5C
:109F00000C321393C0FB0E47D9F8D031D9F88C111D
:109F10001693C1FB0E58D9F88C0115990346DAF84F
:109F20005C00C3FB0016169BC3FB0C580B4616992E
:109F3000C1FB0E361593DAF860E0D9F810C1D9F8F4
:109F40004C01139BCCFB0E32DAF86410CCFB0147BA
:109F5000C1F1000CC0FB0C321393C0FB0E47D9F8C3
:109F6000CC31D9F890111693C1FB0E58D9F8900155
:109F700015990346DAF86400C3FB0016169BC3FB71
:109F80000C580B461699C1FB0E361593DAF868E0AB
:109F9000D9F814C1D9F84801139BCCFB0E32DAF87A
:109FA0006C10CCFB0147C1F1000CC0FB0C321393C9
:109FB000C0FB0E47D9F8C831D9F894111693C1FBEC
:109FC0000E58D9F8940115990346DAF86C00C3FBD2
:109FD0000016169BC3FB0C580B461699C1FB0E3698
:109FE0001593DAF870E0D9F818C1D9F84401139B39
:109FF000CCFB0E32DAF87410CCFB0147C1F1000C37
:10A00000C0FB0C321393C0FB0E47D9F8C431D9F80A
:10A0100098111693C1FB0E58D9F89801159903466B
:10A02000DAF87400C3FB0016169BC3FB0C580B46F2
:10A030001699C1FB0E361593DAF878E0D9F81CC1F1
:10A04000D9F84001139BCCFB0E32DAF87C10CCFB24
:10A050000147C1F1000CC0FB0C3216972746169C35
:10A060002146C0FB0E711691D9F8C001D9F89C1198
:10A070001397C1FB0E58D9F89C4115992746DAF879
:10A080007C40C7FB0416C0FB0C58C0FB0E164FF0FB
:10A09000140C18460C24674602FA04F342FA0CF238
:10A0A00020FA0CF040EA03003EF07CFF119B23F8FD
:10A0B000040C28463D4608FA04F348FA07F820FA4B
:10A0C00007F040EA03003EF06DFF119B169F23F856
:10A0D000020C139807FA04F347FA05F720FA05F083
:10A0E00040EA03003EF05EFF129BA3F87C000846A6
:10A0F00006FA04F346FA05F620FA05F040EA0300F2
:10A100003EF050FF129BA3F87E00119B0433119385
:10A11000129B043B1293B94B0AF1400A9A4509F588
:10A1200080797FF451AE0B9B0D9AD3F800329B1AC5
:10A130000B9A03F00703C2F800320E9B01330E9313
:10A14000109B80331093089B803308930E9B122B37
:10A150007FF4D4AC049B013304930F9B90330F9393
:10A16000059B7C330593149B08331493FEF7EDBED7
:10A17000089B00974FF41060CDE901A3A8F10802F5
:10A180002B4600FB06400A913DF044FC089B48F832
:10A19000040B18330A990893013648370AF13E0A2E
:10A1A0003CE404F58053D3F80822002A04DDD3F8F8
:10A1B0000C22002A3FF73BACD3F80002904F00235B
:10A1C0006FF0404607E054F82320B2F1404F1BDC0B
:10A1D00044F8237001338342F5DB04F58053DFF844
:10A1E00020C2D3F80462002204F510636FF04047E8
:10A1F000B242BFF61CAC1868B0F1404F0ADCC3F89D
:10A2000000C001320433F3E7B2F1804FA8BF44F835
:10A210002360DFE7B0F1804FA8BF1F60F1E7DA07E6
:10A2200020D5D1F830236B6B9AB9D1F84423013291
:10A2300033F912300022211F164617469446BB42BE
:10A2400018DC209B33432093219B13432193FFF77A
:10A25000F2BBD1F8402303EB4203B3F9303003EBF8
:10A260004303E7E704F58052D2E980318B42B8BF5F
:10A270000B46DFE751F8048FD1F8000908EB000E18
:10A28000A8EB0000C1F800E0C1F80009E0468EEA42
:10A29000EE78A8EBEE7846EA0806E64680EAE07E2D
:10A2A000AEEBE07E42EA0E020137C8E7CDE90220BC
:10A2B00009F1F8020192069A009220462A463EF0E1
:10A2C00027F9FFF7D0BBDBF8002042B9584618EE5B
:10A2D000101A3EF045FF6FF00A00FEF788BCDBF86D
:10A2E0000430002BF2D0DBF80C50002DEED0DBF860
:10A2F00014A0BAF1000FE9D0516B1278002A0CBFFC
:10A300000822062231F91260089996FBF8F64822D5
:10A3100002FB04121A44D16B022966D004F5906244
:10A3200055F8227040F226229742D7BF07372027E0
:10A3300097FBF8F701372097013F4FF4106909FBAD
:10A3400004F905EB0900394605EB84050B930A90E7
:10A35000FDF79EFD05F5805C08FB07F7DCF80012B1
:10A36000089B0A980837B9420AEB840505F5805521
:10A37000B8BF3946CCF80012113191FBF8F12191A8
:10A38000D5F8002B22924827D5F8082B239207FBFB
:10A3900004370B9BD5F8102B24921F444FF4906187
:10A3A0003A6C002A08BF00262596DCF8082226927F
:10A3B00020AA0092069A01FB04A1134401F59051D2
:10A3C0000AEB0902FEF776F8C5F8000BFB6BC5F83F
:10A3D000083B259BC5F8103B279BC5F8183B069BFF
:10A3E000483301340693FFF75EBB176C1FB1771E2D
:10A3F00020963FB2A1E720979FE700BF646609005F
:10A40000010000C0069B002503F50053403408936B
:10A41000AA4605F001030B930A9B089A0A9806992D
:10A4200003F5805300EBC510D3F8183B0093D2F826
:10A4300000220B9B3DF0FAFB089B0B99D3F80032EE
:10A440004FF4886202FB0133069A02EB830752F84D
:10A450002310FA6D4FF000735046C1FB0A306FF0C5
:10A460007301C2FB01304FF455797968BA6DC1FBB5
:10A470000930B549C2FB013041F6D478B9687A6D2C
:10A48000C1FB0830B149C2FB013046F2B86CF96833
:10A490003A6DC1FB0C30AE49C2FB0130AD4A39699F
:10A4A000C1FB0230AC49FA6CC2FB01307969BA6C6D
:10A4B000C1FB0C3045F28401C2FB0130B9697A6CF2
:10A4C000C1FB083040F22C71C2FB0130F9693A6CD3
:10A4D000C1FB09307421C2FB01304FF00C08024669
:10A4E0004FF01409184602FA08F342FA09F220FA6A
:10A4F00009F040EA03003EF055FD07F5805124F8CD
:10A50000400C0A684FF0007053464FF4D07CC2FBF9
:10A510000C0341F67C0C4A68C2FB0C0349F2FC7C3C
:10A520008A68C2FB0C038D4ACE68C6FB02038C4AC4
:10A530000E69C6FB02036FF0B30C4A69C2FB0C0341
:10A540004FF4127C8A69C2FB0C03CA696FF01301D5
:10A55000C2FB010303FA08F243FA09F320FA09F0F7
:10A5600040EA02003EF01EFDA4F14003CDE90D4398
:10A57000DFF8F48124F8200CD8F844E0D7F8002163
:10A58000D7F85CC1D8F840104FF000705346C2FBBA
:10A5900001034FF00071D146C2FB0E19CEF100024B
:10A5A000CCFB0203D8F84020CCFB0219D8F84CC0F1
:10A5B000D7F804E1D7F85821D8F84860CEFB060355
:10A5C000CEFB0C19CCF1000CC2FB0C03C2FB06192C
:10A5D000D8F854C0D7F808E1D7F85421D8F850601B
:10A5E000CEFB0603CEFB0C19CCF1000CC2FB0C0316
:10A5F000C2FB0619D8F85CC0D7F80CE1D7F8502197
:10A60000D8F85860CEFB0603CEFB0C19CCF1000C39
:10A61000C2FB0C03C2FB0619D8F864C0D7F810E1DE
:10A62000D7F84C21D8F86060CEFB0603CEFB0C199E
:10A63000CCF1000CC2FB0C03C2FB0619D8F86CC0AD
:10A64000D7F814E1D7F84821D8F86860CEFB0603A4
:10A65000CEFB0C19CCF1000CC2FB0C03C2FB06199B
:10A66000D8F874C0D7F818E1D7F84421D8F870604A
:10A67000CEFB0603CEFB0C19CCF1000CC2FB0C0385
:10A68000C2FB0619D8F87CC0D7F81CE1D7F84021E6
:10A69000D8F87860CEFB0603CEFB0C19CCF1000C89
:10A6A000C2FB0C03C2FB06190C264FF0140C03FA74
:10A6B00006F243FA0CF320FA0CF040EA02003EF0F6
:10A6C00071FC0E9B23F8020F4FF0140C0E930846FA
:10A6D00009FA06F349FA0CF920FA0CF040EA0300F3
:10A6E0003EF060FC0D9B23F8020D0D931D4B08F10D
:10A6F0004008434507F580777FF43EAF089B0B9AEF
:10A70000D3F8003201359B1A089A03F00703122D83
:10A71000C2F8003204F140047FF47BAE1AE55846DB
:10A7200018EE101A3EF01CFD6FF00B00FEF75FBA3A
:10A730006FF00400FEF75BBA6FF00500FEF757BA42
:10A740000020FEF754BA00BFD4F8FFFF7CAFFFFF34
:10A750003CB6FDFF78940400C44902004CE80300B5
:10A760002464FFFF64660900A462090010B54FF07D
:10A770008043D3F80443620707D54FF484704FF049
:10A78000F5FF10B11E4B1B689847A30608D54FF480
:10A790008A704FF0EBFF18B11A4B00201B689847E6
:10A7A000600608D54FF48C704FF0E0FF18B1154BE0
:10A7B00001201B689847210608D54FF48E704FF092
:10A7C000D5FF18B1104B00201B689847E20508D54B
:10A7D0004FF490704FF0CAFF18B10B4B01201B686B
:10A7E0009847A3050AD54FF492704FF0BFFF28B1E8
:10A7F000054BBDE810401B680220184710BD00BF84
:10A80000B4610120B8610120BC610120DFED0A7A4A
:10A810009FED0A7ADFED0A6AA0EE277ADFED097A6A
:10A82000E7EE007AB7EE007AA0EE267A67EE807A3D
:10A8300087EE870A704700BF6BD30DBCBA132FBDDC
:10A84000AEE534BF75AA2A3E0248032200211BF060
:10A8500021B900BF00B000400248042201211BF0D2
:10A8600019B900BF001001400248042202211BF068
:10A8700011B900BF0040024008B5834B8348DA1C81
:10A88000121AC11E22F00302994288BF0022804999
:10A8900048F096FF7F4B8048DA1C121AC11E22F046
:10A8A0000302994288BF0022002148F0C9FF4FF0FF
:10A8B0008053D3F83021082A4ED14FF08042002136
:10A8C000C2F80C11C2F81011C2F8381502F5404256
:10A8D000D3F80414C2F82015D3F80814C2F82415CC
:10A8E000D3F80C14C2F82815D3F81014C2F82C159C
:10A8F000D3F81414C2F83015D3F81814C2F834156C
:10A90000D3F81C14C2F84015D3F82014C2F844152B
:10A91000D3F82414C2F84815D3F82814C2F84C15FB
:10A92000D3F82C14C2F85015D3F83014C2F85415CB
:10A93000D3F83414C2F86015D3F83814C2F864158B
:10A94000D3F83C14C2F86815D3F84014C2F86C155B
:10A95000D3F84434C2F8703515F044FB18B14F4BAE
:10A960004F4AC3F88C2615F03DFB18B14D4BFB2226
:10A97000C3F8182515F036FB70B14FF080414FF049
:10A980008053D1F8E42ED3F8583222F00F0203F0AE
:10A990000F031343C1F8E43E15F024FB20B1424BF2
:10A9A0004FF40072C3F840264FF08053D3F8303193
:10A9B000082B09D14FF08043D3F80024D10744BFBE
:10A9C0006FF00102C3F80024384AD2F8883043F40B
:10A9D0007003C2F88830BFF34F8FBFF36F8F4FF013
:10A9E0001023D3F80C22D2071DD5314B0122C3F816
:10A9F0000425D3F80024002AFBD04FF01022D2F80F
:10AA00000C3223F00103C2F80C32294BD3F8002496
:10AA1000002AFBD00022C3F80425D3F80024002A22
:10AA2000FBD000F069FDD3F80022002A03DBD3F845
:10AA30000432002B22DA1E4B0122C3F80425D3F87E
:10AA40000024002AFBD04FF010221221C2F800127D
:10AA5000D3F80024002AFBD04FF010231222C3F8B1
:10AA60000422134BD3F80024002AFBD00022C3F8A1
:10AA70000425D3F80024002AFBD0D2E70D4B0E4A60
:10AA80001A6034F041FA00BFD40501200000012013
:10AA90001C6C0900946C0120D80501200050004076
:10AAA0004881030000F000400090024000ED00E00B
:10AAB00000E00140000001200090D003014902485D
:10AAC00039F034B8E86001200030004002494FF00E
:10AAD000402039F02BB800BF1C61012008B50748A1
:10AAE000D0F8183143B14FF48C714FF0C3FDBDE87D
:10AAF0000840034847F083BD08BD00BF0030024056
:10AB00008860012008B50748D0F8183143B14FF4E8
:10AB10008C714FF0AFFDBDE80840034847F06FBDB2
:10AB200008BD00BF00F00240AC600120F7B5224C28
:10AB3000022501A851F0D2FA052812D11F4C204E4F
:10AB40004FF40C750DF102012046ADF8025051F0A2
:10AB500065FA28B30C2802D11A4850F0B1FC03B0B2
:10AB6000F0BD019B032B19D004D8022BE1D10023A7
:10AB70002370DEE7A3F10902022ADAD80A2B09D0F2
:10AB8000092B09D00B2B0CBF01204FF0FF3038F000
:10AB9000ADFECEE70020FAE70220F8E72570C8E70F
:10ABA000D6F8DC30002BCDD01F68D3E90112204647
:10ABB00090473B46F6E700BF776C0120F45D01202B
:10ABC000C0610120571309000149024848F090B9BB
:10ABD000D0600120009000400149024848F088B947
:10ABE000DC60012000A000400149024853F08AB80F
:10ABF00050610120002000400149024853F082B812
:10AC000074610120008002402DE9F04FB64BB74A35
:10AC1000D3F80013002385B01C4601201D4621FAFD
:10AC200003F6F6070BD552F8236046B100FA03F697
:10AC3000344342F82350BFF36F8FBFF34F8F01337C
:10AC4000192BECD1E20736D5A74B0122C3F8142506
:10AC5000C3F8102500221546930003F1804303F545
:10AC60001C330132082A5D609D62F5D19E4B5D6206
:10AC70009D64C3F85851D3F80024D3F800140A4354
:10AC8000C3F80024D3F80023C3F80823984AC3F874
:10AC90000423984BDC220021184648F0D1FD4022C5
:10ACA00082820281012101A8CDE9015503958DF829
:10ACB000051011F0EDF914F4006F8E4D08D08A4B99
:10ACC000D3F8A8369BB2A5F8D230012385F8D73047
:10ACD000A3021ED5844ED6F8143513F4807302D027
:10ACE0003CF04CFE0123D6F81025D70540F1368103
:10ACF00095F8D7304BB1B5F8D220002085F8D700B1
:10AD0000012392B2882144F0A6FC0121032044F0E3
:10AD100095FC600226D5744BD3F8006406F4E0621B
:10AD2000F105C3F8002405D50121C3F82C15042032
:10AD300044F084FC72050FD56B4B0122C3F8082543
:10AD40009A65D3F8002312F4001208BFC3F8542107
:10AD50004FF40012C3F80423B30503D501210520E5
:10AD600044F06CFC270237D55F4BD3F880E4D3F86E
:10AD70008424D3F88814D3F88C74D3F89064D3F86F
:10AD800094045FFA81FCD3F89814D3F89C341EF035
:10AD90007F0F5FFA8EF8D2B2FFB2F6B2C0B2C9B27C
:10ADA000DBB201D1052A17D04FF4C06E8DF80D002B
:10ADB0008DF80E1001A80121CDF804E08DF808806F
:10ADC0008DF809208DF80AC08DF80B708DF80C6095
:10ADD0008DF80F3011F05CF9474B23405BB195F8CB
:10ADE000D830002B40F0C2804FF0E023D3F8F03D84
:10ADF000DE0700D500BEDFF8FC80DFF8EC90DFF85E
:10AE000000B1474600264FF0140A06F10C0324FA5D
:10AE100003F3D807F1B222D50AFB0693082ED3F824
:10AE200008273B6853FA82F33B604FF0180303FB9B
:10AE30000653D2B2D88812FA80F080B2D88000F0DF
:10AE400099803889904240F09580DB88BA889BB21F
:10AE50009A4240F28F8011B9584614F0ADFC013689
:10AE6000092E07F11807D0D1244B2340002B6BD0BB
:10AE70001D4BD3F86C94C3F86C94BFF36F8FBFF382
:10AE80004F8F14F4806407D0D3F88044D3F8803413
:10AE90001906C4F3C01479D54FF0000A154F0026E7
:10AEA0004FF0180B29FA06F3DA07F0B201D44EBBC3
:10AEB00044B30D4B142202FB0633FA68D3F808366C
:10AEC00052FA83F2FA600BFB0652518A89B251FAA8
:10AED00083F39BB25382538A398A9BB2994258D9E1
:10AEE0003CF000FD0EE000BF007002400071024027
:10AEF0000514C001E41E0120FCFB1F00000400013A
:10AF00004C7002400136082E07F11807CAD1002400
:10AF10001826012704F1100329FA03F3DB07E0B236
:10AF200003D464B9BAF1000F09D006FB0452B8F893
:10AF30000410D3889BB2994234D93CF0F3FC01341D
:10AF4000082C08F11808E5D11748184B03600023B6
:10AF5000436005B0BDE8F04F05F0A2BA002B7FF4C6
:10AF6000D4AE4FF40013C6F80833CEE6002385F8BC
:10AF7000D83040E7182303FB06530020DA88BA8054
:10AF8000DA88012392B244F066FB68E74FF0010AC9
:10AF900084E7528A40F08001012392B2002044F0FD
:10AFA0005AFBAFE79772CAE7706601209DDF070082
:10AFB0002DE9F0478AB08C46DDE9121E11F001013F
:10AFC000DCF80C400646174602D0012B00F0A280A8
:10AFD000B4F5C87F72DA2011052290FBF2F20292DA
:10AFE00002EB8202821A0392C4F38102049204F0FB
:10AFF00003040022059415461446DCF81480B8F1C9
:10B00000020F40F0BC80DCF81800002808BF4FF0A9
:10B01000010805EB45058148454410F82580CDF829
:10B02000188000EB850568780790A8780890E87884
:10B03000099011B3012B20D10DF108090EF104087C
:10B0400006AB4D4603CD9D42C8F80000C8F8041079
:10B05000A94608F10808F4D10EF114080DF12809E9
:10B060001D4603CD4D45C8F80000C8F804102B4616
:10B0700008F10808F4D1CEF80020DCF81430CCF840
:10B080003C40022B40F0C080DCF81840002C00F05F
:10B09000A3807C1E7D1D0299304653F046FE04F8C5
:10B0A000010FAC42F7D1032301240DF1180A03EB81
:10B0B000430599463D444FF0000877E0B4F5FA7F28
:10B0C00012DAA4F5C874A0100522B0FBF2F20292C5
:10B0D00002EB8202821A04F0030403920022049419
:10B0E00005921446012588E7A4F5FA740320B4FB01
:10B0F000F0F000EB4002A41ADCF8182002900025C2
:10B10000CDE90455039412B1CDE903042A46012484
:10B11000022572E7B4F5B47F04F001024FEA64053A
:10B1200010DA242495FBF4F004FB10550624029059
:10B1300095FBF4F004FB105500240495039005944E
:10B1400003255AE7F32D0CDCB43D281102900024AE
:10B15000C5F3810005F003050495039005940425CB
:10B160004BE7F43D0320B5FBF0F0029000EB40000C
:10B170002D1A00240395CDE9044405253DE74FF041
:10B18000000846E702AB304653F82410019153F013
:10B19000CCFD01992875304653F0C7FD01996875BB
:10B1A000304653F0C2FD08F10108A8755AF8242072
:10B1B000904508EB090305F10305E3DB0134042C9A
:10B1C0007FF475AF002387F83D3087F83C3087F86F
:10B1D0003B300AB0BDE8F087234666E702AB304655
:10B1E00053F8241053F0A1FD08F8010B01355AF86B
:10B1F0002420954205EB0903F0DB0134042C07D130
:10B200000023BB757B75E4E700231C460DF1180A8B
:10B21000994607EB03080025E9E700BFBC360900A3
:10B2200010B5074CD4F800314BB1064B5B6898471A
:10B2300020464FF48071BDE810404FF01BBA10BD9E
:10B240000000014098610120022A2DE9F0415AD105
:10B250003B4B826883FB02423A4E846986FB04546E
:10B2600022440A60384C426884FB0252374FC56959
:10B2700087FB05C52A444A60026883FB0252056ABF
:10B2800086FB05752A448A60314F026887FB0252AB
:10B29000304D066A85FB06C63244CA604FF06046F0
:10B2A000426886FB02C2D0F81CC086FB0CEC6244EC
:10B2B0000A61826885FB02C2D0F818C087FB0CECDB
:10B2C00062444A61426983FB02C28A61026984FB6B
:10B2D00002C2CA61C26883FB02420A62C36887FB7A
:10B2E00003234B62036986FB03238B62436985FB5F
:10B2F0000323CB620023C1E91033C1E90E33C1E956
:10B300000C33BDE8F081144B902404FB023202F1AF
:10B31000480C01F144058C3200F1240E50F8043B36
:10B3200052F804695CF8047B1C4687FB048441F8EE
:10B33000044B86FB0343864545F80439EED1E0E72C
:10B34000D8E3CEB8281C310733C3BEB2CD3C410D83
:10B350009A615FC9669EA0F6646009002DE9F34119
:10B3600090F8653090F86620013BDBB280F86B30D6
:10B37000531EDBB280F86C30012A84BF90F86C3029
:10B3800003F1FF334FF000058CBFDBB2012380F8DF
:10B390006D30044680F86E500126856540F2033713
:10B3A00094F86330EAB2934215D82368324A934244
:10B3B00030D002F58052934257D002F5805293422A
:10B3C00055D002F58032934253D002F58052934219
:10B3D0003FD104231FE0A36C03EB021301A81B7BE6
:10B3E00001934FEA02182AF037FA019A02F5E07247
:10B3F00040F8227094F86D303342A36C4344187BBC
:10B4000005D04FF0A6F97600F6B20135C8E74FF047
:10B4100076F9F8E70023194850F8332000EBC3030E
:10B42000002593F9043001215160002BC2F8045526
:10B43000D160C2F80855C2F810554FF48035C2F8F3
:10B44000045306DB5A0903F01F0399400C4B43F8E1
:10B450002210236801224FF47A715A60DA60C3F82F
:10B4600040151A6002B0BDE8F0810123D3E7022342
:10B47000D1E70323CFE700BF008000403C3B090039
:10B4800000E100E000280DDB4309012200F01F006D
:10B4900002FA00F02033044A42F82300BFF34F8F32
:10B4A000BFF36F8F704700BF00E100E04309012246
:10B4B00000F01F0002FA00F02033044A42F8230093
:10B4C000BFF34F8FBFF36F8F704700BF00E100E005
:10B4D0000028ACBF00F16040064B4FEA4111ACBF01
:10B4E00000F5614000F00F00C9B2B4BF195480F8F4
:10B4F0000013704714ED00E0BFF34F8F0549064B72
:10B50000CA6802F4E0621343CB60BFF34F8F00BF01
:10B51000FDE700BF00ED00E00400FA0570B510EE95
:10B52000105A25F000440123B4F1FF4FB0EE403A29
:10B530000646036004DB60EE003AB0EE630A70BDBD
:10B5400034B9DFEDCA7AB7EE007AC7EE273AF4E7EE
:10B55000B4F1E45F0BDA002DBEBF4FF0FF330360A0
:10B56000B1EE400A1CF072F9F1EE403AE5E7002D29
:10B5700080F2C282B4F1964FE3DAB4F17A5F9FEDC4
:10B58000BC5A78DADFEDB90A20EE050A002000F097
:10B5900021FEF0EE403AF5EE403AF1EE10FAD0D04E
:10B5A00023EE230AB0EEC00A85EE000A1CF04EF925
:10B5B000F5EEC03AF1EE10FA4CBF4FF0FF33012325
:10B5C000B4F17E5FF0EE402A336000F08F82B4F178
:10B5D000804FB1EE433A00F089826B0000F1D281D6
:10B5E000A44B9C4200F3F380B0EE430A1CF02EF90A
:10B5F000A14B9C42F1EE407A40F39B80F7EE003A7B
:10B6000033EEC33A23EE037ADFED9C6A9FED9C6A2A
:10B61000DFED9C3AA7EE266ADFED9B6AE6EE076A4D
:10B620009FED9A6AA6EE876ADFED996AE6EE076AF1
:10B630009FED986AE6EE873ADFED976AE7EE066AD5
:10B640009FED966AA6EE876ADFED956AE6EE076AD9
:10B650009FED946AA6EE876ADFED936AE6EE076ACD
:10B6600063EE833AE6EE873AB6EE007AE3EE473AC7
:10B6700073EEA73AF7E1B1EE407AB0EE470A16F062
:10B6800021FDB4EE407AF1EE10FA19D0B6EE000AC0
:10B6900027EE007AB0EE470A16F014FD37EE400AA6
:10B6A00030EE000AF0EE407AFEEECF7A17EE903AD6
:10B6B000062B39D8DFE803F02312121F1F2B2B00B3
:10B6C000DFED7A7A77EEC37A17EE903A03F0010352
:10B6D00007EE903A9B00B8EEE70AE9E7F6EE007A4B
:10B6E00037EEC00ADFED610A20EE050A00F036FBF6
:10B6F000F1EE403A4FE7F7EE007A37EEC00ADFEDA1
:10B700005B0A20EE050A002000F064FDF0E7F7EE8A
:10B71000087A30EE670ADFED550A20EE050A00F0E0
:10B720001DFBB1EE400AE3E7F0EE007A30EE670A67
:10B73000E5E75F4B9C4264DDDFED5E3A73EE633A12
:10B7400063EEA34A9FED5C6ADFED5C6ADFED5C5A55
:10B750009FED5C5A9FED5C0A24EEA37AE7EE066A41
:10B760009FED5A6AA6EE876ADFED596AE6EE076A30
:10B770009FED586AA6EE876ADFED576AE7EE265A14
:10B78000DFED566AE5EE876ADFED555AE6EE875A39
:10B79000DFED546AE5EE876ADFED535AA7EE255ACE
:10B7A000DFED525AE5EE075A9FED515AA5EE875A42
:10B7B000DFED505AE5EE075AE5EEA36ADFED4E3AAB
:10B7C000E6EEC73AD4EE863A73EEC03A50E74B4BFA
:10B7D0009C4206DDF0EE003A33EEC33ADFED237A09
:10B7E00010E7474B9C4206DDDFED463ADFED1F7A5E
:10B7F00073EE633AA4E7F7EE007A33EE673ADFEDD3
:10B800001B7ADFED416A9FED417A9FED416AA3EE1D
:10B81000267ADFED406AE7EE036A9FED3F7AA6EEF7
:10B82000837ADFED3E6AE7EE036A9FED487AA6EE83
:10B83000837ADFED3B6AE3EE066A9FED3A6AA6EE95
:10B84000836ADFED396AE6EE036A9FED386AA6EE99
:10B85000836AF7EE006AE6EE036A27EE037AC7EE24
:10B86000263ABEEE007AE3EE073A01E70000000058
:10B87000DB0F49406666663F1F4A3B3FA283D337D2
:10B88000679767393F239E3DA1549C3A7E02F23B65
:10B8900001F0893D752C3C384584E23834B6053AD0
:10B8A000C66E3D3B1599A83C661AA53E0000004BAC
:10B8B00007336D3E0C5BEC3E6B7BA53976F4B7BA73
:10B8C00067F8663A85300DBACDCDF83D07E7C73B3E
:10B8D000474D06BD5EB9F73E27F9A3B9FE7771BBA8
:10B8E0003D37933C3C2117BEF7E9AF399916143B1D
:10B8F000FEFC28BC155A843D521CE63117A6DD3FDC
:10B900001FA69D3FC316BB3F5E3C5B3C78756A3EFD
:10B91000DBD5523BB24B7A3FE73ABA3FF400223FC5
:10B92000AF72D53DDFEF443F2D390840BE2E1D409C
:10B9300067FF0538B435F13ABDD7F536E440DA3C57
:10B94000E6DC153E7ACCA63E5A245C3E3F239EBDE3
:10B95000D6EE4B3A54BF983C6E0F303EC5D0383FC0
:10B960003B2DB23FE8C4D5BAD23D5B3A1D7FD63EEF
:10B970005C061CBAFD0C503A610B36BBABAAAA3D63
:10B9800000000000B4F1824FF7EE003A7DDABDEE20
:10B99000C36A5FED197A1FED197A5FED196AB8EE87
:10B9A000C60A16EE103A33EE403A033BA3EE277A6E
:10B9B0005FED1E7AE7EE037A1FED1F7AA7EE837A1A
:10B9C0005FED207AE7EE037A1FED217AA7EE837A06
:10B9D0005FED227AE7EE037A1FED237AA3EE267A53
:10B9E0005FED246AE7EE036A1FED257AA6EE837AFF
:10B9F0005FED266AE7EE036A1FED277AA6EE837AEB
:10BA0000F0EE636AE7EE036A67EE837AC7EEA63A62
:10BA1000F6EE007AE3EE273A042B24D8DFE803F0B1
:10BA2000322F2C290300F1EE087A33EE270AF1EECB
:10BA3000047A73EE277A67EE807AB1EE000A33EE6D
:10BA4000000A60EE277AB0EE080A33EE000A20EE14
:10BA5000270AF0EE007A33EE273A23EE000A1BF0B5
:10BA6000F5FE73EE803A002DBFF667AD72EEE33A55
:10BA700063E5B7EE000ADAE7F7EE007ADDE7F7EE06
:10BA8000007AE0E7B7EE000AE3E7B0EE430A1BF006
:10BA9000DDFEB4F1B94F30EE630A24DA83EE837A27
:10BAA0001FED506A5FED506A5FED503A67EE077A1E
:10BAB000E7EE866A1FED526AA6EEA76A5FED536A4B
:10BAC000E6EE276A1FED546AA6EEA76A5FED556A97
:10BAD000E6EE276AF6EE007AE6EE873A33EE673A4C
:10BAE000E3EE003ABFE763EE003ABCE75FED5C3A95
:10BAF000BCE75FED5D3A20E5B4F17E5FF9D0B4F1CB
:10BB0000804FF6D05FED622A67E500BFF0B510EE1A
:10BB1000105A854A25F00043934285B0044605DC5F
:10BB2000002380ED000A4360002020E07F4A93421A
:10BB300038DC002DDFED7E7A7E4A23F00F0318DD1E
:10BB4000934230EE670A09BFDFED7B7ADFED7B7A47
:10BB500030EE670ADFED7A7A30EE677A30EE470A28
:10BB600080ED007A30EE670A80ED010A012005B011
:10BB7000F0BD934230EE270A09BFDFED6F7ADFEDAB
:10BB80006F7A30EE270ADFED6E7A30EE277A30EEEC
:10BB9000470A80ED007A30EE270A80ED010A4FF067
:10BBA000FF30E4E7674A934274DC9FED677AB0EEBA
:10BBB000C00AF6EE007AE0EE077AFDEEE77AB8EE1C
:10BBC000E77A17EE900ADFED5A7AA7EE670A1F2888
:10BBD000DFED5A7A67EE277AB1EE476A70EE676A50
:10BBE00016EE901A1EDC594E471E25F0004256F8FC
:10BBF000276022F0FF02B24214D0216094ED007A57
:10BC000030EE470A002D30EE670A84ED010AAEDA05
:10BC1000B1EE477AB1EE400A84ED007A84ED010A74
:10BC20004042A4E7C1F3C756DA15C6EBD353082B3D
:10BC3000E3DDDFED417ADFED425AF0EE406AE6EEF9
:10BC4000276A30EE660AA6EE270AF0EE407AD7EEB3
:10BC5000257A76EEE75A15EE901AC1F3C753D31A38
:10BC6000192B04DCC4ED005AB0EE660AC6E7DFED1E
:10BC7000385AB0EE660AA6EE250A76EEC07ADFEDF7
:10BC8000356AE6EE257AD7EE267A30EE677A84EDCD
:10BC9000007AB3E7B3F1FF4F06DB30EE400A80EDE8
:10BCA000010A80ED000A3FE7DA15863AA3EBC2539A
:10BCB00007EE903ABDEEE77ADFED276AB8EEC77A75
:10BCC00077EEC77A8DED017A67EEA67ABDEEE77A58
:10BCD000B8EEC77A77EEC77A8DED027A67EEA67A6C
:10BCE000F5EE407AF1EE10FACDED037A1AD1B5EE09
:10BCF000407AF1EE10FA14BF02230123214601A875
:10BD000000F08CF8002DBFF632AFD4ED007AF1EEE2
:10BD1000677AC4ED007AD4ED017AF1EE677AC4ED6A
:10BD2000017A7DE70323E9E7D80F493FE3CB1640CB
:10BD3000800FC93FD00FC93F0044353743443537E2
:10BD400008A3852E800F494384F9223F582C09000F
:10BD500000A3852E32318D240000804310EE103A6E
:10BD600023F00043B3F1485FB7EE006A05DAFDEE59
:10BD7000C07A17EE902A002A3DD060EE005ADFED1F
:10BD80001F7A9FED1F7ADFED1F6A1F4AA5EEA77A83
:10BD90009342DFED1E7AE7EE257A9FED1D7AA7EE3E
:10BDA000A57ADFED1C7AE7EE257AB0EE667AA7EE8B
:10BDB000A57AF6EE006A65EEA67A67EE256A20EEB1
:10BDC000C07AA5EEA67A04DC37EEC77A36EE470ACB
:10BDD0007047114A9342DABF03F17F4306EE903A6F
:10BDE000F5EE026A77EEE67A36EE660A77EEC77A05
:10BDF00030EE670A7047B0EE460A70474ED747AD3F
:10BE0000F6740F31ABAA2A3D9999993E7CF293B40E
:10BE1000010DD037610BB6BA0000483F2DE9F04F55
:10BE20002DED048BD7B09B460291D11E48BF111D4A
:10BE3000C9104D1C8146581EEB0003930C1A1AAF13
:10BE40000BF1090C9FEDC47AC44B9246A2EBC505D9
:10BE500004EB0C0E3E46002CA4BFE25C07EE902AD9
:10BE600004F10104ACBFF8EE677AF0EE477A74454E
:10BE7000E7EC017AEFD109EB8B0306EB8B0601931C
:10BE80000DF5847EDFEDB47A37464C46F4EC016A5A
:10BE9000019B37ED017A9C42E6EE877AF6D10130BC
:10BEA0008445EEEC017A06F10406EBD1AB48DFEDF8
:10BEB000AC8A9FEDAC9A0B180926049356AB03EBA2
:10BEC000860111ED140A42AB06A94FEA860803EB7E
:10BED00086000F46344660EE287A013CFDEEE77A94
:10BEE000F8EEE77AA7EEC90ABDEEC00AA7EC010A90
:10BEF00030ED010A37EE800AEDD12846059131F088
:10BF00001FFCB0EE408AB4EE000A28EE000A16F0DC
:10BF1000D9F8F2EE007AA0EE678A002D0599FDEEC1
:10BF2000C87AB8EEE70A17EE907A38EE408A37DD25
:10BF300006F1FF3C06ABC5F1080E53F82C4044FA5D
:10BF40000EF0074400FA0EF0241AC5F1070043F87A
:10BF50002C400441002C31DD00200137864651F889
:10BF6000043B002866D123B1C3F5807341F8043C3B
:10BF700001200EF1010E7645F1D1002D03DD012DDA
:10BF80005DD0022D65D0022C18D1B7EE000A30EE3C
:10BF9000488A98B1284631F0D3FB38EE408A0DE04C
:10BFA00005D1701E06AB53F820402412D2E7F6EEFE
:10BFB000007AB4EEE78AF1EE10FA39DAB5EE408A8B
:10BFC000F1EE10FA78D1711E00238C46BCF1080FF7
:10BFD00047D1002B4FD10EA8012150F80449002C65
:10BFE00046D056AB984406EB0B001AAB741CA8F174
:10BFF0004C0803EB80000E44B4423FF75FAF049B54
:10C000001B5D07EE903AF8EE677A4F46E0EC017A56
:10C01000DFED517A0146F7EC016A019B31ED017ABF
:10C020009F42E6EE877AF6D1E8EC017A0134E3E745
:10C03000022491E7C3F1FF0341F8043C99E706F1BC
:10C04000FF3C06AB53F82C1001F07F0143F82C1095
:10C0500099E706F1FF3C06AB53F82C1001F03F01C5
:10C06000F4E706AA52F82C000CF1FF3C0343ADE7BD
:10C070000131B2E7013906AB083D53F82130002BFE
:10C08000F8D02846B7EE000A019131F059FB01992A
:10C090008B001A1D42AB98180B46002B39DA0B4661
:10C0A000002B65DB42A800EB8306DFF8BCC0DFEDA8
:10C0B0002A7A0025C81A45E0039BB0EE480AA3EB94
:10C0C0000A0031F03DFBB4EEC90AF1EE10FA17DBBD
:10C0D00060EE287A06AAFDEEE77A711CF8EEE77AA0
:10C0E0000835A7EEC90AFDEEE77ABDEEC00A10EEEC
:10C0F000103A42F8263017EE903A42F82130C0E765
:10C10000BDEEC00A06AA10EE103A314642F82630BB
:10C11000B7E706AD55F82350019507EE905AF8EEB3
:10C12000E77A013B67EE807A20EE280A60ED017A1B
:10C13000B3E7FCEC016AB6EC017A01350A2DE6EEB4
:10C14000877A01D08542F4DD56AD05EB800040EDE5
:10C15000287A013BA4E700BF00000000D82C0900AA
:10C160000000803B000080430C6B090000000000D1
:10C170002EAB1FED027A13440A46002A1ADAFCB1EC
:10C18000F1EE477A029BC3ED007ADDED2E7A77EE71
:10C19000C77A2FAA0123994215DA0CB1F1EE677A1A
:10C1A000029B07F00700C3ED017A57B0BDEC048B8A
:10C1B000BDE8F08F73ED017A013A37EE277ADCE7BC
:10C1C000F0EE477ADEE7B2EC017A013377EE877A58
:10C1D000E1E700BF10EE103A23F00043B3F1485FEF
:10C1E00004DAFDEEC07A17EE903A5BB320EE007AE7
:10C1F000DFED157A9FED156AA7EE276ADFED147A59
:10C20000E6EE077A9FED136AA7EE876ADFED127AF2
:10C2100060EE076AE6EE077A30B99FED106AA7EE86
:10C22000276AA6EE260A704767EEE67AB6EE006A3F
:10C23000E0EE867AD7EE870ADFED097AE6EEA70A06
:10C2400030EE600A704700BFD3C92E2F342FD7B20B
:10C250001BEF3836010D50B98988083CABAA2ABEBD
:10C26000ABAA2A3E10EE103A23F00042B2F1465F2C
:10C2700016DAFDEEC07A17EE901A39BB431C134351
:10C2800006D1F0EEC07AB7EE007A87EE270A704743
:10C29000012800F09E80FFEE007A87EE800A70474A
:10C2A0004C498A4212DBDFED4C7A002BB8BFB1EE6D
:10C2B000400A37EEC00ADFED497AB8BFF1EE600AF6
:10C2C00077EEE00A30EE800ADFED450A9FED456A21
:10C2D000DFED456ADFED455A3E4920EE007A8A429D
:10C2E00067EE077AE7EE866A9FED416AA6EEA76AD7
:10C2F000DFED406AE6EE276A9FED3F6AA6EEA76A89
:10C30000DFED3E6AE6EE276A9FED3D6AA7EEA56A7D
:10C31000DFED3C5AE6EE275A9FED3B6AA5EEA76A91
:10C32000DFED3A5AE6EE275A9FED396AA5EEA76A85
:10C33000F0EE667AE6EE077A60EE075AF0EE606A93
:10C34000E7EEA56ADFED337AE6EE870AE5EEA70AA7
:10C3500030EE207A1DDB07EE900AF8EEE77A27EE42
:10C36000076A37EE277A9B17C6EE076A03F00203C7
:10C37000C3F10103B0EE007A76EEE00A70EE600AD7
:10C3800000EE103AE0EEC77AB8EEC00A20EE270AB7
:10C39000704701281BD0FFEE007AC7EE876A1E4B5C
:10C3A00017EE102A1A4006EE102A16EE902A36EEE4
:10C3B000400A134070EEC00A00EE103AF7EE007A21
:10C3C000E6EE007AE0EE807AA7EEA60A7047B0EEBD
:10C3D000470A704740A12C3FDA0F493F68212233BA
:10C3E000000000005FAE9BB745F4A3388453D937F3
:10C3F000C8261A3A16696B3BA427B33C8988083EC5
:10C400007AC09538B937813948DEBE3A1F37113CBA
:10C41000D10D5D3DABAAAA3E00F0FFFFF8B50E4678
:10C4200005462649304648F044FA05F10807044617
:10C4300018B390F85030D90602D5214824F0FCF802
:10C4400043F0100380F85030394644F0A5FB95F8CE
:10C450002A3003F00C03002B94F8513014BF012252
:10C46000002262F3410384F8513005D194F8503032
:10C4700043F0020384F85030F8BD1249304648F0CA
:10C4800018FA0446B8B190F82A309A07D5D443F088
:10C490000203394680F82A3044F035F995F82A30FD
:10C4A00013F00C0F204618BF0121BDE8F84008BF6B
:10C4B000002144F016B90448C0E700BFC469080071
:10C4C0003D0408008C650800540408002DE9F74F6E
:10C4D0000646002508466A4601A9019548F02BFD4D
:10C4E0000199022902D8234824F092F87068DFF8F5
:10C4F00088900122890017F0D3FA756007463581CC
:10C50000019BACB2A34205F1010505D85B00776041
:10C51000338103B0BDE8F08F009B53F824A040F2B4
:10C520007342DAF8040002211CF0DAFADAF80800A3
:10C5300040F2CD511CF024FB40F2CD5347F6FF7280
:10C54000494683461CF0BCFADAF80C0040F2D2519E
:10C550001CF016FB4FEA8408B844824640F2D253DE
:10C5600047F6FF7249461CF0ABFA27F824B0A8F84A
:10C5700002A0C5E7170708000080FFFF2DE9F04F74
:10C580002DED028B90468DB0C268BDF864B0DDF829
:10C590006890BDF86C701D9D06468A461C46B0EE3C
:10C5A000408A2AB143689A4200F0B58008F040FF03
:10C5B000BBF11F0F01D81F2F77D9BAF1000F40F040
:10C5C000A080002F554614BF4FF0080A4FF00A0A0A
:10C5D000B8F1000F00F09C8040F20122ADF8182065
:10C5E000621CADF81A200022079206A84FF03CFD0D
:10C5F0008046002853D1182201460DEB020047F077
:10C600001FF99FED460A9FED467A464B079528EEA7
:10C61000008A002FC8EE077A03FB04F408BF4FF02E
:10C62000000942F210734046B4FBF3F40125189B55
:10C630008DF818A0ADF824408DF82D500293ADF878
:10C640000CB0CDF81090B6EE007A77EE877AADF8A0
:10C650001470FCEEE77ACDED087A3DF0E6FE8046F8
:10C66000E8B9314C06AA02A920464FF0DDFC80460D
:10C67000A8B92E49324606F1280004F07DFF9DF945
:10C680007020217828464FF0F9FC804638B9207890
:10C6900029464FF0CBFC804608B9189BF360404612
:10C6A0000DB0BDEC028BBDE8F08FBAF1000F20D0C9
:10C6B0005DB3F0EE0C7AB4EEE78AF1EE10FA69465B
:10C6C000284610D807EE904A9FED197AF8EE677A5F
:10C6D000F4EEC77AF1EE10FA05D83DF022FB6D4674
:10C6E0004FF0020A74E73DF01CFB6D464FF0030A61
:10C6F0006EE7002F554614BF4FF0040A4FF0050AAD
:10C7000066E700254FF0060A62E74FF0010A5FE78F
:10C71000CDE9068869E74FF01108C0E700247449A5
:10C7200000401C4440420F00A7050120C5A506009B
:10C730006666A63F2DE9F843416098464B680B9F1B
:10C7400091469A790A9B80F82C2003858D7D0446BA
:10C7500005F0300605F0060572B34B68D8683EF068
:10C7600008FFE0842DB10023C4E90298C4E9043332
:10C77000A361002384F82D3084F82A30A384089B19
:10C78000E361099B23621AB3EFB11B492246384685
:10C7900004F0F2FE5DB115F0040118BF01216068DC
:10C7A0001ABF84F82B100022012208F017FFDEB117
:10C7B000B20616D4012315E04FF6FF73C3842B464F
:10C7C00035461E46CEE70C48214604F0B9FEE1E7A7
:10C7D00067B10A492246384604F0CEFE26B17307F7
:10C7E000E8D4022384F82B30BDE8F88303482146BF
:10C7F00004F0A6FEF2E700BF87AB0700F3AB07002B
:10C800002DE9F04F89B005469DF8487016465FFA4D
:10C8100081F81C46002B3DD04268DFF890A01379C8
:10C8200012680621C2F80015342202FB03A3002F70
:10C830004FF0020283F82D204FF0000914BF0023AF
:10C8400020234FF6FF77A74228BF2746CDE904797A
:10C85000CDE9066969688DF80C9008798DF80D802E
:10C860004FF0340C0968019303AA00FB0CA037F0C9
:10C87000EFF90D4B9842834603D1E41B019B3E44E4
:10C88000DFD1686829F088FB584609B0BDE8F04F51
:10C8900037F02EB9414609F0F1F8002814BF002006
:10C8A000132009B0BDE8F08F0000AD0BE860012057
:10C8B00013B5124B9889D98993F90040421A92B264
:10C8C000402A28BF4022002C0EDA884212D09968F4
:10C8D0000B48019246F074FF0949019A802002B08A
:10C8E000BDE8104039F0FCBB88424FF0000003D196
:10C8F0000021F4E78020FBE70149F0E7CC1E01208E
:10C900007C550120064A002352F8041B814201D1C4
:10C91000184670470133082BF6D14FF0FF307047AF
:10C92000184601200D4B187801280FD10C4B1B78AD
:10C93000FF2B0DD10B4B1B68D9070AD4DA030AD49D
:10C9400013F4801F0CBF0020042070470228F1D18F
:10C950007047052070470120FAE700BFB86C01203E
:10C96000C86C0120B86401202DE9F041094F05464B
:10C970000E4600244FF6FF7837F81400404503D0E8
:10C98000324629464FF094FB4434B4F5AA7FF3D1E4
:10C99000BDE8F08138060120034B53F8203013B175
:10C9A0009A6801329A6070470C1E012038B5154B09
:10C9B00053F82040FCB120794DF0BDFE054660796A
:10C9C0004DF0B9FE6D0005F4FF75A2790E49E379CB
:10C9D000284300F0030040EA8202A0718A5C1344FD
:10C9E00094F908205BB29342E37105DBE3680133FD
:10C9F000E3600023E37138BD52429342FBDCE368FD
:10CA0000013BF5E738460120BC1409002DE9F04F41
:10CA10000446A9B08A46014640F2894048F006FD26
:10CA20000BAD002844D1CDE915000EAA7E21204689
:10CA30001FF060FDB04B119301224023CDE912237A
:10CA400018AB149311AB1093AC4B0B950C930821BE
:10CA500007A8002451F0EAFE2846CDE9054451F02C
:10CA6000FAF9A146A04627469DF85CB0BBF1000F3D
:10CA700000F0A781284651F0EEF9BBF15D0F00F000
:10CA8000958054D8BBF13A0F48D8BBF12B0F1BD877
:10CA9000BBF1220F00F0CF8007D8BBF10D0FE3D020
:10CAA00038D8ABF109010129DED9954823F0C4FD3E
:10CAB000012120461FF0C6F843680C9300230B9415
:10CAC0000D938DF85C30C2E7ABF12C030E2BECD844
:10CAD00001A252F823F000BF69CA020005CD02008E
:10CAE000ABCA0200ABCA020005CD020005CD0200B0
:10CAF00005CD020005CD020005CD020005CD0200E6
:10CB000005CD020005CD020005CD020005CD0200D5
:10CB100069CA0200BBF1200FA6D0C6E7BBF15B0FCC
:10CB2000C3D1002046F001FC044601261CE0BBF105
:10CB3000740F69D032D8BBF1660F48D0BBF16E0FCD
:10CB4000B3D19DF85C30752BAFD1284651F083F9F5
:10CB50006C28AAD1284651F07EF96C28A5D1284628
:10CB600051F079F900260E24002F40F0FD80204678
:10CB700020F0ACFE8046002E40F00C81BAF1000F90
:10CB800000F02481002C90D0059B002B8DD107A8AC
:10CB900051F024FE204629B0BDE8F08FBBF17B0F99
:10CBA00000F0DE80BBF17D0F7FF47FAF002F3FF4FC
:10CBB0007CAF059B002B00F01481013B069A059386
:10CBC00052F82370384620F081FE80464CE79DF8ED
:10CBD0005C30612B7FF469AF284651F03CF96C283A
:10CBE0007FF463AF284651F036F973287FF45DAFC8
:10CBF000284651F030F965287FF457AF284651F0A8
:10CC00002AF900261E24AFE79DF85C30722B7FF4D2
:10CC10004CAF284651F01FF975287FF446AF2846DF
:10CC200051F019F965287FF440AF284651F013F907
:10CC300000263E2498E7002308939DF85C10002905
:10CC40003FF433AF222909D1284651F004F9DDE938
:10CC5000081021F0EFFD0026044685E75C290CD181
:10CC6000284651F0F8F87528014606D86D2808D8EE
:10CC700062283ED0662808BF0C2107A851F040FD6D
:10CC800033E0A0F16E03072BF7D801A252F823F08E
:10CC9000B1CC02007BCC02007BCC02007BCC02003A
:10CCA000B5CC02007BCC0200B9CC0200BDCC0200A6
:10CCB0000A21E2E70D21E0E70921DEE7042600244E
:10CCC000284651F0C8F840F02000C0B2A0F130036F
:10CCD000DBB2092B84BF5738C3B2013E43EA0414C8
:10CCE000EED1214607A851F012FD284651F0B3F8C5
:10CCF000A3E70821C1E700BF502F08000FDE07009F
:10CD00002D1E080000240894594607A851F0F8FC8D
:10CD10009DF85CB0BBF12E0F18D00BF0DF03452B54
:10CD200014D0BBF12B0F12D0BBF12D0F0FD05846F2
:10CD300037F0FCFA064650B9DDE908105CB1009600
:10CD40003346324623F05AF804460DE701242846BC
:10CD500051F081F8D8E733460A2223F0ADF9F3E722
:10CD6000002048F047F9DFE6214B984514D12146D1
:10CD7000384648F0AAF8002E3FF476AE069BDBB9A1
:10CD8000012103A821F042FB069B1F60204620F0F2
:10CD90009DFD8046274667E6B9F1000F04D1002EBD
:10CDA0007FF483AEA1465FE649462246384647F007
:10CDB000C0FD4FF00009DEE7394603A848F085F8CA
:10CDC000E4E73C46DAE6284651F045F89DF85C6019
:10CDD000304637F0BFFA0028F5D1002E3FF4D2AE2E
:10CDE00063E63C46BAF1000F7FF4D1AEEEE700BF38
:10CDF000F4300800C20713B5044603D5C0F347005A
:10CE000002B010BD830707D102680E4B9A4203D1CE
:10CE100020F04AFDC0B2F3E7204621F051FA48B1B4
:10CE2000204620F0BBFCFCEEC07ACDED017A9DF8E7
:10CE30000400E5E7204620F049FD5E22C188024853
:10CE400023F0EEFBB4F60700AF0F08002DE9F3471F
:10CE50001D46DDE90A98837C5B4288F80030CB07E9
:10CE600007460C46164611D411F0030A03D10A688E
:10CE7000384B9A4206D0204621F022FA78B3BAF114
:10CE8000000F24D12268334B9A4220D1204620F053
:10CE90000BFD0314337003122B7089F80000BB7C68
:10CEA000002B4ED13A7B042A4BD17A7C002A48D001
:10CEB00032782978914244D199F800208A4201BF02
:10CEC00088F8002033702B7089F8003039E0204654
:10CED00020F064FCFDEEC07A17EE900AD9E701AAB3
:10CEE0006946204620F020FC04220321009840F2ED
:10CEF000DE231BF011FE019B1868FFF77BFF019BEF
:10CF000030705868FFF776FF019B28709868FFF72C
:10CF100071FF009B89F80000032BC0D9019BDC68DE
:10CF2000204621F0CDF978B1204620F037FCDFED26
:10CF30000A7A20EE270AFCEEC07A17EE903A88F8BB
:10CF4000003002B0BDE8F087204620F0ADFC88F844
:10CF50000000F6E7B4F6070000007F432DE9F0413A
:10CF6000314ECCB031238DF8083073880124B3F5ED
:10CF70007F7F07468DF809400DD3002402222B48FD
:10CF80000094234602A98DF8092008F079FC204678
:10CF90004CB0BDE8F081022102A800F0E7FA054696
:10CFA00008B10024F3E7B6F8028008F10403BB429D
:10CFB000EDD814F051FC311D04AA08F801500746C1
:10CFC00044F023FD044650B99DF81C30184913F075
:10CFD000100F14D11649384644F0BFFD044638F00E
:10CFE0001BFDB4B9002311480093022202A908F0E6
:10CFF00047FC002CD5D10D4808F02AFCC7E70D4AA4
:10D000001368526803A81B1A9A4206D838F004FD28
:10D01000022402238DF80930E4E7384634F04AFE52
:10D0200004460028DBD1D5E7F85601201C55012025
:10D03000FC560120C06101202DE9F04F0746E1B008
:10D0400059483FF079FE061E09DB584C6588B5F556
:10D050007F7F06D340F25123238030F079FE0025F4
:10D060003EE02B1DBB4200F29D8014F0F5FB271D16
:10D070006A1E04A9D35D2F2B4FF000030CBFBB54D5
:10D080007B554B4A44F0BAFA40F2511347F8043C3E
:10D090000027C4E90177E760054618B103236370F0
:10D0A0003046DAE718A904A844F095FBAA46D8B19F
:10D0B000002104A8DFF800B144F08DFB4FF0000917
:10D0C000C4F808A0CA451AD104A843F09AFF002367
:10D0D000A268638030466260E360A36130F038FE8E
:10D0E000284661B0BDE8F08F9DF87A30002BDFD084
:10D0F00018A904A844F06FFB0AF1010AD7E718A9A0
:10D1000004A844F068FBBDF86A30BDF86810C4F8A4
:10D11000049003F01F025200480A0192C3F3441224
:10D120000092DB0A01F01F0200F2BC70C1F3431150
:10D1300050F06BFB1F4B0022C01842F10001A0FB16
:10D140000B030BFB0133C4E904039DF86C3013F0AF
:10D15000100314BF0123E3600DF17A000DBF189B8B
:10D16000E360A261A36150F0C5F86080804630465C
:10D1700030F0EEFD0027B84502D809F10109A1E71A
:10D18000A8EB0702042A4FF000030DF17A0128BF33
:10D190000422394404480093039208F071FB039A77
:10D1A0001744E8E701259BE71C550120F8560120AC
:10D1B000FC56012080436D3800CA9A3B70B52A4B5B
:10D1C0001D682A4B1B681A68012151641B68284A94
:10D1D000D3F84465002352F8044B14B121798142FD
:10D1E00032D00133082BF6D170BD6369A269EB1A06
:10D1F000B21AC3EB034313444FF6FE714FF6FF72AE
:10D200008B4288BF1346E289218A89B211FA82F2E1
:10D21000A189B2FBF1F001FB1022A16821F81230C4
:10D22000238AA2899BB2934204D2238A01339BB200
:10D23000238216E0E3899BB20133B3FBF2F102FBD8
:10D2400011339BB2E3810CE0E379002BCDD04DF09C
:10D2500072FA6379003818BF0120834201D000239D
:10D26000E3716561A661BFE7A464012050660120F7
:10D27000184601202DE9FF414368DB6853F821502F
:10D2800004460F4640F28740294648F0CFF806464C
:10D2900000284ED0436828469847B36801A95B68C8
:10D2A00080469847B36805469B68002140469847EA
:10D2B00063682449DB6853F8270047F0FAFA06460A
:10D2C00090B1B0F93820B0F93C309A4233D001A97E
:10D2D000383042F01EFC012596F850306FF30413ED
:10D2E00086F850300023B36263681749DB6853F84F
:10D2F000270047F0DEFA064638B101A911F01EFCFE
:10D3000000210546304643F0FEF97DB194F82A30FD
:10D31000DB0704F1180210D4114601A842F0F9FB12
:10D3200094F82A3043F0010384F82A3004B0BDE8B1
:10D33000F0810546BCE70025CEE701A9104642F082
:10D340000FFCEDE7C46908008C650800F8B5194BBF
:10D3500000241C70184BFF271F70184F0D461646EF
:10D3600000F01CFE00230022DFF85CC0C7E90023A8
:10D370002146234620469D420DD158B191ED017AB8
:10D38000DFED0F7A67EE277A17EE900AFAF7D0F9F9
:10D39000C7E90001F8BD56F82320940708D11468A6
:10D3A000644505D110B1074823F046F91146012024
:10D3B0000133E0E7B86C0120C86C0120680A012045
:10D3C00000007A44A50608007C4008002DE9F843D7
:10D3D00090F82A309B0704462ED4BDE8F883DB681A
:10D3E00053F8267040F28740394648F01FF805464A
:10D3F00068B1436838469847AB6804F108019B68F8
:10D400009847013663689A689642E8D3E5E7414653
:10D41000384647F04EFA20B104F1080143F0BCFB56
:10D42000EFE74946384647F044FA0028E9D004F1CE
:10D43000080143F068F9E4E7DFF80880DFF80890B6
:10D440000026DFE7C46908008C65080090F95030B9
:10D45000214930B5002B836AB4BF428A028AB0F9F1
:10D460000C408589002B08BF0B46224494B29A7B5E
:10D47000C2B193F905105A8811FB05F1114409B2A4
:10D48000A0F8461093F905205B8812FB04F21344C0
:10D490001BB29942D2BFA0F84A30A0F84A10A0F8B7
:10D4A000463030BD93F904101A8811FB05F1114480
:10D4B00009B2A0F8441093F904201B8812FB04F26F
:10D4C00013441BB29942D2BFA0F84830A0F84810CC
:10D4D000A0F84430E5E700BF9005012090F95030F6
:10D4E000214930B5002B836AB4BF028A428AB0F961
:10D4F0000E40C589002B08BF0B46224494B29A7B8C
:10D50000C2B193F904101A8811FB05F1114409B254
:10D51000A0F8441093F904201B8812FB04F2134472
:10D520001BB29942D2BFA0F84830A0F84810A0F82A
:10D53000443030BD93F905105A8811FB05F11144B0
:10D5400009B2A0F8461093F905205B8812FB04F29B
:10D5500013441BB29942D2BFA0F84A30A0F84A1037
:10D56000A0F84630E5E700BF9005012013B50C4B4D
:10D570001C780A4644B10B4B1B7843B10A490B781F
:10D580002BB901220A701C46204602B010BD0523AB
:10D590004370002301460093044808F071F9F3E753
:10D5A0008A6C0120C50501202F6B01201C5501202C
:10D5B00008B510EE103A23F00042B2F17E5FF0EEB3
:10D5C000405A10D308D19FED300A9FED306A002BEE
:10D5D000A8BFB0EE460A08BD70EE405ADFED2B7AC8
:10D5E00087EEA50AF7E7B2F17C5F11D2B2F14A5F8C
:10D5F0009FED276A44D920EE000AFDF707F9DFED19
:10D60000257AE0EE657A35EEE70A36EE400AE2E783
:10D61000002BB7EE000AF6EE007A14DA35EE800A37
:10D620009FED1D6A20EE270AF1EEC05AFDF7EEF8D5
:10D63000A0EE256A9FED160A75EE865A30EE650A51
:10D6400030EE000AC7E730EE650A20EE270AB1EE99
:10D65000C05AB0EE407A15EE103A23F47F6323F0FF
:10D660000F0306EE103AA6EE467A75EE067AC7EE7E
:10D67000275AFDF7CBF8E0EE055A36EE250ADFE72C
:10D68000B0EE460AA7E700BFDA0F494000000000ED
:10D69000DA0FC93F6821A2336821A2B308B510EEA2
:10D6A000103A23F000425B00F0EE407A0FD4B7EE60
:10D6B000000A77EEC07ABDE8084037EEA77AA7EEF9
:10D6C000A77AB1EEC70A37EE800A1AF013B8B2F1A2
:10D6D0008B4F13D2FFEE006AE0EE006ABDE808400F
:10D6E000B1EEE67AF7EE006A37EE007A86EE870A48
:10D6F000B0EE007A97EE870A1AF0A8B81AF0A6F8EA
:10D70000DFED027A30EE270A08BD00BF1872313F04
:10D7100070B588B00D460C2000211646039345F0E5
:10D7200088FF0D4B036005AB01930C4B039A0093EC
:10D73000044603233146284646F09EF99DF81830EA
:10D74000059A626023729DF81C3013B1204606F0E2
:10D7500065FF204608B070BD203D08003418090060
:10D7600010B58EB003AB51F8044B0193194B0093E5
:10D77000013803231BF03EF940F2A341606806AA7A
:10D780001EF0B8FE237A5B0043F001030893039B6D
:10D79000099340F626130A93049B5B0043F00103B0
:10D7A0000B93059B6FF0004293421FBF40F2E6428D
:10D7B0005B000C9243F0010314BF0221012106AA71
:10D7C0004FF0020018BF0D9346F0CAFA0E200EB0BB
:10D7D00010BD00BFB417090010B58EB003AB51F8EF
:10D7E000044B0193194B0093013803231BF002F9FA
:10D7F00040F2CB51606806AA1EF07CFE237A5B00E3
:10D8000043F001030893039B099340F626130A9300
:10D81000049B5B0043F001030B93059B6FF00042F8
:10D8200093421FBF40F2E6425B000C9243F00103BB
:10D8300014BF0221012106AA4FF0020018BF0D9368
:10D8400046F08EFA0E200EB010BD00BF7C18090005
:10D8500010B596B003AB51F8044B01932D4B0093D8
:10D86000013806231BF0C6F809AA606840F2CC51C3
:10D870001EF040FE237A5B0043F001030B93039BF1
:10D880000C93049B0D9344F216530E93059B5B007F
:10D8900043F001030F93069B6FF00042934235D093
:10D8A0005B0043F0010344F2F64211931092092306
:10D8B000032116AA02EB830243F6F63042F8340C39
:10D8C00016AA02EB8300079A520042F0010240F8C8
:10D8D000302C089A6FF00040824210D016A800EB5E
:10D8E000830043F6D63440F82C4C16A800EB830393
:10D8F000520042F00102013143F8282CC9B209AAB2
:10D90000032046F02DFA0E2016B010BD0723022189
:10D91000CFE700BF4C180900F0B58DB00D461820B8
:10D9200000211646039345F084FE194B036005ABB6
:10D930000193184B039A0093044607233146284667
:10D9400046F09AF8069D144940F2D12228461BF071
:10D9500007F9089E059F9DF824009DF828109DF862
:10D960002C209DF81C302073C4E901760698617361
:10D97000A2732561237540B1002201213FF0EFFB26
:10D98000022802D1054822F0FFFD20460DB0F0BD6F
:10D99000E03D0800CC170900445E0800FC060800C2
:10D9A0002DE9F341044601F134000E4602F078FD02
:10D9B0002388102B05D0112B3FD0002002B0BDE8EA
:10D9C000F0812F4D002388224FF6FF7102FB03F7F1
:10D9D000785B884203D00133052BF7D104238822DA
:10D9E0005343A188E952EA184FF000080E2307F1CB
:10D9F0006000D3652844234982F85A80A2F87680D3
:10DA0000EA1903F0B9FDC6F81880206961696C371E
:10DA10003D4403C568464EF023FBBDF80030228A22
:10DA20009A4202D8628A9A4203D2A08869464EF08E
:10DA300005FB0023F3600120C0E7A388104F0025F9
:10DA4000882202FB05F1C85B984203D00135052D01
:10DA5000F7D1042539440B4803F0A4FD88235D4326
:10DA60007A194FF6FF737B53002382F85A30D26D38
:10DA70000E2A1EBF5360217A1172B361DBE700BF2B
:10DA800038060120A5B203002DE9F04F044614F03A
:10DA900003058BB00846164603D122682E4B9A42E6
:10DAA00003D02E48F72122F0BBFD012203A91EF06E
:10DAB00083F83046022269461EF07EF8049E019AE1
:10DAC0003146204638F0BEFC03990098324645F0B6
:10DAD00077FE94F80C31022BDDE900780BD0062B91
:10DAE00034D0012B03D1211D3846FAF77DFF0E20DB
:10DAF0000BB0BDE8F08F04F104090DF1280AF434ED
:10DB0000A84507EB050BF2D906AA5B460BF1100EF0
:10DB10001646186859689446ACE803000833734504
:10DB20006246F6D149465846FAF75EFF2146584606
:10DB30003BF03DFB2246334603CB5345106051601A
:10DB40001E4602F10802F6D11035D9E742463946A1
:10DB5000201D3BF0CBF9CAE7383E08003802080028
:10DB60002DE9F043044614F0030587B00846164635
:10DB700003D12268264B9A4203D02648F72122F08F
:10DB80004FFD012203A91EF017F830460222694614
:10DB90001EF012F8049E019A3146204638F052FCDD
:10DBA00032460399009845F00BFE94F80C31022B95
:10DBB000DDE900690BD0062B24D0012B03D1211DF8
:10DBC0003046FAF74BFA0E2007B0BDE8F08304F1B7
:10DBD0000408F4342146A94506EB050708D801F1ED
:10DBE000100351F8042B44F8042B9942F9D1EAE7C9
:10DBF00038463BF0DCFA41463846FAF72FFA103542
:10DC00003946E8E74A463146201D3BF06FF9DAE72E
:10DC1000383E08003802080008B5830703D10268BF
:10DC2000064B9A4203D00648F72122F0F9FC90F8FF
:10DC30000C01400040F0010008BD00BF383E080064
:10DC400038020800F0B58BB0084611461A4605ABFD
:10DC50000193224B0093052345F00EFF00214FF462
:10DC60008A7045F0E6FC1E4B0360044601220598CD
:10DC700002A91DF0A1FF039E26F00803102B04D07B
:10DC8000202E02D0174822F0C3FC069D029F022DD1
:10DC900011DC002D11DD079888B90023089AC4F81B
:10DCA0001021204684F80C51324639463EF0DEFA07
:10DCB00020460BB0F0BD062DEDD00B48E3E7012266
:10DCC00002A946F088FB0028E7D0039B102B03D065
:10DCD0000648102122F0A4FC029BDFE794180900FB
:10DCE000383E08001E040800CD0708005F03080046
:10DCF0002DE9FF410C46D1F80080064601226068FC
:10DD000001A91DF059FFDDE9017517B9124822F08C
:10DD100093FC25F00803102B04D0202D02D00F48CF
:10DD200022F076FC022E0CD90122A06801A91DF078
:10DD300043FFDDE90132102A04D00948102122F006
:10DD40006FFC002340462A4639463EF08FFA0E20EB
:10DD500004B0BDE8F08100BF660508001E0408009D
:10DD60005F03080010B50446A307084603D12268E4
:10DD70000A4B9A4203D00A48F72122F051FC1FF0C7
:10DD800055FD022805DC002805DD84F80C010E2075
:10DD900010BD0628F9D0034822F03AFC383E0800AE
:10DDA00038020800CD0708001FB5084611461A467C
:10DDB00003AB0193034B0093012345F05DFE00206C
:10DDC00022F0E2FBC41809002DE9804885B002AFBB
:10DDD0003B1D0193224B0093054601230E46002074
:10DDE0001AF008FE3146284638F00AFCD7F80490AD
:10DDF000DFF87CB0484620F0D3FA4FEA60084FEADB
:10DE00008803073323F00703ADEB030D0DF1080A78
:10DE10000024444505D1CCB1124840F27E4122F0A5
:10DE2000BBFB6100042241F00101484621F0AAFB3E
:10DE3000830702D102685A4504D00B4840F23911D9
:10DE400022F0EEFB4AF824000134E2E729460120E3
:10DE50003246FFF77BFA0548214647F074FB00BFC6
:10DE6000BC180900F2210800380208000419090052
:10DE7000445E080070B50E460546002844D038F0D0
:10DE8000BFFB324629460020FFF760FA00F02AFA6D
:10DE900000231A4634F01AF91C4B5C6A94BB3EF01E
:10DEA00005FA78B3FEF73EFD012818D002280BD101
:10DEB000174A234656F82340A10702D12168914210
:10DEC00003D001339D42F5D10E24204630F0F0F905
:10DED00000F0DEF8204630F0EBF9204670BD0D4B27
:10DEE0000D491A78234656F82340A00706D120682A
:10DEF000884203D1606800799042E6D001339D42A8
:10DF0000F1D1E1E70E24E3E70E24E6E7C06101204A
:10DF10007C400800C86C0120A83F080070B588B09C
:10DF20000D460C2000211646039345F082FB124B50
:10DF3000036004AB0193114B039A00933146042311
:10DF40000446284645F098FD049850F0C5F99DF820
:10DF500018109DF814209DF81C3011B1084822F0CB
:10DF60006BFB01792F2901D94DF0B8FB6060204689
:10DF70002272637208B070BDA83F0800CC18090077
:10DF8000E923080010B5044C23781BB90DF000F903
:10DF90000123237010BD00BF726C01202DE9F04FEA
:10DFA000354BD3E900C7354BD3E9008E344BD3E969
:10DFB000006387B00024CDE90244019302EB8103A2
:10DFC000059004934FF0FF314FF00109049B9342F9
:10DFD00018D1029B13B1294BC3E9008E039B13B1E7
:10DFE000254BC3E900C71CB1254B019A1E605A603E
:10DFF00001313DD0059B002B35D107B0BDE8F04F76
:10E000000DF0C6B852F8040B8307DFD103681D4D2D
:10E01000AB42DBD1436890F808B01979A1F1200335
:10E02000C1F1200A29FA0AFA09FA03F343EA0A03BA
:10E0300009FA01FABBF1000F0FD04AEA080843EAD7
:10E040000E0ECDF808B0407A0028BFD0019C1C43CA
:10E0500001944AEA06060446B8E701254AEA0C0C90
:10E060001F430395EFE7084A00231360074A137024
:10E0700007B0BDE8F08F00BF500A0120400A012020
:10E08000600A0120A83F0800B8640120726C0120DA
:10E09000F8B5394C394D636823F47F0323F47F438B
:10E0A000AB4223D04FF48072002104F1080045F008
:10E0B000C7FB334A0023137023704FF080434FF4A3
:10E0C0004032C3F80429C3F81429C3F82429C3F83B
:10E0D0003429C3F84429C3F85429C3F86429C3F880
:10E0E00074294FF47C12C3F884296560254E264DAF
:10E0F0000024D5E90001D6E90023C4F1200702433A
:10E100000B430120A4F1200100FA01F120FA07F7E6
:10E110003943A04002400B40134308D0E0B22DF039
:10E12000DFFF204627F0AAFC204627F095FD0134AA
:10E13000402CDED11549164800220023C6E90023F1
:10E14000C5E90023C1E900234FF40033C0F8483388
:10E15000D0F80423920308D5C0F80833D0F844312E
:10E160001BB14FF4A2714CF085FA0A4B002000213C
:10E17000C3E90001F8BD00BFC86C0120AF0000ADCD
:10E18000B86C0120400A0120500A0120600A0120D9
:10E1900000400240680A0120F0B50D4687B0002615
:10E1A0001446002A60D011F0030760D10A68424B80
:10E1B0009A425CD16A464FF4807047F0A4FA10B9D5
:10E1C0003E4822F0E1F9DDE90035042CA5EB03051A
:10E1D00036D0A30732D12368394A934208D0394A4E
:10E1E000934205D0384A934202D0384A934225D10F
:10E1F000012203A920461DF0DFFC049BAB4202D0A4
:10E20000334822F019FA9DF81410039C0022402094
:10E210001AF0C6FC012801D02E48F2E7009B5A19DB
:10E22000B2F5807F02D92C4822F0E0F92B482A462B
:10E230002146184445F0C4FA0E2415E02848C0E7EA
:10E240003946284645F0F5F9009B5A19B2F5807F0A
:10E25000044604D821492A46194445F0B1FA21461A
:10E26000284620F049F90446204607B0F0BD2A466A
:10E27000006800234FF480711DF0A8FC042C0546B3
:10E2800000F1010708D1B7F5807F9CBF134BC65C36
:10E29000740044F00104E7E720461FF0C7FA422368
:10E2A000FF22002104461AF00BFCB7F5807FBAD894
:10E2B0000A4BEC54C0E700BF78320800DB1A0800B4
:10E2C0002C370800502F08006C310800F4F40700C8
:10E2D0001F0808006A2108005E0B0800D06C0120AE
:10E2E000560E080038B5084BD3E9004554EA05033B
:10E2F00005D04FF0F1F8201A65EB010138BD4FF061
:10E30000FF300146FAE700BF680A012070B52DED25
:10E31000028B8AB00D46082000211646039345F073
:10E3200088F9304B036005AB01932F4B039A0093A0
:10E33000044602232846314645F09EFBDDE90505EB
:10E34000B0F10E0218BF0122B5F10E0318BF012370
:10E350009A4202D1254822F06FF90E2838D01FF0DA
:10E360001DFAB0EE408A4FF0B7F8F9F733F9DFED58
:10E37000207A07EE100A0E2DC7EE278A21D00698C4
:10E380001FF0E2FE05462EF0A7FB07A932F036F992
:10E390009DF8223001939DF8213000939DF81F20B5
:10E3A0009DF820309DF81E10BDF81C0034F0DAFAFC
:10E3B000104B281A034407EE903AB8EEE78A38EE7D
:10E3C000288AB4EEE88AF1EE10FA04D50A48C2E7CA
:10E3D0009FED0A8AC7E7204684ED018A0AB0BDECAA
:10E3E000028B70BD7C400800EC1809007208080020
:10E3F00000007A4480BC92C7450A08000000000073
:10E400007FB50C46082000211546039345F011F90D
:10E41000084B036005AB0193074B039A0093294611
:10E420000123204645F028FB05984FF055FF0020BA
:10E4300022F0AAF8F0400800FC18090008B5054BC6
:10E440001B682BB1044A934202D0044822F0CEF854
:10E45000004808BDE00801209C360800670A080053
:10E4600008B5064BD3F8C0302BB1054A934202D011
:10E47000044822F0BBF8014808BD00BFE0080120B5
:10E480009C360800710A08002DE9F843DFF8D4C073
:10E49000DCF800500446BDB1686805F1080320F0BF
:10E4A00003000344DFF8C0802B48D8F80060002E3A
:10E4B00014BFB6468646671C04BFAEEB0304083C97
:10E4C00024B90020BDE8F883244BEBE7A007F8D17E
:10E4D000002914BF3046284644F0010908BB04F166
:10E4E0000807AEEB0300B84220DA002914BF284623
:10E4F000304644F0010350BB002AE2D0184DD5F855
:10E500008431002BDDD00121384645F09EF80028EB
:10E51000D7D0D5F8D4300360C5F8D40044F0020455
:10E520000EE047684F4509D00068D7E751B127F0A2
:10E530000300AEEB0000C8F800000660002AEDD131
:10E540004460BFE71D601846CCF80030F6E741682C
:10E550009942F3D00068CEE700000420D06D01207E
:10E56000C0610120F05D0120E45D012070B58AB03A
:10E570006846F8F745FD124C124E134D241A3068C8
:10E5800000F580600022012120443CF053F8A8B936
:10E590000246012104F5C8403CF04CF84FF4C0435A
:10E5A0000A4A2B600368136053F8042C084922F0D0
:10E5B00003020A60074A1A600AB070BD3368EFE7C9
:10E5C0000000042054020120FC5A0120E8640120CC
:10E5D000E4640120EF2978010A4B1A6852B10A4B12
:10E5E000002808BF1A460023D158814204D10648AA
:10E5F00018447047044AF6E70433382BF4D100205E
:10E60000704700BFA0640120DC55012038B51C46CE
:10E61000084611464FF002121AF0BCF920684FF07C
:10E620005BFE00210446082045F003F8074B036019
:10E63000637905460BB94DF051F820794CF022F87A
:10E64000207905F0BDFD6C60284638BD7841080092
:10E6500008B540683DF04BFB004808BD3233D3C0DD
:10E6600037B5054640683DF042FB314A4FF6FF732F
:10E67000ADF806300323C2F8F03501210023C2F8BB
:10E68000F435C2F8001519461A0102F1804202F56C
:10E69000E0420133082BC2F81415C2F81015F3D16B
:10E6A000234C4FF49053C4F818356B685B79C4F869
:10E6B0001435C4F810350DF10603C4F82C360123C7
:10E6C000C4F830362360D4F80031002BFBD0184852
:10E6D0004FF480714BF0CEFF01236360144CD4F8EB
:10E6E0000431002BFBD012484FF482714BF0C2FF73
:10E6F0000123A360D4F81431002BFBD00C484FF455
:10E700008A714BF0B7FF0023C4F80035BDF906202D
:10E710009A42B8BFADF80630BDF90630181340EA8A
:10E72000830080B2400040F0010003B030BD00BF64
:10E73000007000401C4608B5084611464FF0021212
:10E740001AF028F920684FF0C7FD0021042044F09A
:10E7500070FF034B03604FF48671024821F01CFFE9
:10E76000F0410800F22108002DE9F04F2DED088B53
:10E770008FB009AB01936F4B009305231AF03AF960
:10E780000021099824F072FD002106460A9824F021
:10E790006DFD044600210B9824F068FDE379012B00
:10E7A00005460AD1C379012B07D1A268012A04D9F1
:10E7B0008368012B01D99A4202D05F4821F03CFFC7
:10E7C0006621B0684BF0BFFDE769217904903846B7
:10E7D00002914BF02EFDA368A0690299013B00FB5A
:10E7E0000370B0EE40BA4BF024FD0C98EF690E2890
:10E7F000F0EE40BA26D1297938464BF01AFD0D9833
:10E800000E28F0EE408A20D1A868AB69297901383A
:10E8100003FB00704BF00DFDE3690293EB6903937A
:10E82000049BD6F81CB0D3F81C90B0EE409A4FF081
:10E83000000AB36853450BD804980FB0BDEC088BA1
:10E84000BDE8F08F1EF0AAFFD9E71EF0A7FFE3E7AF
:10E85000584631794BF0EDFCB369B4EEC0BAF1EE35
:10E8600010FAB0EE408A9B4406DDC9ED008A0AF139
:10E87000010A09F10409DCE7F4EEC0BAF1EE10FA7E
:10E8800002D589ED009AF2E7A7680023013FA2694B
:10E890002179A7EB0308B8F1010F34D8029807914A
:10E8A00002FB0300CDE905234BF0C3FC059A029B54
:10E8B000079902FB0730F0EE40AA4BF0BAFC039B2D
:10E8C000D5F81880297905911A46069B08FB032084
:10E8D000F0EE409A4BF0ADFC039B059907FB083026
:10E8E000B0EE40AA4BF0A5FC38EE6A8A30EE4A0A38
:10E8F00079EEEA9A28EE008A88EE290A30EE0AAA12
:10E9000089ED00AAB3E7CDE9061303EB5808029B93
:10E91000059202FB08304BF08CFCB4EEC08AF1EE9D
:10E9200010FADDE90521079B01D94346AFE74746C9
:10E93000AFE700BFE4350900431608002DE9F047B2
:10E940002DED048B86B003AB0193504B0093032352
:10E950001AF050F80398002124F088FC8368012BFA
:10E96000044640F29180C579012D02D0484821F03B
:10E9700063FE007924F0EEFC81460498E6690E28D7
:10E980005CD0002124F072FCC779012F054603D129
:10E99000A26883689A4201D03E48E8E700799FED7B
:10E9A0003E8A24F0D7FC82463046D5F81C80C84702
:10E9B000A36940461E44F0EE408AD047AB69B0EEF2
:10E9C000409A9844A368BB4218D8A368013B07EE5D
:10E9D000903AB6EE000AF8EE677A28EE008A67EE03
:10E9E000887A17EE900A20F0030040F00200A0F1B0
:10E9F000FF4006B0BDEC048BBDE8F0873046C84749
:10EA0000A3694046F0EE409A1E44D04778EEA98AAA
:10EA100030EE499AF0EE486AD9EE286AAB6907EE03
:10EA2000907AB8EE677A9844C6EE877A0137B0EEEE
:10EA3000409A38EE278AF0EE698AC3E70598DFED41
:10EA4000168A1EF0ABFE3046B0EE408AC847A66874
:10EA5000B0EE409AAE4202D828EE888AB5E72A4640
:10EA60002179E0694BF0ACFB07EE905A39EE009A41
:10EA7000B8EE677A39EE689A0135C9EE077AB0EEDA
:10EA8000409A78EEA78AE5E70448B2E7CC3509005A
:10EA9000251F0800151F08000000000002008080EC
:10EAA0001E280CD03E280AD010F0010307D182079F
:10EAB00007D10068044BC31A5842584170470120DF
:10EAC00070471846704700BFB4F60700F0B51B2822
:10EAD0008DB006460C46154672D03CD80E2800F084
:10EAE000988004D8042840F2B180002430E0102837
:10EAF000FBD115F0010206D115F00303F5D1296809
:10EB00006E4A9142F1D128461EF090FE0122054640
:10EB100009A9204600F04EF9102E0A9F3DD1217917
:10EB2000002240201AF03CF8A3686B4300FB03F17D
:10EB3000E06844F099FDA368E0606B43A3606368FC
:10EB40006FF31F2363601DB1013DC319002F34D142
:10EB500020460DB0F0BD1D28CBD02428C5D1012200
:10EB600003A9284645F037FC00285CD0A10712D144
:10EB70002268534B9A420ED1012209A9204600F087
:10EB800019F901230093DDE90901DDE9032343F0CD
:10EB900015FD002858D11E24DAE7A1689DF82C0045
:10EBA000694300F05FF9C3680446CFE71846099946
:10EBB0003A4644F005FE03463B44013DF6D2C7E722
:10EBC00009A90122204600F0F5F806A928460122ED
:10EBD0001CF0F2FF9DF82C100022402019F0E0FFFD
:10EBE000A168079EB6FBF0F6054631449DF82C005F
:10EBF00000F038F90446DDE90912C06844F0E0FD90
:10EC0000E0680A9B069906FB05F2184444F0D8FD1B
:10EC10009EE70A682B4B9A423FF467AF294620468D
:10EC20003BF0C9FD94E7EA0702D5002021F0ACFCD7
:10EC3000AB0703D12A68214B9A42F6D028461FF031
:10EC40003FFB0028A7D0F0E73E2481E7012209A975
:10EC5000204600F0AFF8012206A9284645F0BBFB8C
:10EC6000002898D00B9A012A21D05A2A21DC203280
:10EC70000146089B012B1ED05A2B01DC2033014694
:10EC80009342D2D123F00203642BCED0022E01D0C6
:10EC90000029CAD0079B0093DDE90912069B304684
:10ECA00046F09BFC00280CBF1E243E2450E7422265
:10ECB000DDE70021DDE74223E0E700BFB4F607000F
:10ECC000502F08006C3108002DE9F043012885B071
:10ECD00006460F4608D08B0728D10B68274A934277
:10ECE00002D0274A934221D1012201A9384645F09A
:10ECF00072FBD8B131460022402019F051FF029B2F
:10ED0000B3FBF0F100FB01F5AB4202D01D4821F04E
:10ED100093FC304600F0A6F8019904462A46C068E4
:10ED200044F04EFD204605B0BDE8F08338461FF0A4
:10ED300047FB054600B145102946304600F092F8E1
:10ED40000021044638461CF09BFF4FF000080746A0
:10ED500038461DF025F903460028E3D025B91946A9
:10ED600020463BF0F2FCF3E74246E16808F1010976
:10ED700030461AF0C3FAC846EAE700BFF4F40700C9
:10ED8000502F0800610F0800012807B50B4606D177
:10ED90000B68009340F61623019302206B46014650
:10EDA0000022034820F0E0FA03B05DF804FB00BF46
:10EDB00028F7070070B50D460179044601F07F0180
:10EDC00016464020002219F0EBFEE3682B60A26893
:10EDD00042436A60227902F07F02AA602168094AF0
:10EDE00091420BD194F90420002A01DBB20707D429
:10EDF0006268C2F3172200FB02332B60002070BD53
:10EE00000120FCE76C310800074BC1E9003000230A
:10EE1000C1E90233054B02689A4202BF4368C3F35B
:10EE200017238B6008467047B83708006C3108001C
:10EE300038B50D461C4611462846094A19F0AAFD68
:10EE4000206820F075FA012D007804D1BDE8384023
:10EE5000002100F007B86168BDE83840FFF734BF13
:10EE6000040002007828F8B505460E4602D1114884
:10EE700021F0E2FB00220146402019F091FE002122
:10EE80000746102044F0D5FB0B4A0C4B0571012DB1
:10EE900018BF1346036043686FF31F230446C0E99D
:10EEA0000136002106FB07F044F0C3FBE06020467A
:10EEB000F8BD00BFEF0E08002C370800502F0800E7
:10EEC000F8B50A79012A05460C460DD1194946F0D4
:10EED00090FAD4E90221284621F094FF28461649E9
:10EEE000BDE8F84046F085BA144946F092FAA368A6
:10EEF000002BF3D01249134F284646F07AFA002629
:10EF0000A368B34204D81049284646F072FAE5E7F0
:10EF10001EB13946284646F06CFA3246E16820793F
:10EF200019F018FF0122014628461FF093FD013613
:10EF3000E6E700BFE8360800A0170900F43608002D
:10EF4000FF360800F12D0900D32D09002DE9F04707
:10EF5000044688B00D4616460AB90025BCE011F0FB
:10EF600003078068DFF8049240F0CC800B68794A90
:10EF7000934240F0C78002AA46F0C5FB10B976481C
:10EF800021F002FB2179042E01F07F013A464FF077
:10EF9000400000F0898019F003FE16F003020546D8
:10EFA0004ED137680192384646F03AFD6B4B019AD4
:10EFB000834238D13179402001F07F0119F0F0FD12
:10EFC000A84202D0664821F037FB33684B45D6E9AA
:10EFD000028A04D17368C3F3172305FB03AADDE992
:10EFE00002072368E6683F1A4B45A8EB070729D1BB
:10EFF00094F90430002BB0DA002FE3D16368C3F337
:10F00000172305FB036605FB08F2514605FB00606C
:10F0100044F0FEFB0399A2680298521A40446A43E6
:10F0200005FB016131E04F4B9F4209D1012DC9D150
:10F030002A4605A930461CF0BFFDDDE905A8CEE74C
:10F0400049489DE7002FDEDD6368B7EB132F0BD92E
:10F05000A16839443046694344F006FB6368E060C8
:10F0600067F31F23064663600298A2680399404431
:10F070003A44121A6A4301FB056105FB006044F043
:10F08000C7FB029805FB08F2514605FB006044F0FF
:10F09000BFFB6368C7EB132262F31F236360A3689F
:10F0A0003B44A3600E2517E019F07AFD23684B4519
:10F0B000064615D13946102044F0BBFA054694E8BF
:10F0C0000F0085E80F00029A02EB112363F31F2162
:10F0D0006960039B9B1AAB60284608B0BDE8F087C7
:10F0E000DDE902312079C91AFFF7BCFEDDE9023201
:10F0F000E168D21A0546724306FB0311C06844F06A
:10F100005FFBE9E700232A46014620681CF05EFD0C
:10F1100023684B45024611D16368042E00EB13228D
:10F120000ED094F90430002BBFF617AF2079E168B8
:10F13000334600F07F001AF0E1F8B3E7042EF5D172
:10F140002079E16800F07F0008B0BDE8F04719F0D1
:10F1500001BE00BF78320800DB1A08004DEF020044
:10F16000B1170800F4F40700560E08006C310800CF
:10F1700010EE102A08B522F00043B3F17E5FB0EE26
:10F18000406A12D319BF76EE467A9FED1F7ADFED03
:10F190001F7A9FED1F7A12BF87EE276AE0EE077A8B
:10F1A000B0EE676AB0EE460A08BDB3F17C5F0BD2E1
:10F1B000A3F50003B3F1645FF4D320EE000AFBF77C
:10F1C00025FBA0EE066AEDE7B0EEC06AB7EE000AD6
:10F1D00030EE466AB6EE000A26EE000AB1EEC06ACC
:10F1E000FBF714FB002AF0EE007AA0EE066A9FED12
:10F1F000090AA6EE270A9FED066A36EE406AB8BFF6
:10F20000B1EE466ACEE700BF0000000000008003B8
:10F21000DA0FC93F6821A2B31FB58DED010A019B2A
:10F2200023F00042B2F18B4F00EE102A4FEAD37068
:10F230000BD318F00BFBDFED1E7A30EE270A08B176
:10F24000B1EE400A05B05DF804FB5B0014D5B7EEE3
:10F25000007AF0EE476AE0EE006AF1EEE67A77EEC9
:10F26000807AC7EE276AF0EE007AE0EE276AB0EE09
:10F27000660A18F0EBFAE2E7B2F1665F10D320EE0F
:10F28000007AF7EE006A37EE266AF1EEC67A77EE7C
:10F29000A67AC7EE276A36EE800A18F02BFACEE778
:10F2A000DFED047A70EE277ACDED037A039BC6E793
:10F2B0001872313F0000807B1FB5044690B10E28C4
:10F2C00010D000793EF0A4F960B94FF4F6730393BF
:10F2D00001A9204603AB02AA14F0DAFE0399024802
:10F2E00021F0B2F904B010BDA4000800F4EE400A09
:10F2F000F1EE10FA10B5F0EE407A04D770EE207AF5
:10F30000B0EE670A10BD10EE902AB2F17E5F10EEEB
:10F31000103A03D1BDE8104000F080B8940F04F01B
:10F32000020444EAD37433F0004308D1022C59D0CC
:10F330009FED317A032C08BFF0EE477AE0E732F018
:10F34000004209D1DFED2D7A9FED2D0A14F0010F57
:10F3500018BFF0EE407AD3E7B2F1FF4F10D1B3F10E
:10F36000FF4F04F1FF3407D1022C3ED8254B03EBAD
:10F370008404D4ED007AC3E7022C39D8224BF6E797
:10F3800002F150619942DDD3B3F1FF4FDAD0A1070A
:10F3900003D503F1506393420CD387EEA00AB0EE7D
:10F3A000C00A00F03BF8012CF0EE407A04D1F1EEF7
:10F3B000407AA5E7DFED157A022C0AD0002C9FD009
:10F3C0009FED130A77EE807A9FED120A77EEC07AEE
:10F3D00096E79FED0F0A77EE807A9FED0E0A70EEAA
:10F3E000677A8DE7DFED0B7A8AE7DFED0B7A87E747
:10F3F000DFED067A84E700BFDB0F49C0DB0FC93FB2
:10F40000DB0FC9BFD42B0900E02B0900000000006E
:10F410002EBDBB33DB0F4940DB0F493F10EE102AF6
:10F4200022F00043B3F1994F82B04FEAD2700ED36D
:10F43000B4EE400AF1EE10FA07D69FED410ADFED77
:10F44000417A002808BFB0EE670A02B070473E4913
:10F450008B420BD8B3F1665F5AD212F0FF4FF4D152
:10F4600060EE007ACDED017A019BEEE7374A9342D8
:10F47000F0EEC07A37D8A2F5D002934229D8F0EE48
:10F48000006ABFEE007AA7EEA67A002377EEA67A8E
:10F4900087EE270A5A1C60EE006A9FED2D6ADFEDA9
:10F4A0002D7ADFED2D5A26EEA67AE7EE067A9FED4D
:10F4B0002B6AA7EE876ADFED2A7AE7EE257A67EEF8
:10F4C000877AE6EE267A60EE277A24D130EE670A54
:10F4D000BBE7B7EE007A77EEC76A77EE877A01234B
:10F4E00086EEA70AD6E71F4A93420BD8F7EE086AC2
:10F4F000B7EE007AA7EEA67A022337EEE66A86EE2A
:10F50000070AC7E7BFEE007A87EE270A0323C1E7A1
:10F510004FF0FF33BEE7144A144902EB830201EBBC
:10F52000830393ED007A77EEC77A37EEC00AD2ED07
:10F53000007A37EEC00A002887D0B1EE400A84E78F
:10F54000DA0FC9BFDA0FC93FFFFFDF3EFFFF973F6A
:10F5500025AC7C3D0DF5113E4712DABDA9AAAA3EA5
:10F5600098CA4CBEFFFF1B40EC2B0900FC2B090086
:10F57000F0B50023DFF838C00C4E19460E27DCF832
:10F580000020934201D30E20F0BD346804EB031237
:10F590004FEA031E9568854208BF44F80E1003F138
:10F5A000010304BFC2E90117D160E8E71C5601203E
:10F5B000245601202DE9F04387B0084611461A462B
:10F5C00002AB0193284B0093042344F055FA0298B0
:10F5D0004EF082FE804603984EF07EFE0746049869
:10F5E0004EF07AFE00210646282044F032F81F4BE8
:10F5F00003601F4B9DF814901D68044615B11D480B
:10F6000020F0F4FF186098F8040004F0D9FD387970
:10F6100004F0D6FD307904F0D3FD174B98F80420A0
:10F6200084F82120C3F864253A7984F82220C3F8AD
:10F630006825327984F82320C3F870250122C3F8A5
:10F640000455C3F80855C3F80C25C3F81025C3F8B2
:10F650001C25C3F82055C3F8249531F04BFE2046F5
:10F6600007B0BDE8F08300BF20190900704308000F
:10F67000E85D0120B10108000050024010B50446C9
:10F6800090F823003CF02DFB0A4BD3F8082142B13F
:10F6900094F826206FF3410284F826200022C3F854
:10F6A000082194F8263013F0020F14BF3E201E20CC
:10F6B00010BD00BF0050024010B5044690F8230072
:10F6C0003CF00FFB0C4BD3F8082142B194F82620F4
:10F6D0006FF3410284F826200022C3F8082194F831
:10F6E00026309A0701D400F009F843F0080384F8A3
:10F6F00026300E2010BD00BF0050024008B5014862
:10F7000020F074FF1E0608002DE9F04F2DED028B4E
:10F710000D4689B055F8044B0392064694F8230031
:10F720003CF0DFFA06AB0193754B039A0093294630
:10F730000223701E19F05EF9724B069DD3F8082162
:10F740009DF81C1042B194F826206FF3410284F812
:10F7500026200022C3F8082194F8263098070BD5FC
:10F76000684A0123536094F8263043F0040384F878
:10F7700026302023C2F8083394F82630656061F300
:10F78000041384F8263028463BF049FD08EE100AA1
:10F7900028463BF0F7FC04F12403C00884F8250058
:10F7A000019305AB00930DF112020DF1130301213A
:10F7B00028463BF012FD9DF813309DF81220514F62
:10F7C0005149DFF84C915B0143EA821394F82620FB
:10F7D00003F0600322F06002134384F8263094F8AB
:10F7E0002530013B18BF0123C7F81C3594F824309D
:10F7F0005A1E534253410022C7F82835B7EE007A0B
:10F80000104690461646D7F81C35012B01D18B794E
:10F810004BB33E4DF8EE486A4FF0000CB1F904309E
:10F8200099FBF3FE6B689EFBF3F307EE903AF8EE5C
:10F83000E77AD5F800B0D1F800A076EEE77A0CF1BF
:10F84000010CF0EEE77A87EEA66A0835B4EEC76AD7
:10F85000F1EE10FA41BFB0EE467A1A465846D0464D
:10F86000BCF10B0FDAD10136092E01F10801CAD122
:10F87000244DC5F81885C5F8140594F8240094F8AB
:10F880002530628313FB00F318EE100A5843000181
:10F890004FF47A73B0FBF3F0033020F0030080B232
:10F8A0002083002143F0C5FE0021A060208B43F09F
:10F8B000C0FEE06060683BF0A4FC0023C4E90433B0
:10F8C00084F8203094F8263023F00E0343F002032E
:10F8D000204684F8263014F0A1FE238B9B08C5F83F
:10F8E00050352023C5F804330123C5F800352B60BB
:10F8F00014F076FE0E2009B0BDEC028BBDE8F08F4F
:10F900004019090000500240A819090050190900C7
:10F910000048E80110B5044690F823003CF0E1F9F6
:10F92000064A0123536094F8263043F0040384F818
:10F9300026302023C2F808330E2010BD00500240AC
:10F9400038B5084B1B6800220446C3F80025FF2584
:10F9500000792CF0C5FB607925712CF0C1FB657135
:10F960000E2038BD580201202DE9F0432DED028B09
:10F970008BB0084611461A4603AB01933D4B0093EA
:10F98000072344F079F803984EF0A6FC0646049845
:10F990004EF0A2FC00210546082043F04AFE364BFB
:10F9A00003609DF81870DDF814807A07044602D0D1
:10F9B000324820F041FE089B5B0701D03048F8E751
:10F9C00009989DF81C9088B11DF0E8FEB5EEC00ABC
:10F9D000F1EE10FAB0EE408A06D4F7EE007AB4EEFB
:10F9E000E70AF1EE10FA03DD2648E2E79FED268AEA
:10F9F000307904F0E5FB287904F0E2FB84F8069006
:10FA0000327922712B796371B8F57A5F01D01F4882
:10FA1000CFE7102F01D01E48CBE71E4B9FED1E0AEB
:10FA20001B681E49C3F840256279C3F8442528EEB7
:10FA3000008A4FF00462C3F804250022C3F8202591
:10FA4000FCEEC87A2822C3F81825C3F81C25012229
:10FA5000C3F8002517EE900AC3F86015C3F86425B3
:10FA60001A601CF04FF920460BB0BDEC028BBDE8CC
:10FA7000F08300BFF019090028440800F4210800B1
:10FA8000E506080076040800AE47E13DCC1A080000
:10FA9000BF1A08005802012000007A440C5B0120C4
:10FAA00038B5084B0C681B680022C3F80025207984
:10FAB000FF252CF015FB607925712CF011FB657189
:10FAC0000E2038BD580201202DE9FF4105460E46A3
:10FAD0002B79FF2B104601D12BF00CFC40F2EE31BC
:10FAE00019F04EF840F2EE320021044643F0E6FFF2
:10FAF000B30706D132682F4B9A4202D12E4820F02C
:10FB000043FD022201A9304644F065FC00284FD095
:10FB10009DF80C10029E0022402019F041F8B6FB1F
:10FB2000F0F0A04202D2254820F086FD039B482B2E
:10FB300001D02348F8E7DFF89480019ED8F8003020
:10FB40000122C3F80825C3F86065C3F864451D4B5E
:10FB50004FF4485043F001039847D8F80030002292
:10FB6000C3F80821184AC3F8602501223746C3F8B4
:10FB70006425D8F80030D3F808316BB106EB4406A1
:10FB8000B7420CD1AB7983B124F00104640044F096
:10FB9000010004B0BDE8F08100F0A2FCE9E73B8879
:10FBA000A3F5004327F8023BEAE724F00304EDE75E
:10FBB0000E20EEE7788608007C23080096010800F6
:10FBC0000F120800401A09000C5B012058020120A6
:10FBD00070B588B0084611461A4605AB01931C4B18
:10FBE0000093032343F048FF0021142043F021FD3C
:10FBF000184B036004460122059802A91BF0DCFFA4
:10FC0000049B622B10D0A3F168014A424A4123F0C1
:10FC1000200148290AD0422918D0012B07D00E48CC
:10FC200040F2BB2120F010FD0122F0E702239DF8F5
:10FC300018000799039D029EA073DB0020466660B2
:10FC400023736273A560216108B070BD0123EEE7E4
:10FC5000281A0900F44408002B0A0800F0B51E46D3
:10FC60000F4685B011463846204A18F093FE346896
:10FC70001F4B2340062B05D0A3070AD122681D4B3A
:10FC80009A4206D121461C4844F6E61244F05DF83B
:10FC900004460021402043F0CCFC184B036014F0D4
:10FCA0000302054603D12168154B994202D015483D
:10FCB00020F0AEFC012F16D97068022201A91BF0BA
:10FCC0007BFF40F2BB230298019E4FF48062082123
:10FCD00018F022FF034628463246214604F0B6FDBE
:10FCE000284605B0F0BD13461646F4E704000200AE
:10FCF0000F0080FF28F7070050330800F045080088
:10FD000078860800171308002DE9F04788B00846E8
:10FD100011461A4602AB0193374B0093062343F07A
:10FD2000ABFE40F2B753FF220121029818F0C8FE43
:10FD300040F2CD23054602220498012118F0C0FEAE
:10FD4000DDF81C80B8F1000F064604DC40F2E74104
:10FD5000012018F0ADFE059F082F04D0102F02D00F
:10FD6000264820F069FC05F10B000021800043F0DB
:10FD700060FC234B0360044603989DF818A0C0085C
:10FD80008000E060002143F054FC5FFA85F9FFB287
:10FD9000F6B2606018B9A060E06817F0D7FDE068BF
:10FDA000002143F046FCA06008B96060F4E72774C6
:10FDB00084F8249004F12C07DFF84890E674C4F826
:10FDC000148084F812A00026B846AE4209DB94F8ED
:10FDD000240041461EF0B0FDA062204608B0BDE8F8
:10FDE000F08700231A461946484600F061F80136AC
:10FDF00047F8040B4460E8E7481A0900FD0E0800C4
:10FE0000FC460800FC1B090070B50D4688B055F88B
:10FE1000044B0392064620463BF0B3FF05AB01932B
:10FE20000E4B039A009329460323701E18F0E2FD3F
:10FE300094F824209DF818309A4203D840F2B65026
:10FE400018F0D0FD04EB83049DF81C20E06A0599AE
:10FE500004F0A8FD0E2008B070BD00BFF81A09001C
:10FE600070B50D4686B055F8044B03920646204601
:10FE70003BF087FF05AB01930C4B039A0093294697
:10FE80000123701E18F0B6FD94F824209DF814305C
:10FE90009A4203D840F2B65018F0A4FD04EB830454
:10FEA0000022E36A0E209A6006B070BDB81A0900FD
:10FEB00008B508461146002218F06CFD00211C20F0
:10FEC00043F0B7FB034A0260002282604FF4004215
:10FED000028308BDFC1B09001FB502AB51F8044B9F
:10FEE0000193074B00930138022318F083FD20464D
:10FEF0009DF80C20029904F055FD0E2004B010BDB1
:10FF0000101B09001FB503AB0193134B51F8044BB1
:10FF100000930138012318F06DFD03981DF03EFC9D
:10FF2000F7EE007AB4EEE70AF1EE10FA04DCB5EE73
:10FF3000C00AF1EE10FA02D5084820F07DFBDFED93
:10FF4000087A20EE270A0E20BCEEC00A10EE103A06
:10FF5000238304B010BD00BF781A0900A21708005F
:10FF6000000000471FB503AB0193064B51F8044B4B
:10FF700000930138012318F03DFD00230E20A360FB
:10FF800004B010BDC01A090073B58669069D044609
:10FF90001EB92E60022002B070BD0029016B2960DD
:10FFA00090F93F1008BF00228A4212D190F9401008
:10FFB00000EB810112B2496A01EB42021A60FF2391
:10FFC00080F83F302A68436C03EB520343640120FE
:10FFD000E1E790F83C10B1FA81F1490980F83C1052
:10FFE00080F84010C2F1010200EB810180F83F204F
:10FFF0004E6A1E6043F0AFFC204643F08FFC38B9D8
:020000023000CC
:10000000286094F83E30002B14BF00200220C2E785
:10001000D4E90713A2696068C91A1A4401910092D1
:10002000334601AA6946F8F7BFFDE369019A9B1AB6
:10003000236210B100202860ADE72A68636C03EBEF
:1000400052036364204643F086FC204643F066FC7E
:10005000236AB3F5007F054606D3044B04F108007C
:10006000C4E9023400F01CFA284694E7653A070018
:10007000F0B51E460F4685B0114638461B4A18F0AB
:1000800089FC34681A4B2340062B05D0A3070AD1FC
:100090002268184B9A4206D12146174844F6E612C8
:1000A00043F053FE04460021482043F0C2FA134BAC
:1000B000036014F00302054603D12168104B9942F6
:1000C00002D0104820F0A4FA012F0DD90222706846
:1000D00001A91BF071FDDDE901232846214604F04A
:1000E000B3FC284605B0F0BD1346F6E70400020055
:1000F0000F0080FF28F7070050330800D0480800A1
:10010000788608001713080038B50446406A3BF0AB
:1001100020FE94F83C00236B9FED120A04EB800450
:100120005D08626A23F001031344934210D14CF03E
:1001300088FC07EE905AF8EEE77AC0EE277A17EEC1
:10014000900A20F0030040F00200A0F1FF4038BD0B
:1001500032F9021B07EE901AF8EEE77AA7EEA70A2B
:10016000E3E700BF0000000013B50446406A0191B8
:100170003BF0EFFD0199064844F6E61243F0E5FD39
:100180000146204604F0ACFC0E2002B010BD00BFBA
:100190005033080038B50C460546406A3BF0D9FD9F
:1001A000A30703D12268064B9A4202D0054820F0EB
:1001B0002FFA2846214604F093FC0E2038BD00BFDC
:1001C0007886080017130800F0B587B00846114676
:1001D0001A4603AB01932D4B0093032343F04CFCD1
:1001E00003984EF079F8074604984EF07DF8002108
:1001F0000646242043F01DFA254B0360254BBDF82D
:100200001450D3F8002512F00102044617D003F56C
:10021000A043D3F80015C80711D503F58053D3F8D0
:100220000025D1070AD503F53043D3F80025D207BE
:100230002AD500231848A36020F0D8F902221749D4
:10024000A3608A5C22770022C3F80C25A3680122F0
:10025000C3F81025A2683B792376C2F86035387957
:1002600003F0AEFF3EB1A26833796376C2F8683519
:10027000307903F0A5FFA3682D0A01222046A5824C
:10028000C3F8002507B0F0BD0322D8E7801A0900A3
:10029000F449080000C0014014210800A614090018
:1002A00070B50D4688B055F8044B03920646A06819
:1002B0003BF04AFD06AB0193574B0093701E294655
:1002C000039A022318F096FB2046069D9DF81C60B9
:1002D0003CF051F810B120463CF058F8656084F8C5
:1002E000206028463AF09BFF064628463AF04AFF2F
:1002F0000DF11303C008E076019305AB2846009387
:1003000004F1220204F1210300213AF066FF28469D
:100310003AF044FF059DA076B5F5803F05D340F245
:10032000BB214FF6FF7018F0E7FBAD000021284617
:1003300043F07FF994F82210E06019B9284643F0A1
:1003400078F9206106F574452335B5FBF6F506FB13
:1003500005F35D0805F5740505F51055B5FBF3F5D6
:100360006A08A16802F5740303F51053B3FBF5F2B4
:1003700002EB5602B2FBF6F3013BC1F84835A26826
:10038000C2F828356B1EE382A368C3F80855A3683A
:100390000122C3F8142560683AF033FF1F4A002396
:1003A000114652F8040B90BB41F8234030F0A2FFF5
:1003B000A36800250422A5772046C3F80022294619
:1003C00041F0BAFFA368D3F82025C3F84025A368FD
:1003D000D3F82425C3F84425A368C3F80851A368BB
:1003E000C3F80C51A368C3F81051A368C3F81451A3
:1003F000A368C3F80451A3680C22C3F80423A268BD
:1004000001230E2093606377E57708B070BD013358
:10041000042BC6D1CCE700BFC81A0900C055012083
:1004200010B50C4C206888B10B4B1B687BB94DF0A4
:100430004FF823689842236836BFDB43C01AC018C0
:1004400040F2EE23984294BF0020012010BD00200E
:10045000FCE700BFEC5D01201456012008B50B4BF2
:100460001B6893B90A4B1B787BB14DF031F8094BEF
:1004700018601A6812B91A6801321A60064B012214
:100480001A70064B03F154025A6208BD145601203B
:10049000286C0120EC5D01202A6B0120C061012045
:1004A00010B5044606F010FEE3681BB90A4A11684D
:1004B000A14203D1BDE8104006F018BEA360074B6F
:1004C0001968E160196809B119688C60116801B98F
:1004D00014601C60EEE700BF205601202856012062
:1004E000F7B5134E33680BB3124D06F0EDFD2C78C3
:1004F00024B103B0BDE8F04006F0F8BD0E4A012378
:100500002B703368346014600BB92B70F1E7D3E9BA
:1005100000609F680190C3E9024406F0E7FD0EB158
:100520000198B04706F0D0FD3B46EDE703B0F0BDC3
:1005300020560120506C01202856012008B51DF0DE
:10054000C5F9C188034897290CBF4222972220F0A1
:1005500067F800BFC20F08000749002251F8323087
:10056000834203D801EBC202506870470132002B6E
:10057000F4D11846704700BFA8130900F0B587B042
:10058000084611461A4602AB0193204B0093042300
:1005900043F072FA02984DF09FFE074603984DF023
:1005A0009BFE00210646202043F043F8184B0360D1
:1005B000DDE904238361174B9A4288BF012300F1D0
:1005C000040598BFB3FBF2F304464361394628465D
:1005D0003CF05FFD48B904F10C07314638463CF069
:1005E00058FD28B128463BF06BFE204607B0F0BD11
:1005F0000122114628463CF0B2FD01221146384640
:100600003CF0ADFD20464CF015FBEEE7D81A090092
:10061000984A080020A1070070B50C4688B054F82D
:10062000045B0392064628463BF0B1FB28463BF0AC
:10063000BAFB04AB0193094B039A00932146701E49
:10064000042318F0D7F9079B00932846DDE905231A
:1006500004992BF0E5F80E2008B070BD581B090076
:1006600070B50C4688B054F8045B039206462846E1
:100670003BF08DFB28463BF096FB04AB01930A4B05
:10068000039A00932146701E042318F0B3F9012346
:100690000193079B00932846DDE9052304994EF05A
:1006A0006DFA0E2008B070BD981A090070B50C469E
:1006B0008CB054F8045B0392064628463BF067FB77
:1006C00028463BF070FB05AB01930E4B039A009359
:1006D0002146701E072318F08DF900230193099B12
:1006E0000093DDE90512089B28464EF047FA0B9B64
:1006F000009328460A9B079A05992BF091F80E2043
:100700000CB070BD201B090070B50C4688B054F8C1
:10071000045B0392064628463BF03FFB28463BF02D
:1007200052FB04AB01931D4B039A00932146701EAC
:10073000042318F05FF940F2754301220021059867
:1007400018F0BEF940F267430122002104460698E2
:1007500018F0B6F940F2AB230922082106460798A3
:1007600018F0AEF904990E4AB2FBF1F301FB132223
:100770008AB9EB6104F0010495F8203006F0010617
:10078000A40044EAC60423F00C031C430E2085F8A1
:10079000204008B070BD0133EBE700BF681C0900C2
:1007A00020A107002DE9F04186B0084611461A46FF
:1007B00003AB0193344B0093032343F05DF903989B
:1007C0004DF08AFD804604984DF08EFD0646059852
:1007D0004DF08AFD00210746242042F02AFF0546FD
:1007E0002A4B45F8043B0446414628463CF051FC60
:1007F000024620B140F2D72125481FF025FF94F88A
:1008000020102846C1F380013CF0A9FCBEB104F1E0
:100810000C08314640463CF03CFC024628B12846D4
:100820003BF04EFD40F22B41E6E794F8203043F0D8
:100830000203014684F8203040463CF090FCB7B1FA
:10084000394604F114003CF024FC50B128463BF03A
:1008500037FD1EB104F10C003BF032FD40F21E41A9
:10086000CAE794F8203043F0010384F820300523D0
:10087000E36194F82030204623F00C0384F8203004
:1008800006B0BDE8F08100BF181C0900904B0800BD
:10089000940208002DE9F04F0D468FB055F8044B37
:1008A0000392064620463BF078FA20463BF08BFA4E
:1008B0000AAB0193434B039A0093701E042329460D
:1008C00018F098F80A98022207A91BF075F90B9BFB
:1008D00006930C99089B059305AA06A849F0B5FE56
:1008E000059E002E54D09DF83430039394F82030A8
:1008F000DF07DDE9065802D433481FF09DFE980754
:10090000E76903D5206900213CF016FC454405EB5E
:10091000060804F1140B039E4FF0080A4FF000097B
:1009200094F82030990703D52069F1093CF004FCC4
:1009300094F820100A072FD4384625F095F894F83B
:100940002010A068C1F3800181F0010101F00101D4
:100950003CF0F2FB58463CF0B1FB94F8201040EA22
:1009600049000B075FFA80F923D4384625F07CF85C
:1009700094F82010A068C1F380013CF0DDFB760004
:10098000BAF1010AF6B2CBD105F8019BA845C2D154
:100990000E200FB0BDE8F08FC1F3800181F001019E
:1009A000A06801F001013CF0C7FB384625F05CF877
:1009B000D0E7A068C1F380013CF0BEFB384625F0CB
:1009C00053F8DCE7301C0900230508002DE9F0434B
:1009D0000D468DB055F8044B0392064620463BF079
:1009E000DCF920463BF0EFF909AB0193354B039A54
:1009F000009329460323701E17F0FCFF099801227B
:100A000006A91BF0D9F80A9B05930B99079B049341
:100A100004AA05A849F019FE049FBFB394F820204A
:100A20009207DDE9053502D427481FF005FE1D4475
:100A3000D4F81C802F4415F8016B4FF00809F10918
:100A400020693CF079FB94F820100B0722D4404633
:100A500025F00AF894F82010A068C1F3800181F015
:100A6000010101F001013CF067FB404624F0FCFF6E
:100A700094F82010A068C1F380013CF05DFB760083
:100A8000B9F10109F6B2DAD1BD42D4D10E200DB0D0
:100A9000BDE8F083C1F3800181F00101A06801F09D
:100AA00001013CF049FB404624F0DEFF94F82010A1
:100AB000A068C1F380013CF03FFB404624F0D4FF26
:100AC000DDE700BF501C09002C0508002DE9F04FA0
:100AD0000D4695B055F8044B0392064620463BF070
:100AE0005CF920463BF06FF90EAB01934A4B039A39
:100AF000009329460623701E17F07CFF0E980122F2
:100B00000BA91BF059F8109B1199079306AA0C9B8F
:100B1000069307A849F099FD0F98022208A91BF037
:100B20004BF8129B059304AA099B1399049305A8FB
:100B300049F08BFD069B049A934202D037481FF080
:100B40007BFDB3B194F820200B98059D9707DDE954
:100B5000071601D5D70701D43148F0E73544EB1823
:100B6000E769039300EB010804F1140B039B9D421A
:100B700003D10E2015B0BDE8F08F18F8016B4FF0CF
:100B8000080A4FF00009F10920693CF0D5FA94F801
:100B900020100A072AD4384624F066FF94F8201063
:100BA000A068C1F3800181F0010101F001013CF076
:100BB000C3FA58463CF082FA94F8201040EA490003
:100BC0000B075FFA80F91ED4384624F04DFF94F8E5
:100BD0002010A068C1F380013CF0AEFA7600BAF1B3
:100BE000010AF6B2CFD105F8019BBFE7C1F380013E
:100BF00081F00101A06801F001013CF09DFA384646
:100C000024F032FFD5E7A068C1F380013CF094FAEC
:100C1000384624F029FFE1E7881C0900440F08004A
:100C2000B42308002DE9F0410E2A064686B0084696
:100C3000174602D130481FF083FC8A0706D10968A5
:100C40002E4A914202D12E481FF09EFCC30716D5B2
:100C5000B488431093FBF4F504FB15339CB2ADB29A
:100C6000042F2AB20FFA84F820D1414630463CF0D6
:100C700013FB400040F0010006B0BDE8F08103AA7C
:100C800002211CF07BFD039B18681CF0CFFD039B29
:100C900084B258681CF0CAFDB388A34285B202D959
:100CA000F388AB42DCD817481FF05AFC3846019253
:100CB0001CF0BCFDB37B019A30FA03F3074602D067
:100CC00011481FF0B9FC03A9304601340135ADF8D5
:100CD0000E2001920593ADF80C80ADF81040ADF8F0
:100CE00012500CF0B9FD3046019A3B4641463EF0A9
:100CF00074FF0E20C0E700BF2823080078320800E8
:100D00002F080800BF1B0800CE1B08002DE9F04F7C
:100D10002DED028B91B00AAB0193A14B00930623FA
:100D200017F068FE9F490A9840F21E3217F018FF2C
:100D30009C4940F2265204460B9817F011FF99493E
:100D4000804640F227520C9817F00AFF81460E9811
:100D50000E2825D01CF022FDF0EE408A0F980E28B8
:100D600021D1B7EE008A38EE688A0D998E480AF0D4
:100D7000F5FC6268D8F804309A425FFA80FA0CD128
:100D8000A37B98F80E10994207D1D9F804108A4233
:100D900003D199F80E209A420AD084481FF04CFCE7
:100DA000F6EE008ADAE71CF0F9FCB0EE408ADCE7E8
:100DB0000AF1FF32082A0ED8DFE802F0090D090D0A
:100DC000090D090D0500082B07D07948E6E7102B1F
:100DD00003D07848E2E77848E0E7A388ADF8203010
:100DE0000026E388079607A92046ADF82230099629
:100DF0000CF032FDF0EE687AFEEECC7ABAF1090F13
:100E000017EE907AF0EE487AFEEECC7A17EE905A12
:100E10003ED132464FF67F761AE0A089B8F80CC072
:100E2000B9F80CE002FB00F3A06800EB8300D8F8EF
:100E3000083002FB0CFC03EB8C0CD9F8083002FBE9
:100E40000EFE03EB8E0E0021A388994209DB0132CE
:100E5000E3889A42E1DB0E2011B0BDEC028BBDE8C5
:100E6000F08F1EF801301CF801A06B4307FB0A331A
:100E7000B3420BDC13F1800A48BF03F27F1A4FEA3A
:100E80002A2323EAE37343540131DDE7FF23FAE722
:100E90000AF0FB0303933246E3889A42DBDAA18926
:100EA000A368B9F80CB0514303EB8103B8F80C10F8
:100EB0000493D8F80830514303EB81030593D9F824
:100EC000083002FB0BFB03EB8B0B4FF0000AA388EF
:100ED0009A4501DB0132DFE7059B3BF81A1033F836
:100EE0001A60039B032B03D176BA49BAB6B289B212
:100EF00001F47843314806F4784C6B4307FB0C331C
:100F0000834244DA13F5F84348BFFF331B1223EA48
:100F1000E37303F4784301F4FC6C294806F4FC6E97
:100F200005FB0CFC07FB0ECE864533DC1EF57C7CF6
:100F300048BF0EF2EF4C4FEA2C2C2CEAEC7C0CF460
:100F4000FC6C01F01F01694306F01F0607FB061643
:100F500041F6F0718E4220DC16F10F0148BF06F514
:100F60008771091221EAE17143EA0C0C039B4CEAF8
:100F7000010C032B1FFA8CFC03D19CFA9CFC1FFA7A
:100F80008CFC049B23F81AC00AF1010A9FE74FF476
:100F90007843C0E74FF4FC6CD3E71F21E4E700BFC0
:100FA000501D090024600800A46108000022080008
:100FB000D0020800EA020800FF0B08000085F700D5
:100FC0000FDD07002DE9F04F97B00FAB0193484BB1
:100FD0000093072317F00EFD46490F9840F2A9220F
:100FE00017F0BEFD0122044609A910981AF0E4FD8D
:100FF000139E149DDDE9118A721C08BFA6886B1C24
:1010000008BFE588B8F1000F0CDBBAF1000F09DB6F
:10101000464507DB554505DBA388B34202DBE38881
:10102000AB4202DA34481FF09BFAA5EB0A039DF8A5
:101030002C10A6EB0807002240205F4317F0B0FDFC
:101040000A9BB3FBF0F9159B04900E2B039307D07A
:1010500018461CF0EBFB05904F4504D92748E2E702
:1010600000230593F8E7A37B099F4FF0010909FAD4
:1010700003F909F1FF330693D1464D4534D10023DE
:1010800020460CA9ADF83080ADF832A0ADF8346040
:10109000ADF836500E930CF0DFFB0E2017B0BDE814
:1010A000F08F049B022B19D0042B1AD017F8013BA8
:1010B00003990E2902D00599994208D00699079202
:1010C0000B4020460FFA8BF13EF087FD079A0BF19B
:1010D000010B5E45E5D109F10109CEE737F8023B86
:1010E000E6E757F8043BE3E7C3460FFA89F2F0E777
:1010F000101E090024600800BF1B080042150800EC
:1011000030B589B004AB0193244B0093042317F04E
:1011100071FC2349059840F2255217F021FD40F259
:101120001E321F490446049817F01AFD0799054618
:101130001C480AF013FB0699C3B21B4803930AF03C
:101140000DFB6968039BC2B26068884202D01748F1
:101150001FF05EFAA97B102903D0012901D01448A1
:10116000F6E7511E082910D8DFE801F0050F050F3A
:10117000050F050F0A00A17B102908D00D48E7E7ED
:10118000A17B082903D00C48E2E70C48E0E7284699
:10119000214603F0E7FC0E2009B030BD481E0900CF
:1011A00024600800104C0800A4610800F50E080037
:1011B000811D08009F1D0800AE1D0800F21F0800D9
:1011C00030B589B003AB01931A4B0093052317F098
:1011D00011FC1949039840F21E3217F0C1FC817BC3
:1011E000069B01228A40934202D314481FF024FA3E
:1011F000079C6FF000418C4203D0A24201D81048F6
:10120000F4E7BDF91010BDF91420002902DB858830
:10121000A94201DB0B48E9E7002AFBDBC588AA42AB
:10122000F8DAA34202D000943BF0C2F80E2009B0D5
:1012300030BD00BFB01D0900246008005620080022
:10124000D40E0800991B080070B588B002AB01935A
:10125000174B0093062317F0CDFB0298079D827B66
:10126000012393409D4202D312481FF0E5F9BDF9D6
:101270000C10BDF91020BDF91430BDF9184000293B
:10128000F2DB002BF0DB002AEEDB002CECDB8688A7
:10129000B142E9DA9E42E7DDC688B242E4DAA6420C
:1012A000E2DDCDE900453BF081F90E2008B070BDCC
:1012B000801D0900991B0800F0B58FB008AB0193A1
:1012C000274B0093062317F095FB089E0D9FB37BD9
:1012D00001229A40974202D322481FF0ADF90998A3
:1012E000BDF92810BDF92C20BDF93030ADF808004B
:1012F000002402A8ADF80A10ADF80C20ADF80E30AD
:1013000004943EF0C3FBB388ADF8183002AAF3880A
:10131000059405A91046ADF81A3007943EF0C7FBB6
:1013200002A930460CF098FABDF90840BDF90C301E
:10133000A34202DC0E200FB0F0BDBDF90A50BDF98A
:101340000E30AB4202DC013424B2EFE72A463B46C2
:101350002146304601353EF040FC2DB2EFE700BF9C
:10136000201D0900991B08002DE9F0432DED028B8B
:101370009FB011AB0193474B00930D2317F03AFB3D
:10138000DDE91145A27BAB7B9A4202D242481FF0B5
:1013900053F9A188139849084CF0D4FFE188064618
:1013A000490814984CF0CEFFA988074649081798B9
:1013B0004CF0C8FFE9888046490818984CF0C2FFF5
:1013C0000FAB02930DF13E030193169B1599009309
:1013D0000DF1420210AB814620464CF01FFF0DABD1
:1013E00002930DF1360301931A9B00932846199935
:1013F0000EAB0DF13A024CF011FF1B980E2842D0B3
:101400001CF0CCF9F0EE408A1C980E2808D01CF095
:10141000C5F9B5EEC00AF1EE10FAB0EE408A01D57A
:10142000B7EE008A1D980E2830D01CF0FFF900227C
:10143000BDF934300993BDF936300893BDF9383021
:101440000793BDF93A30CDE90593BDF93C300293DD
:10145000BDF93E300193BDF940300093CDE90A0259
:10146000CDE903582046BDF94230F0EE480AB0EE0F
:10147000680A3A4631463BF04BF90E201FB0BDECEE
:10148000028BBDE8F083DFED058ABDE70122002075
:10149000CEE700BFB81C0900761D08000000000060
:1014A00030B58DB005AB01931F4B0093072317F0A8
:1014B000A1FA1E49059840F2A92217F051FB089C99
:1014C0000699631E012B05D9042C03D01848214628
:1014D0001FF0BAF8079B022B1FDC002B20DD9DF8C4
:1014E0002C2002929DF8282001929DF82420009241
:1014F000224603F06BFC0E200DB030BD0122AA4045
:101500000C4D1540002DEAD1D20209D5012CE6D0B0
:101510000948182221461FF097F81D1F1C2DEDD9F0
:1015200006481946D4E700BFD81D0900246008000A
:1015300099160800111000108516080062160800A0
:1015400038B50C4BD3F8DC3004460D464BB90121BD
:101550000C2042F06EF82A462146BDE8384000F0E3
:101560000BB89A68A24202D15A68AA4201D01B68FD
:10157000ECE738BDC061012070B5094CD4F8DC50EF
:101580002B462BB9C0E900528160C4F8DC0070BD65
:101590009E688E4202D15E689642F8D01B68F0E7E2
:1015A000C061012030B5094A52F8DC3F4BB19C685C
:1015B00084421C6806D15D688D4203D1146000220C
:1015C0001A6030BD1A462346F0E700BFC061012013
:1015D00008B5074B187838B1064843682BB13BF083
:1015E00046FB003818BF012008BD1846FCE700BFC5
:1015F000236B0120F854012008B50348012103F0B2
:10160000B1FD0E2008BD00BFAC5601201FB502ABD6
:1016100001930B4B009304310223013817F0EAF9D0
:10162000084902984FF41D7217F09AFA044603987D
:101630001CF0B4F8204603F0D5FC04B010BD00BF88
:101640005C160900A84E080013B5012103F08AFDBD
:1016500068464AF0E5FC3AF0BEFB00210C2041F060
:10166000E8FF064B03609DF800200DF101015208D0
:1016700004463BF09FFA204602B010BDA84E080079
:101680002DE9F0410646806986B0F8B9114D04464F
:1016900007464FF6FF782B8843450DD0EB6D0E2B98
:1016A00003D1284600F078FCE86506AB03EB840321
:1016B000EA6D43F8142C01340137052F05F1880534
:1016C000E9D101A920461DF037F9B06106B0BDE8A7
:1016D000F08100BF3806012008B501481EF054FF14
:1016E0000C23080010B50C4686B0A068012203A99F
:1016F00042F071FE88B19DF80430227962F347030D
:101700008DF80430039B1A68CDF805209B88ADF84E
:10171000093001A84AF086FC10B103481EF0A0FF72
:101720000E2006B010BD00BF110108002DE9F04FDA
:101730002DED028B95B00CAB51F8044B01935C4B33
:1017400000930138082317F055F90C98012209A9D4
:101750001AF032FA0D9800230E28CDE906330893CB
:1017600003D0012206A91AF027FA119B0BB9514B9D
:10177000119311981CF012F8DFED4F7AB4EEE70ADE
:10178000F1EE10FAB0EE408A06D4DFED4C7AB4EEFA
:10179000E70AF1EE10FA04DD494A4A494A481EF0C8
:1017A00053FF0A9B9DF838509DF83C80109E1F2BDC
:1017B00005D925B1079B13B144481EF051FF13987A
:1017C0000E280FD00DB94248F7E7424940F22A32BD
:1017D00017F0C6F9074694F84430DDF848901BB17D
:1017E0003D48EAE70027F6E7E36813B1204603F037
:1017F0001FFEDDF828A02946504602F0F7FADDF872
:101800001CB02946584602F0F1FABAF11F0F04D96C
:10181000BBF1000F04D03148CFE7BAF1000F02D07E
:101820000FB12F48C9E7002E38D1B8F1000F18BF0B
:10183000B426616819B9FF2011F06EFB6060A168E1
:1018400019B9FF2011F068FBA060DDE9091260689A
:1018500041F0B6FFDDE90612A06841F0B1FFCDE925
:101860000497BDF81C300393A3680293BDF8283099
:10187000019363680093B0EE480A33464246294616
:101880002046FAF77BFE3AF0A6FA01230E2084F8F0
:10189000443015B0BDEC028BBDE8F08F114B124AFD
:1018A00073439342C5D91148B4211EF0D9FE00BF3D
:1018B000D8140900CECC4CBE0AD7A33C0AD723418A
:1018C000CC140900D2140900541608005D23080046
:1018D0008E060800A84E08004621080044020800B1
:1018E0007101080040420F000FBCBA0A500A0800FC
:1018F0002DE9F04F2DED068B93B00AAB51F8044B58
:1019000001937C4B00930138082317F073F80D986E
:101910000E2823D01BF042FFF0EE408A0E9B0BB93D
:10192000754B0E930F9B0BB9734B0F930E981BF0D7
:1019300035FFDFED727AB4EEE70AF1EE10FAB0EEA1
:10194000408A06D4DFED6E7AB4EEE70AF1EE10FAC3
:1019500007DD6C4A6C496D481EF076FEDFED6C8A3F
:10196000DCE7F5EE408AF1EE10FA07D0F4EEC08A1B
:10197000F1EE10FA02D567481EF05EFE0F981BF0DC
:101980000DFFB4EEC08AF1EE10FAB0EE409A01D528
:101990006148F1E70A980023049348B1012203A9A2
:1019A0001AF00AF9039811F0EDFF08B95B48E3E774
:1019B00023699DF83050DDF82CB0109F9DF84480CD
:1019C000DDE903A93BB193F8293013B954481EF05F
:1019D00047FE00232361E36843B16268934202D16A
:1019E000112002F089FA204603F022FD00212C206C
:1019F00041F01FFE4B4B9FED4CAA0646002240F8DB
:101A0000083B59464AF0A0F9002D776214BFFF2722
:101A10001F270021C6E907A907F10800266141F048
:101A200008FE2369586000F10803036087800646BA
:101A3000012038F0FAFC3AF0CEF921693B48FFF773
:101A40007FFD68EE8A6A9FED3A7AC6EE877AF6EEF7
:101A5000009A77EEA97AFCEEE77A17EE907AB7F55E
:101A6000803F01D3334887E737B9F5EEC08AF1EEFE
:101A700010FA01DD30487FE70E22002106A841F070
:101A8000DFFE28EE0A8ADFED2D6AADF81E7088EEC3
:101A9000267A45F4807545EA880525F0FA05314631
:101AA00006A8ADF8185029EE0A9A37EE297AC9EE41
:101AB000267ABCEEC77A77EEA97A17EE103AFCEEDA
:101AC000E77AADF81A3017EE903AADF81C304AF0CC
:101AD000CDFA054640B115482169FFF763FD0023A3
:101AE000236128463AF077F9206913B0BDEC068BE4
:101AF000BDE8F08F2C150900CECC4CBE0AD7233B95
:101B000066D623421815090022150900541608004C
:101B100000000000FE1908007A2008002A070800CB
:101B200004080800FC54080000247449A9D70500E3
:101B300000401C46821E0800DF19080000401C44BB
:101B4000022838B50D46144613D1930701D01E2044
:101B500038BD1268084B9A42F9D1A168A86842F0D2
:101B6000F7FE0028F3D02A7923799A42EFD13E205C
:101B7000EEE70020ECE700BFA84E080010B588B0E3
:101B8000084611461A4603AB0193134B00930223F8
:101B900041F072FF00210C2041F04BFD0F4B036020
:101BA00004460122039805A91AF006F8069B062BA5
:101BB00003D00B4806211EF047FD049A032A03D9DF
:101BC00040F2762016F00EFF20460599D2B23AF088
:101BD000F1FF204608B010BDCC150900A84E080042
:101BE000931D080010B50B4688B0044605A99868F7
:101BF000012219F0E1FF059908780B794A790390E1
:101C00004878029088780190C9780091204602496E
:101C100043F0FFFB08B010BD6C150900062837B56E
:101C20000C4618D18D680D4B2B40062B11D128097D
:101C300049F0F2FC30B901A928461DF051FB019989
:101C400049F0D0FC23795840400040F0010003B037
:101C500030BD6868EEE70020F9E700BF0F0080FFA5
:101C60002DE9F04F97B00DAB0193394B0093043140
:101C70000923013816F0BEFE36490D9840F2015294
:101C800016F06EFF3449064640F2AA520E9816F03E
:101C900067FF0F9DEBB215F0C0050746089303D010
:101CA00040F2844016F09EFE9DF8409048463AF07F
:101CB0008BFF9DF844A050463AF086FF129C002C02
:101CC00004DA40F20A41284616F0F2FE14989DF814
:101CD0004C800E2806D1B8F1000F14D09CB12046DC
:101CE0001CF030FC0DF1280B0122594619F064FF5D
:101CF0000B9BA34204D8B8F1000F06D0A34204D036
:101D000016481EF099FC1648ECE715980E281CD0D2
:101D10001DF00EFB034600212820099341F089FCA9
:101D2000099B104A0260CDE905B3089B0093CDE9F9
:101D30000348CDE9019A3B4600223146054603F0AF
:101D4000E1FB284617B0BDE8F08F0023E3E700BFB2
:101D5000DC150900B8550800505608006115080048
:101D6000883A0800D450080010B54368044653B1BF
:101D700001460648FFF716FC0023C4E90333C4E913
:101D80000633636063610E2010BD00BF05BC060012
:101D900070B52DED028B86B0084611461A4603AB8E
:101DA0000193204B0093032341F066FE1E490398E4
:101DB00040F2CE2216F0D4FE4FF4AD610646B7EEE7
:101DC000000A049816F0B8FE059D002DB0EE408A7A
:101DD00004DC4FF42F71012016F06AFE0021202050
:101DE00041F027FC114B036004460121284641F0D5
:101DF00020FC9FED0F0A666028EE000A0023BCEE6F
:101E0000C00AC4E90305C4E905330A4884ED020A9F
:101E1000E3612146FFF794FB204606B0BDEC028B40
:101E200070BD00BF24160900D4500800D44F08002C
:101E300000007A4405BC060008B501481EF0A4FB6A
:101E4000FB230800C3691BB1D3E902011CF074BD78
:101E5000004870474836080037B58B680192044641
:101E60000D4673B1084943F0D4FAA968019A204697
:101E700000F088FC0549204603B0BDE8304043F03F
:101E8000C8BA0349F8E700BF94150900A017090074
:101E9000A41509001FB502AB51F8044B0193084B80
:101EA00000930138022316F0A5FD20469DF80C2072
:101EB0009DF8081003F092FB0E2004B010BD00BF87
:101EC00044160900084930B50022882505FB02F4B4
:101ED0006318645A844204D00132052AF6D10020E6
:101EE00030BD1846FCE700BF3806012030B587B08A
:101EF00005AB51F8045B01930F4B009301380123AC
:101F000016F078FD6868039000F018F805990398BA
:101F10000BF0D6F86C68204600F010F86368D3E93F
:101F200002011CF009FD6B680446586842F0F0FF9E
:101F3000204607B030BD00BF5416090008B53AF07E
:101F4000ACFE10B901481EF003FB08BDDC00080020
:101F500038B544680F4D2046FFF7F0FF94F8743011
:101F60000BB16B6A93B1B4F86C3007EE903AF8EEAF
:101F7000E77AB7EE047A67EE877A17EE900A20F0D8
:101F8000030040F00200A0F1FF4038BDFEF7A8FAC0
:101F9000E4E700BFC061012010B50446C06D0E2803
:101FA00007D100210C2041F044FB024BC0E9003472
:101FB000E06510BDE051080030B585B003AB51F8C5
:101FC000044B01931D4B00930138012316F012FDC1
:101FD00064681B4D2046FFF7B1FF94F85A30012B7F
:101FE00001D16B6AEBB194F85A30022B22D0012355
:101FF000144984F85A302088114D4AF01DF839F000
:10200000EAFE94F85A30012B01D16B6A63B16B6A16
:1020100083B994F85B1069B1882908D10A481EF089
:102020002DFBFEF75DFAD8E7FEF75AFAE9E7074815
:102030001EF024FB0E2005B030BD00BF3C16090089
:10204000C061012098130900D10B0800930B080010
:102050002DE9F0478CB005AB0193394B0093043167
:102060000723013816F0C6FC3649059840F2CE2207
:1020700016F076FD344940F2AA520646069816F04C
:102080006FFD9DF81CA0804650463AF09DFD9DF8DE
:10209000209048463AF098FD099D002D04DA40F260
:1020A0000A41002016F004FD0B989DF828700E28B8
:1020B00004D187B17DB128461CF044FA012202A95F
:1020C00019F07AFD039BAB4202D837B1AB4204D082
:1020D0001E481EF0B1FA1E48F0E70021182041F01A
:1020E000A8FA1C4BC0F80880C0E90036002304465B
:1020F000838280F816A080F81790DDE902011CF0B9
:102100000BFAE060A7B9B5F5007F05DD124A4FF480
:10211000007112481EF098FA2582A774F3691BB16A
:10212000214630463AF062FD20460CB0BDE8F0870B
:10213000B5F5FF7FF0DD0A4A4FF4FF71E9E700BF14
:10214000E8160900D4500800505608006115080030
:10215000883A08009052080017F00700F5170800A9
:1021600022F0070037B58B68019204460D4673B123
:10217000084943F04EF9A968019A204600F002FB95
:102180000549204603B0BDE8304043F042B9034959
:10219000F8E700BF6C160900A017090078160900BF
:1021A000130670B504460E4615460DD4022A0BD10F
:1021B00040F2632049F042FA0146204643F019F903
:1021C0000549204643F015F92A4631462046BDE828
:1021D00070401BF01FB800BF15F0070010B5436832
:1021E00004464BB101460548FFF7DCF90023C4E97A
:1021F0000233C4E9053323610E2010BD87AB07000D
:1022000008B501481EF018FA430508002DE9F0470B
:1022100088B0084611461A4605AB01932E4B009331
:10222000032341F029FC2D49059840F2CE2216F0F7
:1022300097FC069D002D064604DC4FF42F7101200B
:1022400016F036FC07980E283CD1B6F81280002113
:10225000302041F0EEF9224B03607368B47D9B7926
:10226000074640F2FD10804504F0300228BF80464A
:1022700004F0060413B1134622461C4632B308F19B
:10228000020A05FB0AFA0021504641F0D2F98146C4
:10229000FCB10021404641F0CCF900210546404602
:1022A00041F0C7F904460023CDE902833846CDE961
:1022B000005453464A463146FAF73CFA384608B0CD
:1022C000BDE8F0871BF0B2FA8046C0E7914692461F
:1022D000DEE72546E7E700BF30170900D4500800C5
:1022E000F45308001FB50446084663680BB929F08B
:1022F00001F8022201A919F05FFCDDE90112204674
:102300003AF055FD002803DA414204481EF09CF9DA
:10231000400040F0010004B010BD00BF7022080072
:1023200010B58AB002AB0C460193144B00930431F4
:102330000223013816F05EFB246863680BB928F0AD
:10234000D9FF0298012207A919F036FC039800234F
:102350000E28059303D0012204A919F02DFC059B3A
:102360000093DDE90712049B204603F089FA20EA76
:10237000E070400040F001000AB010BD20170900D5
:10238000F8B5254C254B23603AF0F3FB002842D0EA
:10239000234B1A781AB9234A1278012A09D1224804
:1023A00000221A70436823B1204B1B780BB103F055
:1023B0004FFA194803F05CF8E36813B1164803F0CC
:1023C00037F800231A4DA3614FF6FF7705240E2638
:1023D0002888B84202D0132149F03CFE013CEE654A
:1023E00005F18805F4D14BF077F80B48214602F04F
:1023F000B9FE4FF42A230F4A1B68934205D14FF4CC
:102400003122D2F8FC2F9A4201D000F0F5FABDE853
:10241000F8402FF051B9F8BDAC5601202C4E080001
:10242000296C0120926C01204C550120236B012066
:10243000380601203130444230B589B003AB51F841
:10244000045B01930E4B00930138022316F0D2FA7D
:102450009DF81040039805A9012219F0ADFB84F006
:102460000104E8680094DDE90523D0E9021039F0A1
:1024700042F9002814BF3E201E2009B030BD00BF25
:10248000C816090030B587B0084611461A4604AB95
:102490000193124B0093022341F0EEFA0498104985
:1024A00040F2AA5216F05CFB9DF8142003920546F8
:1024B0000021182041F0BDF80A4B036004460020BB
:1024C00040F033FF039A03462946204637F002FACC
:1024D00039F081FC204607B030BD00BFD816090096
:1024E00050560800B855080037B58B68019204466D
:1024F0000D4673B1084942F08CFFA968019A204645
:1025000000F040F90549204603B0BDE8304042F0F4
:1025100080BF0349F8E700BF9C160900A017090017
:10252000A516090008B501481EF02EF82A06080075
:1025300010B5022888B00B46144624D1A20720D13A
:102540002168124A91421CD19A79012A09D1A279B3
:10255000012A06D19A88A3889A4212D13E2008B057
:1025600010BD184669463AF031FD04A920463AF0FC
:102570002DFD10220DEB0201684641F00FF90028F5
:10258000ECD01E20EBE70020E9E700BF5056080022
:1025900008B58B7813B904481EF062F80B88838065
:1025A0008B78837108BD00BF750B08001FB5837958
:1025B000012B02D106481DF0C3FF69463AF006FD23
:1025C000102168461BF0A8FF05B05DF804FB00BFB2
:1025D0000F1A08002DE9F04106468EB00846114654
:1025E0004FF002121C4616F0D5F90021082041F0E8
:1025F00020F8066005462068C30706D410F00302E1
:1026000012D101683E4B99420ED11BF00FF9B0F583
:10261000803F02D33B481EF00FF80123A880AB7126
:1026200028460EB0BDE8F081374B0340062B05D09D
:10263000002A4BD10268354B9A4247D101A91CF0C0
:102640004FFE019B242B01D03148E4E7037A2D2B68
:10265000FAD1437B2D2BF7D1837C2D2BF4D1C37D75
:102660002D2BF1D1471E00F12304002617F8018F0E
:10267000404631F083FE20B10EAB3344013603F8FF
:10268000208CBC42F2D1202EDED106AC0DF1170811
:10269000002620784BF04DFC074660784BF049FC53
:1026A000023640EA0710202E08F8010904F102045E
:1026B000EFD1BDF8142000238DF814308DF81530BB
:1026C00002A9AA8028463AF069FCA9E7012206A9D6
:1026D00041F081FE08B90F489DE7079B102B01D000
:1026E0000D4898E7069B02AC03F11006186859687C
:1026F000224603C20833B3421446F7D1D9E700BFDC
:10270000B4F60700F10A08000F0080FF28F7070061
:10271000010B0800170B08009D22080010B588B0B7
:1027200003AB51F8044B0193144B0093013802237F
:1027300016F060F90222039805A919F03DFAA07974
:10274000049B069901280CBF1022802203EBD202C1
:102750008A4202D90A481DF06FFF059A012802EB50
:10276000030107D1A088D054A3881B0A4B700E2008
:1027700008B010BD20463AF029FCF8E7A41709007C
:102780004222080010B58A79012A92B004460B460D
:1027900006D18A881E4912B0BDE8104042F039BE09
:1027A0000EA918463AF012FC9DF838300D939DF8AA
:1027B00039300C939DF83A300B939DF83B300A93D7
:1027C0009DF83C3009939DF83D3008939DF83E30CC
:1027D00007939DF83F3006939DF8403005939DF890
:1027E000413004939DF8423003939DF843300293A7
:1027F0009DF8443001939DF8453000939DF84720A3
:102800009DF846300349204642F003FE12B010BD49
:1028100048170900551709002DE9F04F754C87B08E
:10282000002600AFA4F108084FF0880909FB0683D1
:1028300093F87830002B66D04AF04EFED4E91E2380
:10284000801A61EB0301B0F57A7F71F100035AD36E
:10285000002134F8080CF981032307F10E026D46BC
:1028600049F028FC002848D1FB8934F8080C0733CC
:10287000DB08A5EBC3039D4607F10E02032369465F
:10288000EA4649F017FC002837D1B4F8502014F874
:10289000060C02213FF07DFEFB89834658B1C288B9
:1028A0009A4205D100F10801684640F077FF20B355
:1028B000584640F0CAFA00233B7414F8063C3A8AA2
:1028C000F889F88243F4007302F0FE0223F0FE035D
:1028D00013433B82B4F850307B8234F8083CBB820F
:1028E0000FF02CF90222834607F110012BF0BAF801
:1028F000FA89514658464CF011F809FB068300222C
:10290000AD4683F8782009FB068393F87930002BD5
:1029100040D014F8060C002846D0B4F82EA0524639
:1029200001213FF036FE054650B1C288502A04D13D
:102930002146083040F032FF38B3284640F085FA8F
:10294000002022F02BFF04F1490B054614F8062C59
:102950006DBB0123A7F812A04FF0500A62F30005E7
:102960007B74504634F8083C3D74BB82A7F816A02F
:102970000FF0E4F80222054607F110012BF072F87F
:102980005246214628464BF0C9FF09FB0683002228
:1029900083F879200136052E04F188047FF446AFD0
:1029A0001C37BD46BDE8F08FB4F812A0B7E76B78CE
:1029B000012B1AD12B7803F00103934215D1EB8838
:1029C000502B12D10622594605F151007B6040F090
:1029D000E5FE50B97B6821461A4605F1080040F033
:1029E000DDFE10B1284640F030FA284622F0D6FE2F
:1029F0000546ABE74006012073B5104D4FF42A247D
:102A00004FF00106200B2E7049F06AFB08B92BF03D
:102A100019F804F58054B4F5322FF3D1084B019323
:102A200001A901224FF42A202BF01CF805480122AD
:102A300001A92BF017F802B070BD00BF776C012020
:102A400031304442FC1F0B00032A05D11E2914BF5C
:102A50000449054942F0CDBC1E2914BF034904496D
:102A6000F8E700BFBBEF0700C0EF070022F0070048
:102A700017F007002DE9F0470C6888B08046204623
:102A800099460D4692461AF021FF012205A90746F4
:102A9000204619F091F86868012202A919F08CF813
:102AA0009DF810100022402016F07AF80128034605
:102AB00002D01D481DF0ACFDDDE90541B8F1020F63
:102AC00004EB010613D9AA680E2A03D0384619F080
:102AD0007DF80444B8F1030F09D0EA680E2A06D045
:102AE0000699059E0123384619F070F80644A6425F
:102AF00008D3DDE90223CDF800A0311B20463FF0CA
:102B00005DFD28B9B9F1000F0AD008481DF094FD09
:102B1000059BC01A400040F0010008B0BDE8F087F6
:102B20004FF0FF30F9E700BFFE0D0800061E080059
:102B300070B588B00D460C2000211646039340F076
:102B400078FD134B036004AB0193124B039A00937F
:102B5000314604230446284640F08EFF04984BF08B
:102B6000BBFB054605984BF0B7FB29790279069B1C
:102B7000914203D140F26D4015F034FF00226260B3
:102B800029460246204602F0FFFE204608B070BDEE
:102B90004C580800881E090070B50C468EB054F8D9
:102BA000045B03920646A87A39F0C8F8287A39F00F
:102BB00005F90AAB0193174B039A009321460423AE
:102BC000701E15F017FF0B98022207A918F0F4FFEA
:102BD000089B0D99069306AA0C9B059305A847F040
:102BE00034FD069B0393184640F2BB22012140F0BE
:102BF00065FF039B53B10799059A28460A44BDF81F
:102C0000281002F081FF08B11DF0D2FC0E200EB09A
:102C100070BD00BFE01E090070B50C468EB054F8C0
:102C2000045B03920646A87A39F088F8287A39F0CE
:102C3000C5F80AAB0193134B039A00932146042372
:102C4000701E15F0D7FE0B98012207A918F0B4FFEB
:102C5000089B0D99069306AA0C9B059305A847F0BF
:102C6000F4FC01230093DDE90631059A28460A4465
:102C7000BDF82810F9F7C4FD08B11DF099FC0E202D
:102C80000EB070BD681E090070B50C4696B054F8C1
:102C9000045B03920646A87A39F050F8287A39F096
:102CA0008DF80FAB0193234B039A0093701E0723FB
:102CB000214615F09FFE109801220CA918F07CFF08
:102CC0000D9B1399089308AA129B079307A847F036
:102CD000BCFC1198022209A918F06EFF0A9B06930A
:102CE0001599149B059306AA05A847F0AEFC069E0D
:102CF00026B9114840F24E411DF0A6FC059B099CE7
:102D00000C98079ABDF83C1003911C4400230093D3
:102D10000244089B2846F9F773FD30B903993346FE
:102D20002246284602F0F0FE08B11DF041FC0E20BC
:102D300016B070BDA81E09008205080070B50C46CB
:102D400088B054F8045B03920646687A38F0F0FFC6
:102D5000287A39F02EF804AB0193184B039A0093AC
:102D60002146701E042315F045FE40F275430122F2
:102D70000021059815F0A4FE40F2674301220021CE
:102D80000446069815F09CFE40F2AB230646092245
:102D90000798082115F094FEC0B2082802D005203B
:102DA0001DF006FC0499F3B2E2B228463AF02FF97E
:102DB0000028F4D00E2008B070BD00BF881F0900A5
:102DC00070B588B00D460C2000211646039340F0E4
:102DD00030FC164B036004AB0193154B039A009330
:102DE000314604230446284640F046FE04984BF042
:102DF00073FA039005984BF077FA054606984BF066
:102E000073FA0399034618B915B90A481DF014FC62
:102E10009DF81C2012B108481DF0B6FB62602046E8
:102E20002A4602F0B9FE204608B070BD6C59080071
:102E3000001F09009B0408003E03080010B504466B
:102E4000407A38F075FF63681B68D3F82435B3F116
:102E5000805F23D013D8B3F1006F21D00BD8B3F12A
:102E6000007F1FD01248B3F1806F18BF00204000D0
:102E700040F0010010BD0F48B3F1206FF5E7B3F14A
:102E8000804F11D006D8B3F1A05F0FD00A48B3F13C
:102E9000005FEAE70948B3F1004FE6E70848E6E7D4
:102EA0000848E4E70848E2E70848E0E70848DEE7C2
:102EB00090D003000024F40080841E0000127A00E9
:102EC00040420F0020A1070048E8010000093D0032
:102ED0000048E80170B50C468EB054F8045B0392CC
:102EE0000646687A38F024FF287A38F062FF0AAB89
:102EF0000193134B039A009321460423701E15F08F
:102F000079FD0A98022207A918F056FE0B9B06933A
:102F100005AA089B0C99059306A847F096FB059A0D
:102F20005AB1DDE906109DF83430014428463AF0E4
:102F3000A0F810B905201DF03BFB0E200EB070BDAF
:102F4000501F090070B50C468CB054F8045B039216
:102F50000646687A38F0ECFE287A38F02AFF09AB8A
:102F60000193124B039A009321460323701E15F020
:102F700041FD0998012206A918F01EFE0A9B05933F
:102F800004AA079B0B99049305A847F05EFB049ADB
:102F90004AB1DDE905312846194402F021FF10B994
:102FA00005201DF005FB0E200CB070BD701F090040
:102FB00070B50C4694B054F8045B03920646687AE8
:102FC00038F0B6FE287A38F0F4FE0EAB01931E4BB3
:102FD000039A009321460623701E15F00BFD0E98F0
:102FE00001220BA918F0E8FD109B1199079306AA7E
:102FF0000C9B069307A847F028FB0F98022208A90C
:1030000018F0DAFD129B059304AA099B1399049307
:1030100005A847F01AFB069B049A934202D00B487E
:103020001DF00AFB63B10899059A0B980A440799A9
:103030000144284602F098FE10B905201DF0B8FAA8
:103040000E2014B070BD00BF201F0900440F0800FF
:103050002DE9F04F2DED028B9BB0084611461A4624
:103060000EAB0193B84B00930C2340F005FD0F9875
:103070004BF03AF907460E984BF036F9064618B968
:1030800017B9B2481DF0D8FA40F2AB2311980922C3
:10309000052115F015FD129DAD4B9D4282461DD0B8
:1030A000AC4B9D420CBF02250025139896230222AB
:1030B000012115F005FD14981AF070FBB5EEC00A59
:1030C000F1EE10FAB0EE408A06D4DFEDA37AB4EE4A
:1030D000E70AF1EE10FA03DD33F0D6FA0125E4E752
:1030E00016984BF001F9814617984BF0FDF8804691
:1030F00018984BF0F9F89DF864300393012183464A
:103100002C2040F0A6FA954A02605FFA8AFA109BDA
:103110000493BAF1080F1599039B044605D0904813
:10312000082240F2AB211DF08FFABBF1000F00D155
:1031300013B18C481DF028FA43608B4B1A68D2F803
:10314000002512F00F0206D09A68D2F80025120767
:1031500040F0F880012203EBC20363600EB9002F38
:103160008FD01FFA81FB40F2A7420121584640F060
:103170009CFC022D01D17D4884E7B9F1000F3BD1C1
:10318000B8F1000A18BF4FF0010A00238DF837305C
:10319000002E34D033790793002F33D03B79089336
:1031A000B8F1000F31D098F804300993B9F1000F4D
:1031B0002ED099F804300498CDE90A3410F058FF65
:1031C000002D4FF0030318BF0E258DF835A00C908D
:1031D0008DF834308DF836506568654A2B79242196
:1031E0004B4302EB030A9AF82010039199B1614A0C
:1031F0006149624842F09AF94FF0010AC5E74FF081
:10320000FF33C8E74FF0FF33C9E74FF0FF33CCE798
:103210004FF0FF33CFE707A92846059337F02EFA82
:10322000534A059B5649CAF804100B99D1509DF892
:103230003430286805934FF4887147F01BFA2868EA
:103240004FF4907147F016FA28684FF4927147F0E6
:1032500011FA28684FF4A27147F00CFA28684FF46D
:10326000AC7147F007FA2A684649C2F80413059B77
:103270002868194640F30730F8F72AF9286840F320
:10328000073035F0A2FF2B680822C3F80025039B06
:10329000CAF814300122CAE906338AF8202087B11F
:1032A000594604F1100048F04FFD28B9606822F03B
:1032B00099FF584614F04AFB387984F8270000F04B
:1032C0007FFF9EB3307984F8260000F079FFB9F1D2
:1032D000000F2FD099F8040084F8290000F070FF47
:1032E000B8F1000F2AD098F8040084F8280000F004
:1032F00067FF9FED250A049BA36028EE008A002348
:10330000BCEEC88A84F82530606884ED038A04F135
:10331000240122F0E3FE1D4B984202467FF468AF81
:1033200020461BB0BDEC028BBDE8F08FFF2384F874
:103330002630CCE7FF2384F82930D1E7FF2384F837
:103340002830D6E712489DE6A81F0900331F080061
:103350006C5A0800905A08000000C842D85A080069
:10336000260608009C0708007C0201205A06080077
:10337000506101200500AD0B95120800BCF4070058
:10338000BDDC07001003420000007A440000AD0BD2
:10339000701F080010B51EF017FD044690F82700B6
:1033A00038F0C0FCD4ED037A9FED077AF8EE677A27
:1033B000C7EE877A17EE900A20F0030040F0020073
:1033C000A0F1FF4010BD00BF00007A4410B51EF010
:1033D000FBFC044690F8270038F0A4FC63681868EA
:1033E00040F30730002801DBF8F760F80023C4E958
:1033F0000733A36163681B681A0B43F30733002B81
:1034000007DB02F01F0101228A405B09024941F8F3
:1034100023200E2010BD00BF00E100E038B50D46AE
:103420001EF0D2FC044690F8270038F07BFC2846BA
:103430001AF0B4F9B5EEC00AF1EE10FA06D4DFEDD9
:10344000097AB4EEE70AF1EE10FA01DD33F01CF967
:10345000DFED057A20EE270A0E20BCEEC00A84EDCF
:10346000030A38BD0000C84200007A4407B50A4B81
:103470008B4214BF4FF4C9714FF4AC7140F2EB139F
:103480000191009305494FF4107340F2BF2241F0BF
:10349000C0FF03B05DF804FB6C5A08000820090067
:1034A00037B50C462046114606221D4615F072FA25
:1034B00034B92146012003B0BDE83040FBF7D2BC4F
:1034C0002968CA0705D48B0708D10A680F4B9A42AE
:1034D00004D1012C08D00E481DF09AF8012003B049
:1034E000BDE83040FBF7F0BB08461AF09FF90146F3
:1034F00001902046FBF7B6FC019A04460021C06803
:1035000040F09EF9204603B030BD00BFB4F607007E
:10351000F2200800084608B5194612B104481DF00B
:1035200033F818B1BDE8084000F006B8014808BDFE
:1035300073170800883A080070B50546086810F04F
:10354000030390B00E4603D10168414A914228D04E
:10355000404C00EA0402062A04D033BB02683E4B0A
:103560009A4222D1023D012D6ED80CA91BF0B8FE63
:103570000546306800EA0403062B14D1000948F020
:103580004BF804460C9A34B911462846019248F08B
:1035900029F8019A04462E48002141F0B7FDC56084
:1035A000446010B070BD4468ECE7012D4CD110F0C0
:1035B000010413D0421002D500201DF03DF8114641
:1035C0000CA801924BF044F9019A0E98002140F0AA
:1035D00037F90CA91E481BF043F9E2E703AAB22110
:1035E00018F0AEFF039B2BB103AA2146204640F002
:1035F000B7FBD6E730682A4605A940F0ECFE20B1BB
:10360000DDE905011AF088FFCBE730681AF0D8FE33
:1036100098B910210CA84BF009F9306808A918F0E6
:103620002FFB0446204618F0BBFC0028D1D01AF02E
:10363000FDF8FF2803D90948BFE74110EAE7C1B206
:103640000CA84BF05DF8EDE705481CF0E1FF00BF6A
:10365000F4F407000F0080FF28F707006D0F080043
:10366000F2200800F0B585B0054617460C461AF062
:103670002DF96946064628461BF032FE042F054602
:1036800022D1A307009814D12268104B9A4210D17E
:1036900001AA214642F037F810B90D481CF074FF1A
:1036A000DDE901123046521A29441BF039F905B000
:1036B000F0BD014600232246304618F087FA285C08
:1036C000400040F00100F2E70020F0E77832080007
:1036D000DB1A08008B072DE9F14F04460D4616460C
:1036E00011D001F00F03022B17D1D7074FEA1111A8
:1036F00004D401B0BDE8F04F07F09ABA01B0BDE8BC
:10370000F04F06F0A3BF4968CBB22D2B00F08380A9
:103710000BD8062B0ED02C2B13D0534A294620460B
:1037200001B0BDE8F04F07F097BA2E2B00F088806B
:103730009D2BF2D1002EF0D105F10802090A204696
:1037400083E0022A02D0A96806F0B6FFEF68002FD6
:10375000E3D017F00309E0D17B68DAB28E2AB846CD
:103760000DD1022E4FEA132805D007F1080A08F1FF
:10377000FF3BD94515DB08F1010857F8288098F878
:103780000430312B27D1022E13D1A06A40F0A3FDC3
:10379000A06A56226FF0020101B0BDE8F04F3DF083
:1037A0001CBB5AF8041B204606F086FF09F10109EC
:1037B000DFE7D8F80810204606F07EFF012EE7D19B
:1037C000A06A582202213DF008FBA06A01B0BDE8C2
:1037D000F04F40F0ACBD322B9FD1012EA06A0AD130
:1037E00040F0BBFCD8F80810A06A090901B0BDE898
:1037F000F04F40F060BC022E01D140F070FDD8F8CF
:103800000830A06A1B0918226FF0010101B0BDE861
:10381000F04F3DF0EBBAAA68002A3FF47EAF002ECD
:103820007FF47BAF5168090A022907D1D3682BB115
:10383000980703D11B79AC2B3FF46FAF08327EE7BA
:10384000002A7FF46AAFA96821B901B0BDE8F04F42
:1038500000F00CB88E0703D10B79922B0A46E1D009
:1038600005F1080201216AE79B0F08002DE9F743E3
:103870000D460139044690464FEA012900264FF0D3
:10388000FF3719F5807F0CD17B1C04D1A06A2B4631
:1038900030223DF0EBFA0026AE4221D103B0BDE864
:1038A000F08358F826307BB19A070DD11A79222A75
:1038B0000AD101370CD1A06A019149EA06033122ED
:1038C0003DF0D4FA019937460136A9F58079D8E759
:1038D000094A1946204603B0BDE8F04307F0BCB9D9
:1038E00058F82610B74208BF896800222046FFF723
:1038F000F1FE0136D0E700BFCB18080001F00F033E
:10390000022B2DE9F34705460C4605D1090902B003
:10391000BDE8F04706F002BD00295FD011F00306B4
:103920005CD10B792C2B41D1896806F0C5FEE66885
:10393000002E53D016F0030850D17768FAB28E2AC1
:10394000334609D13F0A06F1080907F1FF3AC2459B
:1039500019DC013756F827301A79312A1BD19968BA
:10396000284606F0A9FEA86A019040F093FC019851
:1039700040F0B1FC019856226FF0020102B0BDE8A0
:10398000F0473DF02ABA59F8041B284606F094FE89
:1039900008F10108DBE7322A20D19968A86A0222DF
:1039A000090902B0BDE8F04740F06ABB2D2B15D1E4
:1039B0008C689CB163681B0A022B01D1E36843B990
:1039C00004F108076368B6EB132F0FD302B0BDE80C
:1039D000F0879A07F4D11B79AC2BF1D1074A214625
:1039E000284602B0BDE8F04707F036B957F8041B87
:1039F0002846FFF783FF0136E4E700BFE50F080024
:103A000010B5137803F06003202B144647D1254BE3
:103A10009288187890420ED093F8B80890423ED120
:103A200003F6B80301206278203A032A37D8DFE88A
:103A300002F00414172B0020F5E729B90722991D7D
:103A400020462FF0D1FE06E0022904D1164A12B119
:103A5000991DAFF30080012022E00029FBD1EDE7A2
:103A600019B920462FF0AEFEF5E70229F3D162889E
:103A70001A7102F0010181F0010483F82C40C2F3B5
:103A800040022FF0F7FDE6E70029EAD00229E2D153
:103A9000064B002BDFD06188AFF30080DBE700200E
:103AA00010BD00BF9C0C01200000000000000000C1
:103AB000F8B5294B41F27012002118463FF0C0FEC4
:103AC0000346082601244FF48235067300F13801BD
:103AD0004FF0FF0C4FF4424783F8C46803F50F66BC
:103AE0000022016180F805C04FF47841C78004814D
:103AF0004561C3F8C86840F2FF7003F5876E03F5AF
:103B00004F66DA83C3E909E51A8498835A86598394
:103B10009A8683F82C40A3F8D6281886D98583F88E
:103B2000BDC8A3F8BE78A3F8C048C3F8CC58A3F822
:103B3000D408A3F8D218A3F8D828C3F8DC68C3F8CF
:103B4000E05883F8E448A3F8E808A3F8E618A3F8D7
:103B5000EA28A3F8EC28F8BD9C0C01202DE9F743D6
:103B60004B79022B04D00025284603B0BDE8F08332
:103B70008B79022BF7D1DFF8A09099F802701FB172
:103B800099F8BA38ABBB012740F6B8067E438B786C
:103B900009F806300C7809EB06080C44092563780F
:103BA000242B20D1AA4219D26378042B12D1637935
:103BB0000A2B0FD12778F31C02364E4402220096BE
:103BC0004B441146E0194AF046FA90B10E3517FA07
:103BD00085F5ADB2404636F079F9C5E723781D4446
:103BE000ADB21C44DBE7052BDED1204632F068F98C
:103BF00038B94FF0E023D3F8F03DDB07B3D500BE72
:103C0000B1E740F6B80202FB0797A3787B702378F0
:103C10001D44ADB21C44C7E79C0C012070B50F4C8D
:103C2000002504F110002560257149F006FF04F11C
:103C3000240049F002FF012604F6C80084F82C6035
:103C4000C4F8B85884F8BC5849F0F7FE04F6DC0014
:103C500049F0F3FE84F8E46870BD00BF9C0C0120BD
:103C60002DE9F7433D4C1D46E3788B420E4617D0B5
:103C7000A3788B4214D094F8BB388B422ED094F8A2
:103C8000BA388B422AD04FF0E023D3F8F05D15F01C
:103C9000010501D000BE0025284603B0BDE8F08331
:103CA0000027E378B34214D104F63808AAB241469B
:103CB00004F1100049F04DFF6379FF2B04D005F6A5
:103CC0003809A144C8450DD1254BD3B9204636F05B
:103CD000FDF8A378B3421ED00125DDE704F6B80451
:103CE0000127DEE7617918F8013B9942EAD1E28BBE
:103CF000238C92B29BB29A42E4D038462FF042FD18
:103D0000E0E7E28B238C92B29BB29A42DED0384637
:103D1000AFF30080DAE7134B13B13846AFF30080FE
:103D200038462FF0F3FC0028D6D104F1240049F0E6
:103D30008FFE0028D0D1002DCED015F03F02CBD180
:103D4000A078019232F0A2F8019A05460028C3D06B
:103D5000A078114632F0C4F99EE700BF9C0C012008
:103D6000000000000000000010EE103AC3F3C7523C
:103D7000A2F17F01162982B013DC002913DB124A5D
:103D80000A411A420DD0DFED117A30EE270A002BDE
:103D90008DED010AA8BF9B18019923EA020300EEEA
:103DA000103A02B07047DFED097A30EE270A002B97
:103DB0008DED000A009A04DB5A0018BF4FF07E53C5
:103DC000EDE74FF00043EAE7FFFF7F000000807B54
:103DD000054B4FF0FF32072843F8202084BFC0185E
:103DE00080F85020704700BF24600120FF2808B5EC
:103DF00002D821B1EE2802D901481CF01DFC08BDF3
:103E000083010800830773B5044603D102680A4B97
:103E10009A420AD0094E0025204616F8011B0123BC
:103E20006A4618F0C7FB009808B1012002E001358E
:103E3000032DF1D102B070BD0CF70700643B0900FF
:103E400038B50023C3714FF0FF33C36405463FF01C
:103E50004CFD044630BBB5F84E224AF655239A4233
:103E600022D114490B2205F150003FF097FCE8B134
:103E700095F85030EB2B03D01833DBB2012B17D859
:103E80000D49032205F186003FF088FC40B10B4943
:103E9000052205F1A2003FF081FC002818BF022492
:103EA000204638BD0424FBE70324F9E70124F7E7A3
:103EB0000224F5E7AF2D0900BB2D0900BF2D090035
:103EC00008B501481CF092FB2403080008B5074B15
:103ED0000340062B05D0830706D10268044B9A42A3
:103EE00002D104481CF094FB08BD00BF0F0080FF06
:103EF00028F70700FE0D08000D2808B5014612D06E
:103F000006D804280BD0072810D00A481CF0A8FBBC
:103F100043F202039842F8D107481CF019FB074905
:103F2000074841F0F8FA07480021FAE706481CF074
:103F300083FB00BFA00B0800150608000006080060
:103F4000A0F40700A42E0800EC030800012808B51F
:103F500005D0022808D1054840F22B3102E0044880
:103F60004FF4F6711CF070FB08BD00BFE7030800BA
:103F7000A400080008B510B901481CF05DFB08BD9D
:103F80005003080073B504461E460D4651B118682B
:103F9000019219F09BFC6368019A834202D00548A4
:103FA0001CF036FBA0683346294602B0BDE87040DD
:103FB00015F09CBE360E08002DE9F04F2DED028B5A
:103FC00083078DB004460D4609D10368784A9342B1
:103FD00005D111F0030802D10A689A4202D075484F
:103FE0001CF016FB46F04DF918B1284646F049F989
:103FF00008B97148F4E7267930461FF0ABF9029012
:1040000028791FF0A7F90690304621F0CFF8D4E9BF
:10401000037305903246E07901930AA9CDE90A3786
:1040200046F075F9C3690493D4F81CB0EB69DDF868
:1040300010A003930646D946B8454CD105F10C01B2
:104040006622E879089146F062F90899C3690590FB
:104050006622E879079346F05AF9C1694FF00008E3
:1040600089468A46B84567D1019A049B746904FB66
:104070000234079B01EB870503EB8709A7EB020BD3
:104080009046019B08F1FF3A534500F28C80059859
:104090000DB0BDEC028BBDE8F08F48460793029B44
:1040A0009847059B504698477269079B9244A269BE
:1040B00001339144019A9342EFD1D6E90523019946
:1040C00002FB11339A44D4E9053202FB11339944BF
:1040D00008F10108B0E70023ECE7CDE908315846C4
:1040E000029B9847FAEC017AA269089B0999A0EE15
:1040F000278A934401339845EFD10398069B089192
:104100009847029B584630EE488A9847C8EE007A96
:10411000CA466FF0030303FB08AA0899E9EC017A89
:10412000D4E9053202FB18339B44039AAB691A4465
:10413000039208F1010895E79FED208A0023DAE752
:10414000029B2046CDE9032198470499B369F1EC1D
:10415000017A039AE0EE278A1C440132BA42EFD377
:104160004745B06935ED018A2CBFD8464FF00008AD
:104170004FEA8B0308F1010838BF0023A3EB880343
:1041800000FB184899444046029B984738EE688ADD
:104190000BF1010BC8EE007AC9ED007A7469A8EB47
:1041A0000404D0466DE7DFED058A49464246D5E76F
:1041B000C8A008006E130800DD150800000000000C
:1041C0004109064A012300F01F0003FA00F052F8EB
:1041D0002130184342F82100704700BF605601208B
:1041E0002DE9F04F042997B080460C4635D0A64EF5
:1041F00030680EF003FB002C4BD0A44B9C4248D0FF
:10420000002503AB04932A46A14B0593214604A83D
:1042100003951AF0BBFB039804300122294620F0D5
:10422000030036F007FA3060B8B103680A939DF8CE
:104230002C30039A43F001038DF82C3008ABCDE904
:10424000082506932A46934B0793214606A81AF0A1
:104250009DFB33681A68039BD5548F4C8F4B2068A5
:1042600000251D600FF0C6F925608D4C8D4A23682E
:10427000934211D16268A24202D3631C9A4229D9A7
:10428000894D106851682B4603C3906818606560BB
:1042900020E000233360E0E78449D4F8C0208B425B
:1042A000E8D083498B420DD1824B9A4240F09081F5
:1042B000D4F82831A34240F08B810121204639F007
:1042C0006FFA07E07C4A934204D1626804F1080562
:1042D000AA42D6D1D4F8C030784A934240F09E80AA
:1042E0007748012139F00CF87648002109F0DCFB11
:1042F0007548764F01F0BCF8734801F099F8D7F88B
:10430000DC50002D40F0A9802CF08CFBD7F8A46085
:10431000002E40F0B18027F0FFFE0DF0A9FAD7F88B
:10432000E49048460FF02EFB0546002840F0A88098
:10433000DFF8C0B10890C7E938990DF1200A02F002
:10434000C3FEDBF80000D146002840F0D780089B70
:10435000CBF800305E4B01901E605E4B5E4E1870D5
:1043600002F0C4FE30F0F2F9BB8A0198C7F8900160
:104370000133BB820EF076FF0198C7F884014046F6
:104380000EF03CFA0FCE4D460FC50FCE0FC50FCE27
:104390000FC596E8030085E80300DFF85CA1002361
:1043A000D346DAF800601EB13568002D40F0BF80BA
:1043B000002BF2D1DBF800301BB15A68D20700F1B4
:1043C000DD80D7F8D430002B40F0DC80434B444DE7
:1043D0001B684449444AC5F80090002B00F0F58062
:1043E0001B684B62118B0B4453622268304B9A421C
:1043F00003D12B48002103F085FA22682E4B9A4204
:1044000005D1E069FAF7E8F800B10068E06100233F
:104410002B6017B0BDE8F04F2DF0C4BC334A934277
:104420003FF462AF234A93427FF462AFD4F828018D
:1044300019F04CFA70B12E4B98420BD02048012154
:1044400039F058F81F48002109F02EFB012384F8A9
:1044500022314DE727F0FAFD4AE7D7F884314BB116
:1044600069688B4206D8D7F88831994202D2A86889
:10447000FDF798F82D6844E7304611F049FC45E710
:10448000D9F80C904DE700BFAC6401201462012004
:10449000C7F20600B9E707001C5601202456012088
:1044A000E008012078640800E80801201866080088
:1044B000F89108007C710800E4950800F06208009B
:1044C000A0090120A8090120AC560120C0610120EB
:1044D00028560120506C0120DC5501204C6601203B
:1044E000A0640120F00301209C0301200C6408005B
:1044F0009C36080020560120F05D0120D7F8842169
:1045000083682AB1904203D3D7F88821904207D319
:10451000CAF80000064600F1080A8560184613E74D
:104520001022002101933FF08BF9019BF6E772689E
:10453000900720D56A68D1071DD506F10800FAF763
:104540004BF805F10803036072682B68336022F0B2
:10455000030202F108086B6801934246314628467F
:104560003FF056F905EB0802019B45F808505360EF
:10457000CAF800200123DAF800A012E71B68CBF884
:10458000003017E71D68144A1668C5B93368136010
:1045900073680836304623F00308FAF71DF8012245
:1045A000824629464046F9F76FFF00F1080342466C
:1045B000314618463FF02CF9CAF8000001E7B54231
:1045C00038BF1A462B462D68DEE753624B620CE774
:1045D000024803F037F97DE694620120E0080120EB
:1045E00013B540F281516A4617F084FF00216A46F4
:1045F00008463FF0B5FB084C40F03FFC08B102B064
:1046000010BDFBF76DFF616A0029F8D16A460846C4
:104610003FF0A6FBF0E700BFC061012070B5044683
:104620009AB04068FFF7DCFF002040F0D4FC012284
:104630006946064617F0C0FA07A845F0EEFF0546A2
:10464000B8B9606803AA40F2CB5117F053FF237A40
:104650005B0043F0010303AA29460220CDE9053699
:104660003FF07EFB21F0DCF8606837F03FFD1AB0C8
:1046700070BD606837F03AFD089D0649286819F05A
:1046800061FE18B1217A04481BF0DEFF284621F0B4
:104690009FF800BFFC2D08001105080070B52DED36
:1046A000028B0646B0EE408A1DF076FB9FED1F0A96
:1046B00080ED068A28EE008A4289BCEEC88A04464C
:1046C00018EE103A9BB29A4209D005894268416AB5
:1046D0004381B3F5807F02FB05F503D159B9BDECE9
:1046E000028B70BD39B928463EF0A3FF216A606293
:1046F0002A463FF065F80023AB420AD194F82830EF
:10470000002BECD0BDEC028B3046BDE8704037F09A
:1047100098BDA27C0AB19A0706D0D4E90812608934
:10472000D25C42431212CA540133E5E700008043D1
:1047300083B5F9F727FCF9F7D5FD154C154F019115
:104740000125A560064665602420BD71F6F79AFE36
:10475000114B6560C4F84833C4F808330F4B104C54
:1047600000254FF47A40BD7143F00103984740F2B1
:10477000FF33278823802DF02BFF019927804FF4EA
:1047800080632A4630462DF0A1FC27F07FFC00BF55
:1047900000400240536C012003000F00A0130900E9
:1047A000A005012038B5F8F7BDF8012807D0022888
:1047B00019D10E480E4B03600023436038BD0B4AED
:1047C0000C490D4B136008780C4C0023536054F8CF
:1047D00033100D79854202D151600448EEE7013370
:1047E000302BF4D1F9E70E20E8E700BFD0550120C7
:1047F0007C400800C86C0120A83F0800187708001A
:1048000070B5104B0122002604465A60C3F80065BB
:10481000FF2590F8210027F063FC94F8220084F82B
:10482000215027F05DFC94F8230084F8225027F0F3
:1048300057FC054B84F823501E60BDE870402CF0F7
:104840003FBD00BF00500240E85D012070B5044646
:1048500090B00163164601F1080000221D460023B6
:104860003CF0D8FB206B06AB102207A908303CF0C7
:1048700002FF10B105201BF09BFE069B102B0BD1F5
:104880004249042207A83EF089FF28B9404908227E
:1048900009A83EF083FF18B140F26E3014F0A2F880
:1048A000206B06AB042205A908303CF0E4FE00288A
:1048B000E0D1069B042B02D1059A142A02D935486F
:1048C0001BF0BAFE206B06AB0BA908303CF0D3FE00
:1048D0000028CFD1BDF82C300599012B0CD1BDF8A3
:1048E0002E20022A08D8BDF83A30102B04D81229FD
:1048F00004D1BDF83C1009B12748E1E7206B0C99C1
:10490000A16284F82420A376042206AB04A908300F
:104910003CF0B1FE0028ADD1069A042A06D11F4909
:10492000019204A83EF03AFF019A08B11C48C7E77B
:10493000206B06AB03A908303CF09DFE002899D1FE
:10494000069B042BA8D1039B6361236B1B6C238301
:1049500035B16D0866602E44E562E66010B070BD4A
:104960004FF48070E06229463EF063FE606018B943
:10497000E560E06A12F0EAFFE06A29463EF059FE7F
:10498000E0600028EAD16560F3E700BFA02B0900D2
:10499000A52B090007040800130C0800B7CC080079
:1049A0005E0108007FB5044608460D46164636F0FF
:1049B00036FC63685B69984202D01F481BF03CFEDE
:1049C000284636F0EBFB6368DB7C834201D01B4852
:1049D000F4E7284636F0D6FB63681B7C834201D09F
:1049E0001748EBE70DF10903019303AB00930DF1B9
:1049F0000B020DF10A030021284636F0EEFB636836
:104A00009A7C9DF80A309A4201D00E48D6E7284693
:104A1000A560267336F0F5FB04F1140204F11001D1
:104A2000284636F0C7FB63699B086361431E584202
:104A30005841607304B070BD930908007B090800F9
:104A400063090800A8090800F8B504464FF400609F
:104A5000C4E907000F46002115461E463EF0E9FD59
:104A6000A06128B9204637F050FCE06912F06EFFD3
:104A70004AF0DEF8606030B9204637F046FC16494F
:104A8000164840F048FDEB0744BF06F1FF360135FC
:104A9000B6F5105F09D3656205F59055A5623946F4
:104AA0002046BDE8F84000F01BB800214FF49050BC
:104AB0003EF0BFFD606228B9204637F026FC4FF477
:104AC0009050D3E700214FF490503EF0B2FDA06229
:104AD0000028E4D1F0E700BF26010800A0F4070099
:104AE00030B5044689B00D4602F0EEFA0022A56307
:104AF000002305F108003CF08DFAE36923624FF4CE
:104B00007F43E38720463EF0AFFF20463EF006FF9E
:104B10004FF490520021606A3EF092FE4FF49052A2
:104B20000021A06A3EF08CFE01A9204613F0EAFEA7
:104B3000054602F0DBFA1DB90849094840F0EBFCD4
:104B4000039B6363029B84F83D30059B5A009B00E6
:104B5000E36200232263636409B030BDA60208004B
:104B6000BCF407002DE9F04F91B002AF07EE901AA8
:104B7000C188396141687960032A8188F9610646F4
:104B80005AD0D11FD1F1000802F0FD0248EB010814
:104B9000052A01D148F002088B4AF86952F82350DF
:104BA000FB6969784FF0020B1BFB013303EB4303F6
:104BB0005B0007336A46DB08A2EBC3039D46FB6933
:104BC0004FF0030919FB013901EB81035B0002ACD3
:104BD00003EB800304EB410204EB49091C44034648
:104BE0001F3368465B11A0EB43139D46EA4617EE60
:104BF000900AFA62C7F830907C6300234AF8081BD9
:104C000041463DF044FC6B7800934A4601234146FF
:104C10003DF03DFC6B78009322465B4641463DF0FB
:104C200036FC4FF000094C463B69994580F2BD8047
:104C3000FB6ABB61002322E04FF00108ACE7BA69D0
:104C400032F9132014447F2CCCBF012200220AF831
:104C50000320CCBFFF220022A41A24B2E91C4FF08B
:104C6000000C2A78944501F1030144DBAA7812FB79
:104C700004F4002CB8BFFF3444F30F240133FA6965
:104C80009342DCDB52464946304649F0F0FE7B6BEE
:104C9000D7F830B07B613B63BB697B6309F10103EB
:104CA000FB60D7E903239342C7F82CB07DD06B7823
:104CB0000093BA6909F1030317EE900A41463DF0EB
:104CC000E6FBFB69013B31D2F9685246304649F0B8
:104CD000CEFE7B69FB62BB69C7E90C3B6B78009336
:104CE00017EE900A09F104035A4641463DF0CFFB06
:104CF00009F1020998E711F9022C07F1380000EBDD
:104D0000820211F9030C52F80CBC11F9012C184461
:104D100012FB04F23BF810E0002AB8BFFF320EEBA2
:104D200022222BF810200CF1010C9AE73BF81320FB
:104D3000144422B27F2AD4BF00210121802AB4BFAB
:104D40000022FF22A41A0AF8031024B2E91C4FF033
:104D5000000C2A78944501F1030108DBAA7812FBC4
:104D600004F4002CB8BFFF3444F30F24AAE711F970
:104D7000022C07F1380000EB820211F9030C52F803
:104D80000CEC11F9012C181AB860B86812FB04F287
:104D90003EF81000002AB8BFFF3200EB2222B868AC
:104DA0000CF1010C2EF81020D3E77A68002307F1EC
:104DB00020013046C7E909233B6208F04DFD3C372E
:104DC000BD46BDE8F08F00BFC02B09002DE9F04FB4
:104DD0002DED028B91B000AF984697F870307B6252
:104DE00097F874303B6197F87830FB60837B08EE6E
:104DF000101A012101FA03F30646013B18EE100ACE
:104E00009246FB6116F01EFF7368B861002407F13B
:104E100034013046C7E90E347C6308F01DFDB388C9
:104E2000FC6208FB03F303EBCA034FEACA02013B2F
:104E300093FBF2F30AFB03F3BB62033323F0030299
:104E40007A61BA6A23F003030132073322F00102C8
:104E5000DB083A627B60B6F80690FB6A4B4505DBDF
:104E60004437BD46BDEC028BBDE8F08F6B4608EEC3
:104E7000903A7B686A46A2EBC3039D46FB686D4689
:104E8000A3B1FB6A09F1FF39A9EB030900233B63D6
:104E9000BB69BA6A5C68294618EE100A07F130034C
:104EA000A047396B29B108461BF082FBD7F82C903C
:104EB000ECE7BB6A834202D0494840F02CFB3B69D7
:104EC000A3B1BAF1020F0CD0BAF1040F0ED17A6976
:104ED0002B46A9188B4209D01A6812BA43F8042B42
:104EE000F8E73A6A2B4651198B4210D108F1FF338B
:104EF000AB460024BB600FFA89F9B3889C420BDBF8
:104F000018EE903A9D46FB6A0133FB62A3E71A88CC
:104F100052BA23F8022BE7E7B8F1080F0BDCB8F11F
:104F2000000F11DDBB68072B0ED8DFE803F00F2759
:104F30000D360D0D0D45B8F1180F42D0B8F1200F08
:104F40004AD0B8F1100F39D0002309E07B6AE11094
:104F50008BB1E34303F007026B5C134103F00103E1
:104F6000FA6921B2134030464A463AF036FE01341F
:104F70000BF1030BC1E704F00702EDE77B6AA11018
:104F800043B1E34303F003035A006B5C134103F0A6
:104F90000303E5E704F00303F6E77B6A611043B11E
:104FA000E34303F001039A006B5C134103F00F032A
:104FB000D6E704F00103F6E72B5DD1E735F81430AE
:104FC000CEE79BF801309BF800201B0243EA024326
:104FD0009BF802201343C3E755F82430C0E700BF15
:104FE000002D080070B52DED028B8AB002A9B0EE3D
:104FF000408A34F096FE0E22002106A83EF020FCE6
:105000009FED480A9FED487A28EE000AA023C0EEE3
:10501000077AADF81A30ADF81C3004AA01248DF8D7
:105020001940B6EE007A77EE877AFCEEE77A17EE53
:10503000903AADF81E303D4B186A596A03C23C489D
:1050400001A9FCF77DFA00238DF8063004AA234657
:1050500006A902A846F0F4FF044630B1344801A97D
:10506000FCF7A0FA204636F0B6FE9DF8063063B194
:105070002F4801A9FCF796FABDF804604FF6FF73BC
:105080009E4205D12B481BF0EBFAFBF729FAECE71F
:10509000002020F083FB0446B8B16378012B34D1A3
:1050A0002378DB0731D506220DF1090104F1510007
:1050B0003EF074FB48BB04F1240204F13601304693
:1050C00046F0CAFFB0FA80F464090025694630460C
:1050D0008DF800508DF8015046F0C0FF4FF400717C
:1050E000304646F0D1FF29462A46304646F0AAFF10
:1050F000114B882101FB05F2D018D25AB24206D0DA
:105100000135052DF6D10D48BDE72046C1E7012345
:10511000837080F85A40FCF73FFF0AB0BDEC028B69
:1051200070BD00BF0024744900401C4690EF07008A
:1051300073F206009C020800380601208502080070
:10514000074A00234FF6FF7132F81300884205D159
:105150004433B3F5AA7FF7D1002070470120704790
:10516000380601202DE9F04790B00D46044637F08F
:1051700000FDA84200F02D81002D00F01481974918
:105180000B7853B10020F6F77DF9954A00231360A0
:10519000944A0B701360944A1360944E944930689B
:1051A000029002A846F0C1FF002840F08F8091498C
:1051B00091F816335A09EC231341DB0740F1F080D4
:1051C0008D4B9A68002A00F0E7801A6842F480024A
:1051D0001A608A4A0023C2F8DC30894A012713701A
:1051E0004FF00508874A0392032308A920208DF871
:1051F00020708DF82280ADF8243046F00BFF002897
:1052000064D1CDE90900804B039A089308A9402096
:1052100046F000FF002859D1CDE908000A90039A12
:105220008DF8207008A922208DF8228046F0F2FE29
:1052300000284BD1CDE908000A904FF40073039A7F
:105240008DF8207008A92320ADF8223046F0E2FE48
:1052500000283BD1CDE908000A9038438DF82000A2
:10526000039A08A9A02046F0D5FE78BBCDE9090035
:105270004FF4DC53039A089308A9A12046F0CAFE14
:1052800020BBCDE908000A904B23039A8DF820300B
:1052900008A9384646F0BEFEC0B903A846F0BCFED9
:1052A000A0B99DF8103004A93B4302208DF81030BE
:1052B00046F008FF50B9554A7068516806AB03C301
:1052C00006A846F0CFFE08B946F0B4FE01900FF0F4
:1052D00005FC019836F07FFD002D67D04C4DDFF8BE
:1052E0004C9100273E46A5F1080A882303FB07A33B
:1052F0004FF6FF7845F8046C25F8088C502283F8A7
:105300005A60002105F8066C28463EF099FA0137EC
:10531000A5F108014846FCF745F9052F25F8088C4A
:1053200005F18805E1D13B4B3B4DC4E90D3406A89E
:1053300046F076FE36F04FFD9DF81A30374A384871
:105340006E73190903F00F03515CD35CAB729DF8C7
:1053500019306972190903F00F03515CD35CE972CB
:105360002B7330491F2308AA3BF02FFC002833DDA4
:1053700010AB184400F8206C08A837F009FC2A4943
:10538000224604F11C00FCF7F7F82BF04BFB10B0A1
:10539000BDE8F047FDF740BA4FF480030B6018E713
:1053A00042F2020092E746F0BEFE8FE71E48214619
:1053B000FCF7F8F8E36813B1204600F039F80F4A1B
:1053C0000023C2F8DC300E4AC4E90333C4E90133D8
:1053D000137010B0BDE8F0872846CEE7696C012055
:1053E000B4610120B8610120BC6101205AEF0700BF
:1053F0003BCA070000E100E090640120C061012089
:10540000776C012000E00020010404015EEF07003A
:1054100040060120E9B70600B705012088130900FE
:10542000511309003E130900A1D90200A5B20300DF
:1054300013B50D4B01901878FF2813D046F0F8FDF6
:10544000019904460948FCF7ADF80023CB6081F8C8
:10545000443034F0080305D0204602B0BDE81040C7
:1054600036F0B9BC02B010BDA7050120C5A50600E5
:1054700038B50369044663B146F0FAFD236905486F
:105480000122002583F829205D602169FCF78AF854
:10549000256138BDA9D705002DE9F74304460F461D
:1054A000154648F019F8DFF85890064688466369B3
:1054B0009D4212D80DF1070028F0E2FA04F10C0029
:1054C0002A46394646F066FC04469DF8070028F057
:1054D000FBFA204603B0BDE8F08347F0FDFFA26869
:1054E000831B61EB0801934271F10003E2D2FAF7EA
:1054F000F7FFD9F82430002BD9D00024E9E700BF0A
:10550000C06101202DE9F74FDDE9116B044600274A
:105510000D469DF830009DF83410DDF83C809DF874
:1055200040A0A78291469DF83820A075C4E9015398
:10553000E17522762782E760E6B1244B7268228209
:10554000D3F88411336819B31846019200930EF012
:1055500019FADDE90032C8B1394690B23EF069F877
:10556000228A316807463EF02BF9E76000203DF0C3
:10557000DCFEE061BAF1000F20D1B8F5007F0AD956
:10558000134A4FF4007113481BF05EF8E360EDE737
:10559000E360E161EEE7A4F8128084F826A0AB791D
:1055A00023B1A4F8149003B0BDE8F08F60685A46A8
:1055B000214603B0BDE8F04F37F02ABCB8F5FF7FB5
:1055C000E9D9054A4FF4FF71DDE700BFC061012052
:1055D00017F00700F517080022F00700F0B5478C18
:1055E00085B00C46164617B91B481BF039F84368BE
:1055F0009A791AB919491A483FF08DFFD86835F0E1
:10560000B8FF054637F041FB0023002ECDF80530EA
:105610008DF809304FF0010314BF022100218DF8ED
:10562000043002230C43ADF80A306B44ADF802405D
:10563000ADF80670039301A9284646F02DFD48B148
:1056400020F00203112B02D1FAF74AFFF3E736F0FC
:10565000C2FBF0E705B0F0BDF6040800E722080041
:10566000C88508002DE9F04F43689A7985B0044653
:105670000D466AB1D86835F07CFFA37D0146A08A4B
:10568000C3F340132A4605B0BDE8F04F37F014BB12
:105690004B6890F82610428A21B19A4206D02848D9
:1056A0001AF0CAFF9A4201D22648F9E7A08A2A4690
:1056B0004FF6FF7137F02CFB00264FF6FF7A4FF0C4
:1056C000020B214B33F8167057452FD094F81680F3
:1056D00018F0060F2AD00DF10603618C039302AA7D
:1056E0003846CDF808B046F0E9FC43F20143984251
:1056F00023D10023ADF8063018F0040FBDF8069052
:1057000008D019F0010F05D0A08A01232A46394696
:1057100036F0B6FA18F0020F08D019F0020F05D0D3
:10572000A08A02232A46394636F0AAFA4436B6F54C
:10573000AA7FC6D105B0BDE8F08F36F04CFBDBE7A1
:10574000200C0800300C08003806012008B501487C
:105750001AF0FEFE1506080070B543685D68044641
:10576000E86835F006FFAB790A4601462BB1A08AFE
:105770000023BDE8704037F09FBAA57C5068238AAB
:1057800025B1984206D006481AF056FF984201D932
:105790000448F9E7A08ABDE8704037F0B9BA00BF05
:1057A000200C0800300C080070B5064686B008468C
:1057B0000D46144637F069FA00234FF40072204872
:1057C000019401A9CDE90223ADF810508DF81430F1
:1057D000FBF7B6FE00223146284646F05BFC112856
:1057E0000446F7D030B1164801A9FBF7DBFE20468E
:1057F00036F0F1FA9DF81430B3B1BDF8100037F06F
:1058000044FA01A90E48FBF7CDFEBDF8121089B28B
:1058100091B140F20513994209D040F20F13994219
:1058200008D008481AF01CFFFAF75AFEE2E70648CB
:105830001AF024FF0548FBE7039806B070BD00BFCF
:10584000839D0600830B0800AC030800BD0308001D
:1058500070B50A4D04464FF6FF76A38C9BB213B980
:1058600094F82D302BB1E38C9BB2B34201D06B6A1C
:1058700003B170BDFAF734FEEFE700BFC06101204D
:105880002DE9F3479846C3690A9D04460F4616461C
:1058900013B93A481AF0E4FEC38C4FF6FF799BB275
:1058A0004B4504D14FF0FF3002B0BDE8F08737F030
:1058B00043FA0028F6DB7219904204DA40F25341B1
:1058C0002F481AF0C1FE238D934202DA40F20C41B8
:1058D000F6E7A28C984216FA82F2A8BF18468242D6
:1058E00010D9DFF8A0A0A38C9BB23BB1E38C9BB294
:1058F0004B4503D0DAF82430002B39D0DAF82430C5
:10590000002BCFD1E38C4FF6FF729BB29342C9D0EC
:105910000DF1070028F0B4F894F82A3004EB830363
:10592000D3F81C90A38C9BB22BBB2A464146484619
:105930003DF046FFA38C15FA83F39BB2A384A08CA1
:105940003246394619FA80F03DF03AFFA38C9DF8B3
:10595000070016FA83F39BB2A38428F0B5F894F8F5
:105960002D30354413B9204645F06FFE28469BE79D
:10597000FAF7B6FDB7E70025E1E700BF170D08000D
:10598000780A0800C0610120F0B51646354A0D4678
:10599000117A85B004461F4611B1137D3BBB01212E
:1059A0000C2303FB012262602879012144F078FE78
:1059B0000121307944F074FE0A2020F055F828794E
:1059C000002144F06DFE3079002144F069FE03208F
:1059D00020F04AF8307944F0AEFE70B9307926F004
:1059E0007FFB287926F07CFB1F481AF0FFFD4368F7
:1059F000002BD9D11D481AF01FFE287944F09BFED8
:105A00000028EBD0327901924FF0CC72029207223B
:105A1000ADF80C20164A2B79009397421AD94FF013
:105A2000C862029263723079A072FEF7C9FB2879CE
:105A3000FEF7C6FB636801221A726068694620F0AF
:105A4000C7FA0C4B98420BD0204637F0CBFA052012
:105A50001AF0AEFD084A9742E4D94FF08062E0E7C1
:105A600005B0F0BD5C0401208A0508001B1E08007B
:105A70007F1A06000000AD0B8FD0030038B54368D5
:105A80001C681A790623C4F800351E4B05463420DD
:105A900000FB0233022283F82D200023C4F888156E
:105AA000C4F84435C4F8483501232362A360D4F810
:105AB00050311BB9D4F82431002BF8D04FF4A87121
:105AC000204644F0D7FD01236361D4F80431002B54
:105AD000FBD04FF48271204644F0CCFDD4F8243141
:105AE00073B120464FF4927144F0C4FDD4F8C4342D
:105AF000C4F8C4340024686820F04EFA204638BD4B
:105B00000124F8E7E86001202DE9F04F16464268CD
:105B1000DFF880801C46137912688B460621C2F894
:105B20000015342202FB0383022289B0054683F864
:105B30002D204FF6FF794FF0010A69685CB9144BCC
:105B40006868019320F028FA019B184609B0BDE867
:105B5000F04F2DF0CDBF0023CDE905364C4527464B
:105B600028BF4F460793049708798DF80CA08DF84D
:105B70000DB04FF0340C03AA096800FB0C802EF026
:105B800067F8034A90420346DAD1E41B3E44D4E767
:105B90000000AD0BE86001202DE9F04F1D465E4B83
:105BA0000746D3F8000510F00F0085B0144606D064
:105BB000A3F54043D3F800351B0704D10120574B10
:105BC00003EB001078607B6813B955481AF034FD78
:105BD00091F804A0D3F8089087F809A05046FEF782
:105BE000EFFA3CB32479BC722046FEF7E9FA25B3FC
:105BF0002D79FD722846FEF7E3FAD7F804B0494E36
:105C00009BF80480242303FB08631B7F63B9484689
:105C1000FAF7A2FC8146B8F1000F11D1B0F1206F64
:105C200002D0B0F1A05F0ED1384637F00EFA052051
:105C30001AF0BEFCFF24BC72D9E7FF25FD72DCE739
:105C4000B8F1010FF0D1242303FB08F3F11800226F
:105C5000DBF80070F2504A60504644F050FD03A853
:105C6000CDF80CA01FF0F8FD039B03F5E0730122B3
:105C7000FF2C40F8232049D0204644F040FD204628
:105C800044F01CFDFF2D44D000212846019544F02E
:105C900007FD019B242202FB08F20192B21838464C
:105CA00082F82150FF2582F820500222C7F8602593
:105CB0000022C7F808A51146C7F80C45C7F81035EB
:105CC000C7F8249544F062FD019BC7F8C055F3580E
:105CD00013B14022C7F804230721C7F800155BB1B0
:105CE000DBF8000040F30730F5F7F2FBDBF80000CB
:105CF00040F3073033F069FA242303FB08660023DE
:105D000073770123337705B0BDE8F08F4FF0FF3490
:105D1000B8E74FF0FF33BDE700F00240EC0C09009C
:105D2000D21E08008860012010B50D4B42689A42CF
:105D3000044611D010339A4210D10123094A01219F
:105D4000D154607A1FF066FCA07A1FF063FCE07A01
:105D5000BDE810401FF05EBC0023EFE710BD00BFA0
:105D6000EC0C0900606C01202DE9F04F17464268E9
:105D7000DFF86090DFF860A0DFF860B087B0984689
:105D80001368019306460D46B8F1000F01D10120BA
:105D900017E07268019BD468444528BF44464B45D0
:105DA00004D12246294650463DF00AFD706802A9FA
:105DB000CDE90254CDE904741FF0F6FF584503D035
:105DC000002007B0BDE8F08F25442744A8EB040865
:105DD000DAE700BF00F0024000E000200000AD0B59
:105DE0002DE9F04F15464268DFF860A01368DFF830
:105DF0006080DFF860B087B081460E4601930DB930
:105E000001201BE0D9F80420019BD768AF4228BFCE
:105E10002F46534515D13A46314640463DF0D0FC19
:105E20004246D9F80400002402A9CDE90227CDE9B1
:105E300004441FF0B9FF584505D0204607B0BDE81F
:105E4000F08F3246EDE73E44ED1BD8E700F002400C
:105E500000E000200000AD0B10B50446406820F0C3
:105E6000C1F994F8260026F03BF994F8270026F0B3
:105E700037F994F8290026F033F994F8280026F031
:105E80002FF961680A4A4FF6FF73E3842385914234
:105E90004FF00003C4E90433C4E90733A36103D01E
:105EA0000832914203D10123024A0021D15410BD8E
:105EB0007C020120626C01202DE9F3471E464368F5
:105EC0001B68D3F81435013304468846154602D1C1
:105ED0002D481AF0B1FB47F0FFFADFF8B4A00746EF
:105EE0008946A3699D423AD86368186840F3073031
:105EF000002846DA04F110072A464146384645F0A4
:105F000049FF94F8253005468BB104F124010122A4
:105F10003846019145F066FF0199606820F0DEF88F
:105F200094F8290044F0EBFB002384F825306368E3
:105F30001A68130B42F30732002A07DB03F01F0134
:105F400001238B405209114941F822301DB90B231E
:105F500033604FF0FF35284602B0BDE8F08747F0C8
:105F6000BBFAE368C01B61EB0901984271F10003C1
:105F7000BAD2FAF7B5FADAF82430002BB1D00025FE
:105F8000E9E7F5F793FAB5E73505080000E100E029
:105F9000C06101202DE9F04F83B0984643681B682B
:105FA000D3F80C35013300AF81460D46144602D1BB
:105FB0004F481AF041FB002A71D001F0604ABAF153
:105FC000005F10D0802A20D94A4BD3F88431E3B146
:105FD000002110460CF07EFE034629462246184654
:105FE0003DF0EEFB0546D9F80430187920F0EEF8C4
:105FF00090B905F06043B3F1005F10D03E4AC8F895
:1060000000203E493E483FF091FAE31D23F007038C
:10601000ADEB030D6B46E0E7FAF762FAE3E7D9F878
:10602000046096F804B0584620F0D0F808B1354A1C
:10603000E5E7354B242202FB0B324FF4907154619B
:10604000956030687A6044F015FB30684FF4AC71AD
:1060500044F010FB7A68316890685369C1F84405D0
:10606000C1F848353168012088605268E2B10023E8
:10607000C8F80030D9F80430187920F0A7F80028C3
:1060800032D1BAF1005F0AD01A4BD3F8843133B160
:1060900028460DF077FC10B128460DF0ABFA2046EB
:1060A0000C37BD46BDE8F08F3268D2F82001D2F837
:1060B000581118B90029F8D0144A09E00029FBD179
:1060C0000121D1603168D1F85821002AFBD0104A53
:1060D0000D4B242101FB0B33002159610C4BC8F8F7
:1060E00000209A42C3D08CE7FAF7FAF9C2E700BF62
:1060F0003C050800C06101200A00AD0B95120800A4
:10610000BCF407000B00AD0B506101200800AD0B83
:106110000000AD0B10B50379FF2B04460ED0084AE2
:10612000002142F8231000791FF0A8FC20791FF00D
:1061300093FD207925F0D4FFFF23237110BD00BF0C
:106140000C1E01202DE9F04F2DED048B91B00CAF0A
:106150000446B7F87C00786097F8900097F868C01C
:10616000F860002084F89500B7F8548097F888000C
:10617000D7F880B0B7F8946097F89C50CDF828C055
:1061800097F864C0CDF824C097F860C0CDF820C05F
:1061900097F85CC0CDF81CC097F858C0CDE9058CC5
:1061A000B7F850C0CDF810C0B7F94CC0CDF80CC04E
:1061B0000028B7F948C00CBF4FF48070FF2004F1ED
:1061C0000809CDE9010C00904846B0EE408A07F07E
:1061D000C5FB97F86C3084F8923097F8703084F8EB
:1061E000933097F8743084F89430B7F88430A4F87A
:1061F0008C30FB6883F0010384F8963097F88C307C
:1062000084F8973097F8983084F898301DB108F1E9
:10621000FF335D425D41A4F88E604FF47A7384F8D9
:106220009950B3FBF6F64FF0000AA4F890607B6833
:106230009A4533D34F4BA366BBF1000F1BD09BF89D
:10624000040037F0E5F9B0B1002204F168050092CE
:10625000B7F8A0305946284601F00AFA002800F0A5
:106260008380454BA3665946284636F012FF9BF8BB
:10627000040037F0E2F9B0EE480A204600F082F858
:106280003E49484607F010FCF968204637F038F8D8
:106290001437BD46BDEC048BBDE8F08FBB6F03EB3C
:1062A0000A0898F9013098F80150BB6008F1020320
:1062B00009EE103A05F07F05484639F050FE0028F7
:1062C00039D094F8973008EE903ABBB36B4608EE9D
:1062D000903A05F1080303F0F803ADEB030D98F8CD
:1062E00000208DF830200CAB19EE101A6E1C2A46D7
:1062F0000DF131003B603DF063FA00963B68666A41
:10630000A06801220021B04718EE903A9D46484609
:1063100039F073FEBB68002B23DA6E1C023518F8C7
:106320000500FF2808BF4FF4FA70023615F0EAFCAA
:106330005AFA86FA7BE7FAF7D3F8BDE70123009310
:1063400018EE901AA068666A43460122B04700958D
:1063500019EE103A18EE902AA068666A0121B0473B
:10636000D5E72E460A20E0E7054BA366284601F054
:1063700023FA80E79C360800445E0800780101207B
:10638000F89008002DE9F0412DED028B90F898303F
:1063900086B00446B0EE408A1BB9F7EE007A37EEBD
:1063A000C08AA36E324A934210D1DFED327A68EE92
:1063B000277A04F16800FCEEE77A17EE903A99B27A
:1063C00037F0B2F984ED228A012015E02A4A93427F
:1063D0000CD1DFED2A7AE06EB4EEE78AF1EE10FA26
:1063E000CCBF0121002136F0A7FEEBE7B4F88C30DA
:1063F000B3F5807F05D1002006B0BDEC028BBDE86F
:10640000F08104F10808404639F0A9FD0028F2D0D7
:10641000DFED1B7A94F8976094F88C20676AA06887
:106420008DF8142068EE277AFCEEE77ACDED037A3A
:106430009DF80C305EB18DF81530022300930122D7
:1064400005AB0021B847404639F0D7FDBAE7012532
:106450008DF813302A4605AB31460095B847676A78
:10646000A06800950DF1130332462946EAE700BF04
:10647000F890080000FF7F47445E0800A4707D3F4D
:1064800000007F432DE9F04F2DED028B99B090F87D
:10649000973006AF0446EBB1826EB14B9A4219D1E8
:1064A000683036F00BFE94F89430834208D1002314
:1064B0003B6138694C37BD46BDEC028BBDE8F08FBF
:1064C0002AF0FEFE0021D4E91F2384F8971020460D
:1064D00045F076FFE3680BB90123E9E7204636F083
:1064E00023FF0028E3D104F10805284639F03AFDDE
:1064F00038610028DBD094F86210002900F0A480F5
:106500000023636404F13C09A369A068984720460E
:10651000D4E91D23012145F053FF284639F01AFF25
:106520006B4607F130024946284608EE103A39F02A
:1065300024FD002800F02B817B8EFE8E07F13000B9
:10654000F61A4FF0200A94F85230BAFBF3FA39F0F9
:10655000FDFAB0EBCA1FB6B24FEACA1800F2858046
:106560000123FB6180B2B04680239B004009FB60A1
:106570000130073323F00703F862ADEB030DFB6A2C
:106580009B00073323F007030DF1180AADEB030D51
:10659000B4F89030B3F5807F0CBF01230223BB60B9
:1065A000FB6853447B6000230DF1180B7B627A8EED
:1065B000FB8E9B1AB4F888209BB2B2F5807F3B62B9
:1065C00017D00020B4F88A3094F88610049007F1B0
:1065D0003000039094F89900003818BF0120029011
:1065E00000200190B4F88C000090D2B2284639F017
:1065F00025FDB4F88E3087F82B307B6A012B04BF61
:10660000B4F8903087F82B30284639F0A8FC0123E5
:1066100094F899200093A068666A07F12B03002183
:10662000B047284639F0E9FC0023C7E90533BB8AA7
:10663000FA699A423ED87B6ABA6801337B6297F85E
:1066400024309342B3D3A2E0E06800283FF444AF83
:1066500008F0C8FA814600283FF43EAFB4F888300D
:10666000B3F5807F7FF450AF4AE73B8EB88EC01AF7
:1066700080B2B8FBF0F8B8F1010F38BF4FF0010855
:10668000B6FBF8F308FB13669AB2B6B2FA611EB114
:10669000134601339BB2FB6118FB00F080B2B0FBE4
:1066A000FAF293B20AFB1202002A3FF45EAF013302
:1066B0009BB25AE700237B643B8E7A8EB98EBB87F0
:1066C000BB69A7F84010396AD31888459BB288BFC8
:1066D0003A6AFB8797BFBB699B184344D21888BFAF
:1066E000A7F842303B6A98BFA7F84220A3EB080303
:1066F0009BB207F13C003B6239F028FA94F8523023
:106700000822B2FBF3F3FA6AB0FBF3F39200002124
:1067100058461E463DF094F8FA68002150463DF078
:106720008FF840F20713A4F856307B6A012B19D179
:1067300094F8983063B1062384F8563053465A468D
:1067400007F13C01284639F05BFC94F8963012E0E2
:1067500094F85820002AF8D084F85730EEE700BFAC
:10676000445E080053465A4607F13C01284639F07A
:1067700047FC94F895306BBB284639F0F0FB7B69F9
:1067800001337B61BB6943449BB2BB6158BB18EECC
:10679000103AD9F808909D46B9F1000F7FF4C0AEC9
:1067A0004FF00108284639F0DAFB94F89920CDF82B
:1067B000008004F192034946A068666AB047284603
:1067C00039F01BFC2AF096FD84F89780284639F0B2
:1067D00027FC6EE653467A689342CDD01A68D243BE
:1067E00043F8042BF7E7B3B294F899200093A0681C
:1067F000666A53460121B047284639F0FEFB2DF06A
:10680000A5FF14E710B50C4B426A9A42044611D01A
:106810000021806A36F090FC4FF47A701FF024F962
:10682000A06A012136F088FC4FF47A701FF01CF941
:10683000012010BD0020FCE79C3608002DE9F7433D
:106840001C464B1ED3F1000848EB030815463C4B91
:1068500042690A9F9A4206464FD100258DF807509B
:106860002744BC421CD1C5B19DF807307068C5F102
:10687000080503FA05F501220DF107018DF807500F
:10688000FFF7AEFA0121306A36F056FC01201FF006
:10689000EBF8306A002136F04FFC03B0BDE8F0831E
:1068A000013515F007059DF807307068A14613D132
:1068B00048EA430301220DF107018DF80730FFF785
:1068C0008FFA706801222146FFF78AFA99F80030A2
:1068D0008DF807300134C4E7C5F109029340C5F1D2
:1068E000080208FA02F2134322782A4113438DF872
:1068F000073001220DF10701E6E78069414636F0D5
:106900001BFC012D14D12744BC42C6D001222146D4
:106910007068FFF765FA0121306A36F00DFC01203E
:106920001FF0A2F8306A002136F006FC0134EBE7D4
:1069300070683A46214603B0BDE8F043FFF750BA0D
:106940009C36080010B50A4B42699A4204460CD0A6
:106950000021806936F0F0FB04201FF085F8A06963
:10696000012136F0E9FB012010BD0020FCE700BF4B
:106970009C3608002DE9F0430446A7B0816100224F
:10698000002301F108003AF045FBA06901AB8A221F
:1069900003A908303AF06FFE10B1052019F008FE87
:1069A000019B8A2B06D16A49022203A83CF0F6FE1D
:1069B000054618B140F26E3012F014F8DDF81630CA
:1069C0002381DDF82A30BDF8288084F82180A3F1E6
:1069D000030CDCF1000343EB0C0384F82030DDF8FA
:1069E0001E30A380DDF82230E38001460C20DDF864
:1069F0001A70DDF83A603CF01CFE564B0360B8F1AB
:106A0000100F4FF0807383608580E0612ED1372FA7
:106A100002D894F820300BB3DDF84230E360DDF8A3
:106A200046302361DDF84A30636194F82110A38871
:106A300007294FF008008CBFCA080122B0FBF1F013
:106A400000287CD112FB03F39AB299071CBF22F0F5
:106A500003020432628127B0BDE8F0834FF47873FB
:106A60004FF4F840C4E903031F23DDE7B8F1080F32
:106A700057D816B9012606FA08F6002110203CF076
:106A8000D8FD354B0360B3B2054683600C2000216E
:106A900058433CF0CEFD012E686036D04FEA86099F
:106AA0001FFA89F9002148463CF0C3FD8046A069E1
:106AB0000022002308303AF0ADFAA06907F10E0277
:106AC00092B2002308303AF0A5FAA06902AB4A4618
:106AD000414608303AF0CFFD074600287FF45DAF0D
:106AE000029B994507D01D4819F0A6FD58F82120B2
:106AF000284636F0C3FCB9B28E4207F10107F5D83B
:106B000040460CF077FDE5618FE7002211462846EC
:106B100036F0B4FC6FF07F423146284636F0AEFCCA
:106B2000F1E70C2F81D0282F3FF47FAF27F010031F
:106B30006C2B3FF47AAF0A48394619F085FD4B4378
:106B4000DA061CBF23F01F032033DB08638182E7D2
:106B5000C82B0900D860080090670800410B0800A6
:106B60006D06080070B5634CD4F8C03033B92368A3
:106B7000002B66D1BDE870402BF084B85E4DAB426F
:106B8000F5D05E4A934233D1002104F1C00036F0C3
:106B9000B7FBD4F8CC302BB193F82A206FF3410225
:106BA00083F82A20D4F82831554A934219D1D4F8D1
:106BB0002C615448544B002250F8041BB14208BFCA
:106BC000197802F1010204BF01F1FF311970042AA2
:106BD00003F10103F0D14D4836F091FDC4F8C050E7
:106BE000C5E74B4A9342F9D1484835F069FBF5E7D0
:106BF000484A93421FD194F8573173B104F1C00051
:106C000030F056FC2AF05CFB0021D4E94F2304F15C
:106C1000C00084F8571145F0D3FBD4F8CC302BB129
:106C200093F82A206FF3410283F82A20D4F8282110
:106C3000374B9A42D7E7384A9342CFD125F006FA2C
:106C4000CCE72D4EB34295D0344A934210D16068C0
:106C5000334B984201D136F0F8F9A06936F07DFD4A
:106C6000206A36F07AFDA06A36F077FD266081E76B
:106C70002C4A93420DD16068294B984201D136F0DD
:106C8000B1F96269224B9A42F0D1274835F018FBDE
:106C9000ECE7264A93421ED1002594F830002844A0
:106CA000C0B2013525F01CFA082DF6D1E368187939
:106CB00025F016FA6369187925F012FA636A1879D3
:106CC00025F00EFAE36A187925F00AFAE3691879D3
:106CD00025F006FACAE7164A934203D1054800F0A8
:106CE000B1FDC3E7134A9342C0D1024801F07CF9D9
:106CF000BCE700BFE00801209C360800F0620800F5
:106D0000F8900800AC140900646C0120080A012006
:106D1000445E08000C6408007C7108007864080078
:106D2000E808012018660800F4080120D08B08004C
:106D3000F8910800E4950800F8B5C38A13B916481D
:106D400019F07AFC90F850301B070ED500F12401A1
:106D500000231D46048B9AB2944218D890F8503004
:106D600043F0020380F8503002E0416A0029EFD17D
:106D7000F8BD94B20CFB0414013204F80E50478B9A
:106D8000B0F818C096B2B742F3D80133E2E7002258
:106D90001FFA83FEF3E700BF070A08007FB5044629
:106DA000C08A984202D8294819F046FC94F850004D
:106DB000050746D504F12400258B02FB050043544A
:106DC00094F85030258BD807238CA1EB030191FB5D
:106DD000F5F305FB13110EB254BF04F12C0001A80A
:106DE000002EA38BBCBF49190EB213FB06F39BB256
:106DF0000380A18B0B448380638C618BD21A92FB3E
:106E0000F1F301FB132215B2002DE38BBCBF521826
:106E100015B213FB05F39BB24380E28B1344C3808E
:106E200094F85030DB0705D504F12C0201A9104677
:106E300038F096FE94F8503043F0010384F8503057
:106E400002E0606A0028B7D104B070BD070A0800EC
:106E5000F0B591B040236A4604460F4639F0B5FEBE
:106E6000051E24DB3F2D1CDD0021681C3CF0E1FBEE
:106E70002B46064602463946204639F0A6FE00213A
:106E8000715510203CF0D5FB0A4B0360C0E9025657
:106E900004462946304644F0A5FB6060204611B008
:106EA000F0BD2946684617F0C5FC0446F6E70E24F7
:106EB000F4E700BF28F707002DE9F04F2DED028B16
:106EC0001F46002380F89030044681668FB04FF44F
:106ED00091600D46904619F00BFBE066C369002BEC
:106EE00000F09E802846984786B2E36EA06E1B692C
:106EF000984783B208EE103AE36EA06E5B6998473C
:106F000083B208EE903AE36E5B6A04F1080B002B43
:106F100000F08880A06E9847B0F1000918BF4FF0CC
:106F20000109E36EDD6A15B1A06EA8470546E36E60
:106F30009B69002B7DD0A06E98475FFA80FAE36EC4
:106F40001B6B13B1A06E98470346E26E526B002A8A
:106F500072D0A06E0D9390470D9BCDE909300021B2
:106F60004FF48073CDE90033CDE9075A18EE903A1B
:106F7000CDE90569CDE9031118EE102A02915846B2
:106F800006F0ECFCE36E1B6A13B1A06E984783B267
:106F9000A4F88C30E36E9B6B002B4FD1B4F84830D3
:106FA00094F852205343DB10A4F88E30E36EA06EA9
:106FB0005B6804F170019847B4F88C30B4F84A006B
:106FC000B4F88E1040F2873200FB0131606F3CF064
:106FD00075FD87F0010384F89130E36E9B6A002B06
:106FE00034D0A06E984780B2A4F888004FF47A732A
:106FF000B3FBF0F0A4F88A00B8F1000F03D04146CB
:10700000204600F027F81249584606F04DFD394653
:1070100020460FB0BDEC028BBDE8F04F36F06ABAE7
:10702000102662E7072E8CBF4FF000094FF00109D0
:1070300077E74FF0020A82E710468EE7A06E984786
:1070400080B2A4F88E000028B0D1A7E73C20CBE79F
:107050007801012010B5B0F84C305A2B04462CD0E2
:10706000A3F5877CDCF1000343EB0C035A2926D0FF
:10707000A1F587704242424193421FBFB4F84830A5
:10708000B4F84A20A4F84820A4F84A3004F10800D3
:1070900039F012F90B4B9C4207D12AF0F3FDB4F8FA
:1070A0004A10B4F848002AF077FCE06848B104F1CF
:1070B0002C01BDE8104039F026BB0123D6E70122A0
:1070C000DAE710BDA009012010B5064C236813B9FA
:1070D000054826F0D5FCBFF35F8F2368013323609A
:1070E00010BD00BF80640120516C012010B50F4B12
:1070F0001A6812B9022024F0DDFF1A68013A1A60FA
:107100001B6893B9BFF35F8F094B9A686AB1094A4C
:10711000127852B9EFF3108072B607491C680C6000
:107120005C684C609A6000B962B610BD8064012052
:1071300090640120516C012000E100E00C4B1868C4
:10714000A8B1C10710D4820710D4430706D5094B54
:107150001B78002B14BF03200220704710F4D81FA7
:1071600014BF032006207047042070470520704795
:10717000B8640120B86C01202DE9F04FA04BADF2AE
:10718000944D16010190894617460FCB03AD85E853
:107190000F0004362A46002352F8044BD4F800B5F9
:1071A000BBF1000F10D1D4F8601500290CDAD4F827
:1071B0006415002908DAD4F86815002904DAD4F82F
:1071C0006C150029C0F2B5800133042BE4D10024F2
:1071D0002546D4E0012231460CF062FCC6E00132C3
:1071E000D20019F800B092B280201BEA000F48F2DA
:1071F0000C0E08BFE64625F813E001339BB293421C
:107200004FEA5000F1D101318AB2D30097429BB2CC
:107210001046E4D84FF4004225F8132001339BB206
:10722000760825F81320B6B200231422C4F80C35D2
:10723000C4F80435C4F80825C4F81435C4F810356A
:10724000C4F82055C4F82465C4F82835C4F82C3592
:10725000019B5B681B79C4F8603501254FF0FF3353
:10726000C4F864354FF48871C4F868352046C4F812
:107270006C35C4F8005543F0FDF9A560D4F8103121
:107280000BB34FF48871204643F0F4F90023C4F89F
:1072900000354FF0FF33C4F86035C4F86435C4F8E6
:1072A0006835C4F86C35002022F0B8FC043041F198
:1072B0000001CAE900010DF2944DBDE8F08F0021F4
:1072C00048F2050CA0E7F9F70BF9D7E719F802B077
:1072D00008214FF0800CD4F804E0AEEB030EBEF1B1
:1072E000460FF8D96368D5F808E51BEA0C0F4EEA9B
:1072F000060EC5F808E512D0D4F804E0AEEB030E94
:10730000BEF1280FF8D9D5F80CE501394EEA060E82
:10731000C5F80CE54FEA5C0CDDD101325CE0D4F835
:1073200004E0AEEB030EBEF1110FF8D9EBE762B645
:10733000B9E740F284439E4221D9DFF8D48085F832
:1073400000B0284644F0F3FED8F80020DFF8C4A0CF
:10735000B24212D2DAF8D80008B1C8F800B02A78E0
:10736000002A3FF437AF31463CF07EF9CAF8D80026
:10737000DAF8D8200AB1C8F80060DAF8D850DFF897
:1073800098A0002022F04AFCDAE90023904271EB39
:107390000303F6D30DB1002C91D172B6019B194CA9
:1073A0005B6802A81B7902931EF056FA029B164AEC
:1073B00001269E40D2F8FC3043F08073C2F8FC30C6
:1073C00023684FF4307843F001030546236008FB3F
:1073D00007F800226068134691B28F423FF676AFFD
:1073E0006268D21A462AFBD963681B1A43459ED3AA
:1073F000064B4FF4964043F001039847E9E700BF7E
:1074000070EF0700001000E000ED00E090140900AC
:10741000A8640120C0610120580A0120F7B5044684
:1074200000270DF106000D468DF8067044F07FFE32
:107430009DF80630E3B10DB9012011E00DF1070010
:107440008DF8077044F06BFE9DF807606EB1AE4298
:1074500028BF2E46F1B2204644F063FE10B1002052
:1074600003B0F0BD3444AD1BE5E7F9F739F8E2E7C6
:107470000D4E4FF48071304643F0FCF80123336029
:107480002544AC4202D101207060E9E7D6F8003112
:10749000002BFBD04FF48071304643F0EBF8D6F868
:1074A000083504F8013BECE700D0004010B50A4B6A
:1074B00082699A4204460CD00021C06935F03CFE36
:1074C00004201EF0D1FAE069012135F035FE0120DB
:1074D00010BD0020FCE700BF9C3608002DE9F347F3
:1074E000044600200D4616469846F5F70BFA00288C
:1074F00002DA002019F048F82D4B770043F82040BD
:10750000002138463CF095F8A06010B9384610F0DC
:107510001DFADFF8C09099F80070E7B91EF04EFA36
:10752000DFF8B4A0CAF8000010B9224819F05EF8DC
:10753000214B224A1F60224B6946CDE900371EF0DD
:10754000B1FCDAF80000394643F034F9DAF80030DB
:107550001B6801221A6099F80030013389F8003065
:107560002B79237101220023E381A3712382A68159
:10757000E27184F805806361A3612879FCF720FE3D
:10758000104B20791A88ADF800209B780E4A8DF8B0
:10759000023069461EF0DCFA0C4B984201D00C48D0
:1075A000C4E720791EF08CFA02B0BDE8F08700BF76
:1075B0001846012014210800A4640120292906008E
:1075C000040003076CEF0700BDD102000000AD0B03
:1075D00000200800746C01205066012010B504469C
:1075E0000079FF2821D01EF049FA20791EF034FBE3
:1075F0002046F5F787F9002802DA002018F0C4FFCA
:107600000A4B002243F82020207924F069FD084A23
:10761000FF2323711378013BDBB213702BB9054BA9
:10762000BDE8104018681EF0E9B910BD18460120E9
:10763000746C01205066012008B5836893B102691B
:107640001279C3F86025043036F059F8064A1378E9
:10765000013BDBB213702BB9044B1868BDE808403E
:107660001EF0CCB908BD00BF756C01205466012026
:107670002DE9F04F85B000259DF838B004460F463F
:107680009246A94698461BB9022005B0BDE8F08F86
:107690000DF10D020DF10E01184603F035FF002823
:1076A000F2D0BDF80E309DF80DC0414801932A4636
:1076B00050F8046BD6F8001511F001036CD0BBF143
:1076C000000F64D1D6F808E5019B9E455FD1D6F83E
:1076D0000C3563455BD15B4603F5AC7E56F82EE076
:1076E000BEF1FF3F50D101F001054FFA83F966600A
:1076F000002E5BD0237AE76069F3060323723879A2
:10770000FCF75EFD237AC4F814806BF3C713237271
:10771000E368187942F0D2FF63680022C3F80025BD
:10772000FDB96368234A93420CD002F5A04293420C
:1077300035D002F58052934233D002F53042934265
:1077400031D10325E8B224F019FE63689DF80D10CD
:10775000C3F80C15BDF80E200021C3F80415C3F8BA
:107760000825237A6268397903F07F0303F5AC7347
:10777000204642F8231063680122C3F800255146D1
:1077800035F0D2FF002080E70133042BA4D1013271
:10779000042A8DD10026AAE799461D46A7E70125B0
:1077A000D0E70225CEE74FF0FF35CBE706206CE7A8
:1077B000AC14090000C0014030B40B4B0B4C00224C
:1077C00054F8041B45688D4208BF197802F1010284
:1077D00004BF01311970042A03F10103F0D1C36819
:1077E00030BC187935F029BF646C0120AC14090055
:1077F00008B5072817D8DFE800F01804060A0D0FAF
:10780000111443F06BFF40F2893011F0EBF8074898
:1078100018F012FF0648FBE70648F9E7064818F09B
:10782000E5FE0648FBE70648F9E708BD0603080041
:10783000CD230800B420080014210800002008000F
:107840001B0108002DE9F0410446D0F8840030B156
:107850001EF0F8F81EF0D2F80023C4F88430284B4C
:1078600094F8B7701A6804F11406964204BF002217
:107870001A60002504F18C08AF4235DC94F8B8702A
:10788000002504F1AA08AF4234DC04F1B4003BF057
:1078900070F804F1B5003BF06CF804F1B6003BF071
:1078A00068F8636A93B1304631F09EFFA06B18B15F
:1078B00035F063FF0023A363E06D18B135F05DFF81
:1078C0000023E365606A08B135F057FF702200219C
:1078D00030463BF0B5FFA06835F04FFF0023C4E908
:1078E0000033A360BDE8F08108EB05003BF041F8F0
:1078F0000135C1E708EB05003BF03BF80135C2E775
:10790000700A01202DE9F04F012685B0044680F869
:10791000BB60D0F884000D461EF094F81EF014FBF6
:10792000002D00F0858004F108013246284665608C
:10793000019114F041F90199606803223CF04BFD7C
:10794000002814BFC82348232361606815F0BEFFD8
:10795000B4F88820E168013AB2400023324314F0C1
:1079600035F904F114067022002130463BF068FF1F
:1079700094F8BD2094F9BE300AB15B425BB2D4F8F2
:107980008490002B08BF0123B9F1000F00F0A682FC
:1079900094F8B750B4F88A8084F87B300627B5FB9A
:1079A000F7F594F8B87094F8B50094F8B9E094F845
:1079B000B4C094F8B61094F8BC20A4F87080052DDB
:1079C00028BF0525052F28BF0527002BB8BF5B4220
:1079D00084F8765005EB4505DBB26D0013FB08F328
:1079E000EDB24FF0000884F84800C4F81490A4F8F1
:1079F000723084F879E084F8777084F875C084F880
:107A0000581084F87C20C4F85C80C4F8388028467C
:107A100035F0A8FE606218BB02252046FFF712FF72
:107A2000022D00F05582032D00F04F8243F056FEE8
:107A3000A06835F0A2FE606A35F09FFEE06D35F07B
:107A40009CFEA06B35F099FEB4F88800656035F0B7
:107A500089FEB4F88830E360C823A060236180E722
:107A6000380135F07FFE8146E06500285AD004F1E8
:107A70008C01606A2A463BF0A3FE04F1AA0143464A
:107A8000DAB2974246D8C14BD4F884001E601DF08C
:107A9000D9FFBF4ABF491EF005FA636A002BBBD06D
:107AA00094F87530039303A81DF0D6FE0025804698
:107AB0002F464FF0010994F876105FFA85FA01EB32
:107AC0004103BAEB430F33DB17F07F4F14BF08239A
:107AD000002317F47F0F18BF43F00403FAB217F422
:107AE0007F4F18BF43F002030AB143F00103013B8B
:107AF00001250B2B00F23981DFE813F02F002F0056
:107B000033012F003701370137012F0037013701CB
:107B100037013301E26D11F8010B02EB031201335F
:107B20001073ADE7606A35F028FEC4F8249073E75F
:107B3000636A03A813F80A3003931DF08DFE804595
:107B400005F1010540F0CC81636A13F80A3003F0B7
:107B50001F0309FA03F31F43ADE784F8745094F848
:107B6000773094F8792094F8740005FA03F3B4F8A8
:107B7000725084F87A300735DBB205F4FF655D4357
:107B8000554394F87C304543256603B16D0011FBE5
:107B900000F1062000FB015035F0E4FD0346A06330
:107BA00000283FF439AF2B44A3622A4600213BF062
:107BB00047FE94F8740094F87530012840F0EC808A
:107BC000626A03F01F03127800FA03F3C2F3C102E2
:107BD000E3623B43236384F87820002394F8762003
:107BE0005F1C02EB4202DBB2B3EB420FC0F2BF807C
:107BF00094F8791094F87A204FF47A43B3FBF2F3B7
:107C000001228A40013AB3FBF2F3632B40F20A816E
:107C1000A366A36E6366002594F8483084F87E500E
:107C200003A803931DF018FE00F5A16094F84830F6
:107C3000E06303A803931DF00FFE94F8483001277A
:107C400003F01F0307FA03F300F20C50206463648F
:107C500003A894F8583003931DF0FEFD00F5A160D1
:107C600094F85830E06403A803931DF0F5FD94F8F0
:107C7000583003F01F039F4000F20C5094F8753009
:107C80002065676503A803931DF0E6FD039B03F5DC
:107C9000E07340F2033740F8237094F8750042F027
:107CA0002EFD94F84830039303A81DF0D5FD039BE7
:107CB00003F5E07340F8237094F8480042F01FFD8C
:107CC00094F85830039303A81DF0C6FD039B03F5F9
:107CD000E07340F8237094F8580042F03AFD94F8AD
:107CE000763005F1010803EB4303EDB2B5EB430F2A
:107CF000C0F29A8094F87730012505FA03F3023B2D
:107D0000DBB284F881300027A84640F2033994F8AA
:107D10007720FBB29A4200F2988094F87530039372
:107D200003A81DF099FD00F5A16094F87530A061DD
:107D300003A803931DF090FD00F20C50E061304663
:107D4000F3F70CFBB4F88A20A168304631F04DFA05
:107D5000304631F082FD002384F8BB3005B0BDE829
:107D6000F08F022384F87430F9E60423FAE7D4E9AB
:107D70000921D25C94F8785002F01F0200FA02F256
:107D8000ED00EA40CA543B4628E700BF700A0120D4
:107D9000FDC30500CC2B090003F01F03012101FAEC
:107DA00003F3022847EA030721D1626A1278C2F37B
:107DB0000012C4E90B3784F87820002394F8762069
:107DC0005F1C02EB4202DBB2B3EB420FBFF610AF17
:107DD000D4E90920D25C94F8785002F01F0201FA2D
:107DE00002F22D01EA4020F813203B46E6E700228C
:107DF000C4E90B3784F87820134694F876205D1C8C
:107E000002EB4202DBB2B3EB420FBFF6F1AED4E9B4
:107E10000920D25C02F01F0201FA02F240F823208E
:107E20002B46EAE76423F3E6636A03A85B5D0393EA
:107E30001DF012FD039B03F5E07340F82370636AA5
:107E4000585D42F05CFC454649E7D4F85CB04FEA27
:107E5000031A0BEB031303A81B7B03931DF0FCFC1D
:107E600000F5A1604BF80A00E36D03EB0A0B03A8D1
:107E70009BF80C3003931DF0EFFC00F20C50CBF894
:107E80000400E26D524403A8137B03F01F0308FAB9
:107E900003F39360E36D53441B7B03931DF0DCFC01
:107EA000039B03F5E07340F8239094F881302B4254
:107EB000E36D5344187B05D042F04BFC6D00EDB2EE
:107EC000013724E742F01BFCF8E73D2010F08AFD63
:107ED000044905484FF402723DF028FB03259CE558
:107EE00001259AE57B020800A0F40700F7B50171AF
:107EF00013794371194B43F821001646427943F830
:107F00002200174B1A88ADF804209B78154A8DF88B
:107F1000063004460D46007901A91DF019FE124BEA
:107F20009842074602D0114818F060FB0D4A60796C
:107F300001A91DF00DFEB842207902D01DF08CFE83
:107F4000F1E71DF0BDFD60791DF0BAFD2846FCF794
:107F500037F93079FCF734F903B0F0BD3846012029
:107F6000B8EF0700ADC902000000AD0B002008000B
:107F700010B50179FF2904461BD00E4B002243F8AF
:107F80002120417943F8212000791DF077FD6079A7
:107F90001DF074FD20791DF05FFE60791DF05CFE20
:107FA000207924F09DF8607924F09AF84FF6FF7359
:107FB000A38010BD3846012010B50446002021F0F2
:107FC0002DFE054A830A506843EA8153184421462E
:107FD000BDE810402AF000BDBC6C012008B5014886
:107FE00018F02AFB6322080010B50E4B02689A4273
:107FF000044615D1406804F10803984201D135F0D8
:1080000024F8A06935F0A9FBE069F6F7E5FA0AF073
:10801000F5FB20463422BDE8104000213BF010BCA7
:1080200010BD00BFE4950800F0B50D4697B00021E3
:108030000746102016463BF0FCFA04460560284629
:1080400045F058F900239E42E36014BF3E231E23EF
:1080500001931E23C4E9010702931749206845F0E4
:1080600020F858B103A842F0D8FA38B9284635F0BC
:1080700002FB1DF0D5FB112018F09AFA03A928463F
:1080800019F02EF8012807D96368012B02D0436844
:10809000012B01D00120EFE701AB022240F22C417D
:1080A00020463DF064FD054BD3F8E420E260C3F8C0
:1080B000E44017B0F0BD00BF5BB30800C061012011
:1080C00070B5104A1346014653F8E40F10B9162054
:1080D00018F06EFAD0E902548D420FD11C60D2F82C
:1080E000E030984202D10023C2F8E0300023BDE81E
:1080F00070401A4640F292513DF039BD00F10C0338
:108100002046E3E7C06101202DE9F74F99460C9B1B
:108110004360044688460420002117463BF089FA54
:108120004FF48033636148F28002002320616FF0D6
:10813000404B03804280ADF80230ADF8003001932F
:10814000019DBD4211D36A460DF10201204645F062
:108150002CFBBDF80000400080B2A08100213BF064
:1081600068FAA06003B0BDE8F08F08EB05030026B5
:1081700013F8011B01F07F0009062A4640EAC616E3
:1081800005F1010558D5BD42F2D10195284648E0D8
:1081900001AA3946404642F0BBFDE38A03EB0B02DD
:1081A000236903EB820305469E7893F803A0B0424F
:1081B00001D05045C4D16A460DF10201204645F078
:1081C000F4FAB5424FF0800220D15146204632F0F9
:1081D000E3F9B5E701AA3946404642F099FDE38A42
:1081E00003EB0B02236903EB82030546DA78802A4E
:1081F000A6D19E786A460DF10201204645F0D5FAD7
:10820000802E02D132462946E0E72A463146DDE794
:1082100001AA3946404642F07BFD91E7B84202D3BD
:10822000019823F07DF818F900300332002B0192F9
:1082300086DAF5E7019783E70C9B5E43BDF80230D1
:10824000B6FBF9F61E4418F80530ADF802601B09BC
:10825000901C083B0190072BE3D801A151F823F0B3
:1082600091810300D5810300118203001182030074
:108270001D8203001D82030011820300358203006A
:1082800013B500230DF107008DF8073021F0C6FC6F
:108290000A4CA0FB0432400840EAC17004FB0122F2
:1082A00018189DF8073042EB510147F236725343DC
:1082B000C01841F1000102B010BD00BFB2E60E00CF
:1082C00070B5184B1A7812F0010204460D4625D1FC
:1082D000154B164E1870002842F65671144808BF08
:1082E0000E2614F0E9F900B146601CB10F4B0022D4
:1082F0001A7301240F4B0E480F4E1D70002D4FF0C6
:10830000000243F2860108BF0E2614F0D5F900B131
:1083100046602DB1084B1C73284670BD0025FBE755
:108320000125F9E7306B01208C6C012084040120C9
:10833000A80401208D6C0120940401202DE9F34153
:108340000F461946054614461E463AF099FC284445
:1083500040F2BA4290F84610204610F0C1FB45F0BA
:10836000BBF810F5FA6841F1000545F0B5F8404555
:1083700071EB050306D32BF069FA50B919491A4875
:108380003DF0C9F82BF062FA0028F4D1F8F7A8F80C
:10839000EBE7164D68782DF079FD08B91449EEE742
:1083A000A6B13F2C28BF3F2422462E72394605F144
:1083B000090001343BF004FAE2B20E4968782DF06E
:1083C0008FFE0028EAD002B0BDE8F081402C2246A2
:1083D000394628BF402205F1080001923BF0F0F930
:1083E000019AEAE7B60A0800FC2D0800F02F0120E8
:1083F000EB0A0800F82F0120F8B5174B1C7814F091
:10840000010406460D4624D115F0CAFF11284FEA93
:10841000600303DD1148082118F016F9104F3B6086
:10842000104B1D70104D3B689C4203DB2DF01AF978
:108430000120F8BD6100042241F00101304617F02F
:10844000A1F85822014628463BF0BAF901345835C4
:10845000E9E70020EDE700BF306B01207005080060
:108460009C6401204E6C01201C5B012008B5014872
:1084700018F0CEF8750F0800F0B585B0DDE90B7681
:10848000044601AD85E80E00384640F2CD5126F095
:1084900065F93046A78240F2D25126F05FF995E89F
:1084A00007000A9B2361231DE68283E807003D4BFA
:1084B000A361238CA3830023636204F128060123B4
:1084C00084F834303146A3689847A269E08A977BE4
:1084D00092F90410B2F800E092F90550A38AB2F8BC
:1084E00002C0002F3ED010FB01F715FB03F57744C7
:1084F000654400293FB22DB208DCB4F92E30618DFD
:10850000C3F10103C1F101016185E38592F90530F1
:10851000002B08DCB4F92C30228DC3F10103C2F129
:1085200001022285A385B4F92A30228D6285238534
:10853000A28DB4F92E30A385E285304637F0A6FA35
:10854000238D13FA87F32385638D13FA85F36385EF
:10855000A38D13FA87F3A385E38D13FA85F5E585DB
:1085600005B0F0BD13FB01F315FB00F57344654442
:1085700000291FB22DB207DC238DC3F1010323852F
:10858000A38DC3F10103A38592F90530002BD4DC40
:10859000638DC3F101036385E38DC3F10103E385BB
:1085A000CBE700BF9005012010B5037A022B0446EB
:1085B00006D1074BD3F884314BB1064818F016F8B2
:1085C000054B1B680BB12AF09DF90023237210BDE7
:1085D000C06101205C0C08005866012070B515468A
:1085E000C2072DED028B04460E4609D4830703D142
:1085F0000268194B9A4203D0204615F061FED8B1AB
:10860000204615F0CBF83046B0EE408A15F0C6F89B
:108610002846F0EE408A15F0C1F8B4EEE88AF1EE93
:1086200010FA17D4B4EEC08AF1EE10FAD8BF25467E
:10863000BDEC028B284670BD29460222204600F080
:1086400037F8BDEC028B014603223046BDE870408E
:1086500000F02EB83546EBE7B4F607007FB50646C6
:108660000D4600F025F80446F00709D4B10703D100
:1086700032680E4B9A4203D0304615F021FE90B17D
:10868000EA0709D4AB0703D12A68084B9A4203D002
:10869000284615F015FE30B16946204613F0F0FA71
:1086A00013F07EFC0446204604B070BDB4F607000B
:1086B0002DE9F04F0C4689B0002191461AF0D6FD05
:1086C0000021834620461AF0D1FD4FF00008824673
:1086D000414608208DF81F803AF0ABFF41460590D7
:1086E00008203AF0A6FF4146074608203AF0A1FFCD
:1086F000059BCDE9007006460DF11F025146584614
:1087000041F052FC059B10B9B54817F095FFB9F13F
:10871000000F0CD10222CDE9016200979DF81F20C5
:10872000514658463EF01FF809B0BDE8F08FB9F148
:10873000010F01D10522EEE79BF80420DBF81C5065
:10874000DAF81C40422A40F0B4819AF80420422A08
:108750004ED119469DF81F0041F0D9FDB9F1020F25
:10876000C36922D14FF0000E227829788A4228BFAF
:108770000A461A708269D0F810C0D6F804901344E3
:108780000EF1010E7A68F44515444C44ECD8396872
:108790000CFB121132680CFB19221444C26808F158
:1087A000010842450D44DDD8BEE74FF0000E2278A7
:1087B00029788A4238BF0A461A708269D0F810C0F8
:1087C000D6F8049013440EF1010E7A68F44515446E
:1087D0004C44ECD839680CFB121132680CFB19229E
:1087E0001444C26808F1010842450D44DDD89BE7F6
:1087F000622A51D119469DF81F00682241F087FD79
:10880000B9F1020FC36923D14FF0000E94F9002093
:1088100029788A42A8BF0A461A808269D0F810C017
:10882000D6F8049013440EF1010E7A68F44515440D
:108830004C44EBD839680CFB121132680CFB19223E
:108840001444C26808F1010842450D44DCD86BE7C6
:108850004FF0000E94F9002029788A42B8BF0A46EA
:108860001A808269D0F810C0D6F8049013440EF133
:10887000010E7A68F44515444C44EBD839680CFB7A
:10888000121132680CFB19221444C26808F1010865
:1088900042450D44DCD847E7482A4ED119469DF899
:1088A0001F0041F034FDB9F1020FC36922D14FF02E
:1088B000000E228829788A4228BF0A461A808269D7
:1088C000D0F810C0D6F8049013440EF1010E7A6867
:1088D000F44515444C44ECD839680CFB121132684D
:1088E0000CFB19221444C26808F1010842450D44EA
:1088F000DDD819E74FF0000E228829788A4238BF68
:108900000A461A808269D0F810C0D6F80490134441
:108910000EF1010E7A68F44515444C44ECD83968E0
:108920000CFB121132680CFB19221444C26808F1C6
:10893000010842450D44DDD8F6E6682A52D11946B1
:108940009DF81F0041F0E3FCB9F1020FC36923D188
:108950004FF0000EB4F9002029788A42A8BF0A46D9
:108960001A808269D0F810C0D6F8049013440EF132
:10897000010E7A68F44515444C44EBD839680CFB79
:10898000121132680CFB19221444C26808F1010864
:1089900042450D44DCD8C7E64FF0000EB4F9002084
:1089A00029788A42B8BF0A461A808269D0F810C076
:1089B000D6F8049013440EF1010E7A68F44515447C
:1089C0004C44EBD839680CFB121132680CFB1922AD
:1089D0001444C26808F1010842450D44DCD8A3E6FE
:1089E000F61A0800662A40F0F1879DF81F00194624
:1089F00041F08DFCB9F1020FD0F81CA04FF000023D
:108A00002BD14FF000082B78D4ED007A07EE103A06
:108A1000F8EEC76A08F10108F4EEE76AF1EE10FA21
:108A200048BFF8EE477ACAED007A8169D0F810C0E5
:108A3000D6F804908A447968C4450D444C44E2D881
:108A40003B680CFB113E31680CFB19110C44C168EA
:108A5000013291427544D4D866E64FF000082B7875
:108A6000D4ED007A07EE103AF8EEC76A08F1010873
:108A7000F4EEE76AF1EE10FAC8BFF8EE477ACAEDF5
:108A8000007A8169D0F810C0D6F804908A447968D9
:108A9000C4450D444C44E2D83B680CFB113E3168A0
:108AA0000CFB19110C44C168013291427544D4D8B1
:108AB0003AE6622A40F0C2819AF80420422A51D153
:108AC00019469DF81F00682241F021FCB9F1020F00
:108AD000C36923D14FF0000E227895F900108A4225
:108AE000A8BF0A461A808269D0F810C0D6F8049050
:108AF00013440EF1010E7A68F44515444C44EBD84A
:108B000039680CFB121132680CFB19221444C2683C
